:020000040800F2
:1000000000200010F1D60208B1620208D54B0008AA
:10001000AD620208A9620208A562020800000000A1
:10002000000000000000000000000000A1620208C3
:100030009D62020800000000996202084110000859
:1000400059D7020859D7020859D7020859D70208C8
:1000500059D7020859D702089D250008C92600086B
:100060008D2600085126000815260008453A00088C
:10007000353A0008253A0008153A0008053A000804
:10008000F1390008DD39000859D7020859D70208AC
:10009000E566020859D7020859D70208D925000891
:1000A0001152000841520008015200085152000844
:1000B000315200082152000859D7020859D70208C6
:1000C00059D7020859D7020859D7020859D7020848
:1000D00059D702086D110008F110000875100008CA
:1000E0006125000859D702088962020859D7020819
:1000F00059D7020859D7020859D7020859D7020818
:1001000000000000000000000000000059D70208B5
:1001100059D7020859D70208693101084D31010841
:10012000C9390008B5390008A13900088D3900081F
:100130007939000859D702080000000000000000CB
:1001400059D7020859D7020859D702080000000001
:10015000000000000000000000000000000000009F
:10016000000000000000000059D7020859D702081B
:1001700059D7020800000000000000000000000045
:080180000000000059D702083D
:1001880070B4EFF31186502383F31288436B1A6817
:10019800D20720D45D686DB9446A826A944217D048
:1001A80081691144D9600ED9A21A5A60846200226A
:1001B80080F850201A6842F00102F1B21A6081F307
:1001C800118870BC704701698A1A5A608562EEE727
:1001D800012380F85030F1B281F3118870BC704768
:1001E800436A8269D154436A0169426B01338B4285
:1001F80028BF00234362002A2FD0EFF31181502338
:1002080083F31288436B1A68D2072CD470B45E68E3
:100218006EB9456A826A954217D084691444DC60D5
:100228000ED9AA1A5A608562002280F850201A68EE
:1002380042F00102C9B21A6081F3118870BC70479C
:100248000469A21A5A608662EEE7012380F85030EA
:10025800C9B281F3118870BC7047C26C136843F04F
:10026800800313607047C9B281F31188704700BFDB
:10027800026B10B462B1036CC2684469D11A013BC5
:10028800615C5DF8044B08BF13460364C8B270474D
:10029800016A4369C4685B5C0131A14228BF114609
:1002A80001625DF8044BD8B2704700BF436B13B1CD
:1002B80090F850007047836A406A181AB0FA80F0C4
:1002C80040097047416A836A99420AD3CB1A416B45
:1002D800026961B14968501E0B4483420AD2C01AB0
:1002E800704702691144CB1A416B0029F2D1501EA4
:1002F800C01A704700207047036B43B1026C5B68FB
:1003080093422FBF981AC0689B1AC0187047C269D9
:10031800036A9A422FBFD01AC0688018C01A704763
:100328000A4B30B503F1140493F900205D78072ACD
:10033800C8BF143A811804330D7313F8025C85544E
:1003480013F8012C0A76A342EED130BD3C02030813
:1003580003682DE9F041DF691FB13B46BDE8F04174
:100368001847002A164611DD04460D460E4400E0E3
:1003780023689B68204698470028F9D0236815F819
:10038800011B1B6820469847AE42F1D1BDE8F081B9
:1003980000232522027043708370C37070472D2399
:1003A80043702E2303712F23C371704740F2E93342
:1003B80000E09BB10289013B12F0020F9BB2F8D01A
:1003C800017340F2E93300E043B10289013B12F0C6
:1003D800010F9BB2F8D0007BC0B27047064B984221
:1003E80001D0FF207047054A538B01339BB25383DA
:1003F800508BC0B2704700BF003800400065002035
:1004080030B4836813B11C689B882385436840F225
:10041800E93401E0002C3FD01D89013C15F0020FA2
:10042800A4B2F7D0197303F10C0540F2E93101E0E9
:1004380000293BD01C89013914F0010F89B2F7D08B
:100448002B78436840F2E93100E0D9B11C890139C1
:1004580014F0020F89B2F8D01A7303F10C0440F2B9
:10046800E93200E072B11989013A11F0010F92B234
:10047800F8D02378836813B11A689B8893610120A8
:1004880030BC70470F4A9342F4D10F4A538B013363
:100498009BB25383538BEDE70A498B42D2D10A4C66
:1004A800618B013189B26183618BCBE705498B424E
:1004B800C7D105494B8B01339BB24B834B8B4368A8
:1004C800C0E700BF0038004000650020F0B4848910
:1004D8004FF6FF764FF47A740BB300292ED00F78BD
:1004E800013101E0B44217D00589013CAD07A4B23F
:1004F800F8D507734FF47A7402E0BCB2B4420BD05B
:100508000589ED0704F1FF37F7D5057BEDB20AB190
:1005180015700132013BDFE7094B984202D00120F8
:10052800F0BC7047074A538B01339BB25383508BFF
:1005380080B2003018BF0120F0BC7047FF27D3E716
:10054800003800400065002070B50646806810B18C
:1005580004688088208541F08001706840F2E934A1
:1005680000E0F4B10589013C15F0020FA4B2F8D0FF
:10057800017300F10C0540F2E93100E0D9B10489BA
:10058800013914F0010F89B2F8D029787068002178
:10059800FFF79CFFB36813B11A689B889361012029
:1005A80070BD0A498842F2D1094C618B013189B288
:1005B8006183618BEBE705498842E7D10448418BA9
:1005C800013189B24183418B7068E0E7003800400F
:1005D80000650020002870B51EDB0928044620DDD0
:1005E800012303EB83035B00B0FBF3F2092AF8D87D
:1005F8007BB10E4EB4FBF3F00928CCBF5722302252
:10060800A6FB03E5024403FB1044EB0801F8012BA9
:10061800F0D100230B7070BD2D230B7040420131C7
:10062800DBE7303001F8010BF3E700BFCDCCCCCCD1
:10063800884230B44FF001042ED301FB04F4B0FB20
:10064800F4F58D42F9D284B1AAB901E0B0FBF4F512
:10065800092DCCBF572230222A4404FB150003F889
:10066800012BB4FBF1F4002CF0D100221A7030BC3D
:100678007047B0FBF4F5092DCCBF372230222A444D
:1006880004FB150003F8012BB4FBF1F4002CF0D1A6
:1006980000221A7030BC70470546002AEBD1D7E714
:1006A80003685A1C02601970704700BF2DE9F047B3
:1006B800089C2578002B804689460CBF4FF0200AFD
:1006C8004FF0300A661C35B3002A29DD334601E0B5
:1006D800024698B113F8011B501E0029F8D1971E45
:1006E80060B13D46013D51464046C8476B1C002B52
:1006F800F8DC257827EAE770013055B1041B294654
:100708004046C847301916F8015B002DF7D1BDE8FF
:10071800F087BDE8F087002A04DC2846BDE8F087AA
:100728000020EBE7571EDCE783684268D0ED037AC8
:1007380000EB83010133934281ED040A836004BF17
:100748000023836000EB830393ED047A036870EE63
:10075800277A9A42C0ED037A77EEC77AC0ED037A1A
:100768000CDA013307EE103AF8EEC76AB7EE007AF2
:1007780087EEA60A036030EE070A704707EE102AD4
:10078800B8EEC77A87EE870A704700BF90ED057A02
:1007980090ED004AD0ED066AD0ED014AD0ED047A1A
:1007A80090ED035AD0ED025AA4EE007AB0EE406AFA
:1007B800B0EE470AB0EE667AA6EE247A67EEC07A03
:1007C800A0EE457AE6EE257A80ED057AC0ED067A48
:1007D800704700BFD0ED057A90ED013AD0ED003AB0
:1007E800D0ED064A90ED024A90ED077A90ED035A53
:1007F80090ED086AD0ED045AC0ED067AF0EE406A32
:1008080027EE830AC0ED056AA3EEA60A80ED087AF2
:10081800A4EE240AA5EE470AA5EEC60A80ED070A4B
:10082800704700BFD0ED007A90ED017A30EE670A8C
:10083800E7EE007AB0EE670AC0ED007A704700BFB5
:10084800704700BF0A44914214D030B40139551E94
:1008580041F2210211F8014F082380EA0420040420
:100868004CBF82EA40004000013B80B2F7D18D4284
:10087800F0D130BC704700BF4FF48053838270477B
:1008880090F8203033B1012B03D14FF400638382F9
:10089800704770474FF480638382704770B5044691
:1008A80082B01430E56D06236A464321A847B0B1EB
:1008B8009DF804009DF800609DF801109DF8025015
:1008C8009DF803209DF8053041EA062143EA0023FC
:1008D80042EA0522A187E287A4F84030012002B04D
:1008E80070BD00BF70B5044682B00830656A062343
:1008F8006A463B21A847A8B19DF804009DF800600E
:100908009DF801109DF802509DF803209DF80530D0
:1009180041EA062143EA002342EA0522E1822283D2
:100928006383012002B070BD50F8043C012280F8B6
:100938004520103803B11847704700BF10B490E83D
:100948000600047B40690223A3404B6013685DF8EE
:10095800044B4FF6FE710B40136011E470B4046849
:10096800037B2268022101FA03F31A4213D0426979
:100978000A49582000FB02124FF6FE765068528949
:10098800C5680068296831402960C168D24392B2BD
:100998000A40C260636070BC704700BFB85D002049
:1009A80030B4094B1C7864B1084B002503EBC40430
:1009B8001A6899885562D06808330143A342D16008
:1009C800F6D130BC704700BF786000207C60002002
:1009D80010B40268047B11680223A340194209D0AD
:1009E8000649406800240C7001684FF6FE742140E7
:1009F800016053605DF8044B704700BF57510020F9
:100A0800F0B4334C00EB800004EB80046468002CE5
:100A18005BD0304E49004FF42040CDB23060A16920
:100A2800090444D460682C4F45F08071384041F483
:100A3800903101434FF420406160306003E0411E73
:100A4800002838D00846A1698F07F8D54FF4204010
:100A5800A262306002E0421E68B31046A269110625
:100A6800F9D562681C4945F0007545F480350A409F
:100A780015434FF420406560306002E0421ED0B15B
:100A88001046A2699207F9D5A362A3694FF42040E2
:100A98009B06306005D4431E68B11846A3699B06BF
:100AA800F9D520233060E3610120F0BC7047411E76
:100AB80008B10846B3E7094A138801339BB24FF0DF
:100AC800FF3131601380F0BC70472046F0BC70479E
:100AD800D0640020F8640020009800FCFC6400202A
:100AE800134601200A4668218AE700BF30B504464C
:100AF800C06C61710368A26823F00103036087B0CA
:100B0800A379009213F004023DD04FF4805213F001
:100B18000203019244D102934FF4806300220393AD
:100B280011F00103059237D1049308238D07694614
:100B380048BF049325F020FD6079E36CA17900F0AB
:100B48000202002A15BF4FF440324FF480324FF4AE
:100B58000034002410F0010F586808BF2246CC0763
:100B68004CBF024320EA02025A609A6809074CBF48
:100B780042F0080222F008029A601A6842F0010264
:100B88001A6007B030BD13F0020301920BD04FF486
:100B9800005513460295C1E7042304930C23C5E7C7
:100BA8004FF40053B7E70293B8E700BF10B5044607
:100BB800C06CA160036823F001030360A37986B0C9
:100BC80013F00402009141D04FF4805213F0020355
:100BD800019244D102934FF4806362790393D10761
:100BE8004FF000030493059345BF0423049308239F
:100BF8000C236946920748BF049325F0BDFC607931
:100C0800E36CA17900F00202002A15BF4FF44032CC
:100C18004FF480324FF40034002410F0010F58686C
:100C280008BF2246CC074CBF024320EA02025A60A2
:100C38009A6809074CBF42F0080222F008029A603D
:100C48001A6842F001021A6006B010BD13F00203E0
:100C5800019207D04FF4005113460291BDE74FF4BB
:100C68000053B7E70293B8E70023192203604270E4
:100C78001A22C270012243604271C37170472DE984
:100C8800F341056906460F467DBBD0F80080C8F3DE
:100C98000A0323B30023D6F8008001931BF03CFE1F
:100CA800042819D1214C236943F001032361BBB205
:100CB800A8F800301BF030FE04282ED108F10203FA
:100CC8000193019B3F0C1F801BF026FE236904281B
:100CD80023F00103236125D06FF0010505E01BF027
:100CE8001BFE042805D04FF0FF35284602B0BDE8AA
:100CF800F0810E4C236943F002032361C4F8148089
:100D0800236943F0400323611BF006FE236904288E
:100D180023F002032361BDD0E5E7236923F0010333
:100D28002361D9E7336804333360DEE700200240EB
:100D3800F8B504460D468E180027B54201D1206942
:100D4800F8BDE368591CE160234415F8012B1A72B9
:100D58000429F2D1A1682046FFF791FFE7602061DE
:100D6800EBE700BF70B582B004466946143022F044
:100D7800ADFAB0B19DF805009DF801609DF802102C
:100D88009DF803509DF804209DF8063041EA06219D
:100D980043EA002342EA0522A187E287A4F840300B
:100DA800012002B070BD00BF0846194629F0E6B917
:100DB8002DE9F04FDFF830C1474A4849484E494DC0
:100DC8008046102718F1FF38C0F08480DCF8043022
:100DD800C3F30803002B5CD1EFF31183002B58D128
:100DE8000B68946800BF08688342F9D1D6F8009070
:100DF8004FF47A7000FB09FEAEEB040EBEFBF9FE61
:100E080000FB03EEDCF80430C3F308034FF47A74F4
:100E18000120FBB9EFF31183E3B90B68D2F808A0FE
:100E280000BFD1F800904B45F7D1D6F800B004FBCD
:100E38000BF9A9EB0A09B9FBFBF904FB0393A3EB34
:100E48000E03B3F57A7FBDD2DCF80430C3F3080390
:100E5800002BDFD0EFF3118A87F31288D2F808B09D
:100E68001368DB0344BF2860D2F808B00B68D5F8D4
:100E780000905FFA8AFA8AF31188D6F800A099449C
:100E880004FB0AF3A3EB0B03B3FBFAF304FB0933EC
:100E9800D5E7EFF3118487F31288D2F80890136826
:100EA800D80303D501232B60D2F808900B68286873
:100EB800E4B284F31188D6F800A04FF47A7400EBFA
:100EC800030E04FB0AF3A3EB0903B3FBFAF304FBD9
:100ED8000E3E97E7BDE8F08F10E000E06C57002069
:100EE800705700206857002000ED00E0204B5B6839
:100EF800C3F3080330B4BBB9EFF31183A3B91D4B97
:100F08001D4C1868A16800BF1A689042F9D11B4BA4
:100F18001C684FF47A7202FB04F3591AB1FBF4F11E
:100F280030BC02FB00107047EFF31182102383F3EB
:100F3800128811498C680B6813F4803F104B02D05B
:100F4800012018608C680B49D2B20D68186882F3CA
:100F580011880A4B19684FF47A72284402FB01F38E
:100F68001B1B30BCB3FBF1F302FB0030704700BF22
:100F780000ED00E06C57002010E000E07057002002
:100F8800685700202DE9F84F8046FFF7AFFF254E40
:100F98002549DFF8A0E0254A254D844610274FF45F
:100FA8007A740120DEF80430C3F30803D3B9EFF3F1
:100FB8001183BBB90B68D2F808A000BFD1F8009024
:100FC8004B45F7D1D6F800B004FB0BF9A9EB0A0999
:100FD800B9FBFBF904FB0393A3EB0C034345E1D3F3
:100FE800BDE8F88FEFF3118A87F31288D2F808B0BA
:100FF8001368DB0344BF2860D2F808B00B68D5F843
:1010080000905FFA8AFA8AF31188D6F800A099440A
:1010180004FB0AF3A3EB0B03B3FBFAF304FB09335A
:10102800DAE700BF705700206C57002010E000E09E
:101038006857002000ED00E030B4EFF31183102270
:1010480082F312880649074C0A68074801320025CE
:101058000A602560DBB2026883F3118830BC7047F0
:101068006C5700206857002010E000E01D4B70B559
:101078009C68E36C226BDD69C2B1636B2BB12B07F3
:1010880002D5E36C08221A6270BD2A06F7D5A26A57
:10109800616A8A421FD0511CA069A162825C2069E2
:1010A800E66C81423285EAD3A362E8E7A906E4D573
:1010B800E26A1AB1988C80B29047DEE7E1699B8CAE
:1010C8006069DBB24E1CE6614354E169E36899420A
:1010D80028BFE261D1E7E26C136823F08003136054
:1010E800CDE700BF843100201D4B70B55C68E36C10
:1010F800226BDD69C2B1636B2BB12B0702D5E36CA0
:1011080008221A6270BD2A06F7D5A26A616A8A4265
:101118001FD0511CA069A162825C2069E66C8142E3
:101128003285EAD3A362E8E7A906E4D5E26A1AB1F0
:10113800988C80B29047DEE7E1699B8C6069DBB2EE
:101148004E1CE6614354E169E368994228BFE261B5
:10115800D1E7E26C136823F080031360CDE700BF8A
:10116800843100201D4B70B51C68E36C226BDD696F
:10117800C2B1636B2BB12B0702D5E36C08221A624C
:1011880070BD2A06F7D5A26A616A8A421FD0511C2F
:10119800A069A162825C2069E66C81423285EAD34B
:1011A800A362E8E7A906E4D5E26A1AB1988C80B28E
:1011B8009047DEE7E1699B8C6069DBB24E1CE66113
:1011C8004354E169E368994228BFE261D1E7E26CE0
:1011D800136823F080031360CDE700BF843100203B
:1011E80003685B6A03B11847704700BF03681B6A4E
:1011F80003B11847704700BF03682DE9F041DF6964
:101208001FB13B46BDE8F0411847002A164611DDDC
:1012180004460D460E4400E023689B682046984724
:101228000028F9D0236815F8011B1B682046984749
:10123800AE42F1D1BDE8F08103689B69184700BF51
:1012480003685B69184700BF0368DB68184700BF7D
:1012580003689B68184700BF03685B68184700BFAE
:1012680003681B68184700BF014B1868F8E700BF00
:1012780058610020054B53F8203033B11A689B8819
:10128800918A0B4218BF1B0493617047385700209E
:1012980003682DE9F04F03F13845644EAD0A012487
:1012A800755D05F01F066D09022D04FA06F400F0BD
:1012B800A280032D00F0A480012D52D08088B0FABE
:1012C80080F4C4F11F04A4B2E50803EB850504F01B
:1012D80007042E6AA4000F27A74026EA07062E62F5
:1012E8002E6A01F0030702FA04F47A1E3443012A35
:1012F800C1F3810CC1F300182C62C1F3411135D937
:10130800C60700F19780850700F1A380440700F124
:10131800B180020700F1BF80C60600F1CD808506C6
:1013280000F1DB80440600F1E980020600F1F78055
:10133800C60500F10581850500F11381440500F11A
:101348002181020500F12F81C60400F13D81850449
:1013580000F14B81440400F15981020455D4BDE8E1
:10136800F08F334D6E6934436C61A7E70024224641
:101378004FF0010E4FF0030904E00132102A04F186
:101388000204ECD00EFA02F636EA0005F5D1D3F8DD
:1013980008A009FA04F5ED430AEA050AC3F808A00B
:1013A800D3F808B00CFA04FA4AEA0B0AC3F808A002
:1013B800B3F804A01FFA8AFA2AEA06069E80B3F850
:1013C80004A008FA02F646EA0A06B6B29E801E682B
:1013D8002E401E60D3F800A007FA04F646EA0A0673
:1013E8001E60D3F80CA001FA04F605EA0A0A46EAD8
:1013F8000A05DD60C1E70E4DAE693443AC615DE7B7
:101408000B4DEE693443EC6158E71A6822F040420C
:101418001A601A6842EA87771F60DA6822F0404249
:1014280042EA8171D960BDE8F08F00BF4026030809
:10143800001002401A6822F003021A601A683A4340
:101448001A60DA6822F003020A438507DA607FF53A
:101458005DAF1A6822F00C021A601A6842EA870225
:101468001A60DA6822F00C0242EA81024407DA6064
:101478007FF54FAF1A6822F030021A601A6842EA04
:1014880007121A60DA6822F0300242EA0112DA60C2
:1014980002077FF541AF1A6822F0C0021A601A6885
:1014A80042EA87121A60DA6822F0C00242EA811220
:1014B800C606DA607FF533AF1A6822F440721A6004
:1014C8001A6842EA07221A60DA6822F4407242EA8D
:1014D80001228506DA607FF525AF1A6822F440629A
:1014E8001A601A6842EA87221A60DA6822F44062AF
:1014F80042EA81224406DA607FF517AF1A6822F4BF
:1015080040521A601A6842EA07321A60DA6822F40E
:10151800405242EA0132DA6002067FF509AF1A68E2
:1015280022F440421A601A6842EA87321A60DA687E
:1015380022F4404242EA8132C605DA607FF5FBAE0A
:101548001A6822F440321A601A6842EA07421A609E
:10155800DA6822F4403242EA01428505DA607FF512
:10156800EDAE1A6822F440221A601A6842EA8742ED
:101578001A60DA6822F4402242EA81424405DA60BD
:101588007FF5DFAE1A6822F440121A601A6842EA40
:1015980007521A60DA6822F4401242EA0152DA600D
:1015A80002057FF5D1AE1A6822F440021A601A6863
:1015B80042EA87521A60DA6822F4400242EA81520B
:1015C800C604DA607FF5C3AE1A6822F040721A606A
:1015D8001A6842EA07621A60DA6822F0407242EA40
:1015E80001628504DA607FF5B5AE1A6822F04062C0
:1015F8001A601A6842EA87621A60DA6822F0406262
:1016080042EA81624404DA607FF5A7AE1A6822F0E4
:1016180040521A601A6842EA07721A60DA6822F0C1
:10162800405242EA0172DA6097E600BF036803F1AC
:1016380038422DE9F04F920A584DAA5C02F01F0576
:1016480052090124022A04FA05F400F08C80032AC6
:1016580000F08E80012A3CD001F003077A1E012A8F
:10166800C1F3810CC1F300188088C1F3411135D949
:10167800C60700F19780850700F1A380440700F1B1
:10168800B180020700F1BF80C60600F1CD80850653
:1016980000F1DB80440600F1E980020600F1F780E2
:1016A800C60500F10581850500F11381440500F1A7
:1016B8002181020500F12F81C60400F13D818504D6
:1016C80000F14B81440400F15981020455D4BDE86E
:1016D800F08F334A55692C435461BDE700242246F4
:1016E8004FF0010E4FF0030904E00132102A04F113
:1016F8000204ECD00EFA02F636EA0005F5D1D3F86A
:1017080008A009FA04F5ED430AEA050AC3F808A097
:10171800D3F808B00CFA04FA4AEA0B0AC3F808A08E
:10172800B3F804A01FFA8AFA2AEA06069E80B3F8DC
:1017380004A008FA02F646EA0A06B6B29E801E68B7
:101748002E401E60D3F800A007FA04F646EA0A06FF
:101758001E60D3F80CA001FA04F605EA0A0A46EA64
:101768000A05DD60C1E70E4A95692C43946173E769
:101778000B4AD5692C43D4616EE71A6822F04042BF
:101788001A601A6842EA87771F60DA6822F04042D6
:1017980042EA8171D960BDE8F08F00BF4026030896
:1017A800001002401A6822F003021A601A683A43CD
:1017B8001A60DA6822F003020A438507DA607FF5C7
:1017C8005DAF1A6822F00C021A601A6842EA8702B2
:1017D8001A60DA6822F00C0242EA81024407DA60F1
:1017E8007FF54FAF1A6822F030021A601A6842EA91
:1017F80007121A60DA6822F0300242EA0112DA604F
:1018080002077FF541AF1A6822F0C0021A601A6811
:1018180042EA87121A60DA6822F0C00242EA8112AC
:10182800C606DA607FF533AF1A6822F440721A6090
:101838001A6842EA07221A60DA6822F4407242EA19
:1018480001228506DA607FF525AF1A6822F4406226
:101858001A601A6842EA87221A60DA6822F440623B
:1018680042EA81224406DA607FF517AF1A6822F44B
:1018780040521A601A6842EA07321A60DA6822F49B
:10188800405242EA0132DA6002067FF509AF1A686F
:1018980022F440421A601A6842EA87321A60DA680B
:1018A80022F4404242EA8132C605DA607FF5FBAE97
:1018B8001A6822F440321A601A6842EA07421A602B
:1018C800DA6822F4403242EA01428505DA607FF59F
:1018D800EDAE1A6822F440221A601A6842EA87427A
:1018E8001A60DA6822F4402242EA81424405DA604A
:1018F8007FF5DFAE1A6822F440121A601A6842EACD
:1019080007521A60DA6822F4401242EA0152DA6099
:1019180002057FF5D1AE1A6822F440021A601A68EF
:1019280042EA87521A60DA6822F4400242EA815297
:10193800C604DA607FF5C3AE1A6822F040721A60F6
:101948001A6842EA07621A60DA6822F0407242EACC
:1019580001628504DA607FF5B5AE1A6822F040624C
:101968001A601A6842EA87621A60DA6822F04062EE
:1019780042EA81624404DA607FF5A7AE1A6822F071
:1019880040521A601A6842EA07721A60DA6822F04E
:10199800405242EA0172DA6097E600BF10B50409C6
:1019A800013C022C17D80D4B33F8142000F00F001F
:1019B80042FA00F313F001030DD0012303FA00F0FB
:1019C800013810402BF07CFE054A064B125D10448E
:1019D80003EBC00010BD002010BD00BF3424030875
:1019E8003C240308B85B0020564B574A57482DE95A
:1019F800F04F4FF080069E874FF48076A3F844603E
:101A08004FF40076A3F84C604FF48066A3F8546056
:101A18004FF400664FF09041A3F85C604FF4805695
:101A28004FF400554FF480444FF0010B4FF0020A79
:101A38004FF004094FF008084FF0100C4FF0200E3B
:101A4800402719609960196199611962996219634F
:101A5800996319649964196599651966996619678E
:101A68009967A3F864604FF400414FF08006A3F82B
:101A780004B0A3F80CA0A3F81490A3F81C80A3F852
:101A880024C0A3F82CE09F86A3F86C50A3F87440F8
:101A9800A3F87C10A3F8BC604FF48076A3F8C46068
:101AA8004FF40076A3F8CC604FF48066A3F8D460B6
:101AB8004FF40066A3F8DC604FF48056C3F880202A
:101AC800A3F884B0C3F88820A3F88CA0C3F89020AA
:101AD800A3F89490C3F89820A3F89C80C3F8A0209A
:101AE800A3F8A4C0C3F8A820A3F8ACE0C3F8B020BA
:101AF800A3F8B470C3F8B820C3F8C020C3F8C8204E
:101B0800C3F8D020C3F8D820C3F8E020A3F8E460D5
:101B1800C3F8E820A3F8EC50C3F8F020A3F8F44089
:101B2800C3F8F820A3F8FC10C3F80001A3F8045187
:101B3800C3F80801A3F80C41C3F81001A3F8141165
:101B4800BDE8F08FB85B002000040048000800489A
:101B5800002867D003682DE9F04F03F138445C4E44
:101B6800A40A0125345D04F01F066409022C05FA55
:101B780006F558D0032C00F0A580012C58D0808899
:101B8800B0FA80F4C4F11F04A4B2E50803EB85059C
:101B980004F007042E6AA4000F27A74026EA0706C8
:101BA8002E622E6A01F00307A2407C1E3243012CEC
:101BB800C1F3810CC1F300182A62C1F341113CD969
:101BC800C60700F18980850700F19580440700F178
:101BD800A380020700F1B180C60600F1BF80850628
:101BE80000F1CD80440600F1DB80020600F1E980B7
:101BF800C60500F1F780850500F10581440500F16F
:101C08001381020500F12181C60400F12F818504AA
:101C180000F13D81440400F14B81020400F1598137
:101C2800BDE8F08F70472B4CA6693543A561A6E740
:101C3800284C666935436561A1E7002422464FF0C8
:101C4800010E4FF0030904E00132102A04F10204E6
:101C5800E6D00EFA02F636EA0005F5D1D3F808A068
:101C680009FA04F5ED430AEA050AC3F808A0D3F80F
:101C780008B00CFA04FA4AEA0B0AC3F808A0B3F849
:101C880004A01FFA8AFA2AEA06069E80B3F804A07E
:101C980008FA02F646EA0A06B6B29E801E682E4088
:101CA8001E60D3F800A007FA04F646EA0A061E608A
:101CB800D3F80CA001FA04F605EA0A0A46EA0A056E
:101CC800DD60C1E7034CE6693543E56157E700BFCE
:101CD80040260308001002401A6822F003021A6026
:101CE8001A683A431A60DA6822F003020A43850741
:101CF800DA607FF56BAF1A6822F00C021A601A6876
:101D080042EA87021A60DA6822F00C0242EA81028B
:101D18004407DA607FF55DAF1A6822F030021A6076
:101D28001A6842EA07121A60DA6822F0300242EAB8
:101D38000112DA6002077FF54FAF1A6822F0C0027D
:101D48001A601A6842EA87121A60DA6822F0C0023A
:101D580042EA8112C606DA607FF541AF1A6822F4BA
:101D680040721A601A6842EA07221A60DA6822F496
:101D7800407242EA01228506DA607FF533AF1A68BD
:101D880022F440621A601A6842EA87221A60DA6806
:101D980022F4406242EA81224406DA607FF525AFE8
:101DA8001A6822F440521A601A6842EA07321A6026
:101DB800DA6822F4405242EA0132DA6002067FF51C
:101DC80017AF1A6822F440421A601A6842EA87324A
:101DD8001A60DA6822F4404242EA8132C605DA60C3
:101DE8007FF509AF1A6822F440321A601A6842EA8D
:101DF80007421A60DA6822F4403242EA0142850555
:101E0800DA607FF5FBAE1A6822F440221A601A687D
:101E180042EA87421A60DA6822F4402242EA8142A2
:101E28004405DA607FF5EDAE1A6822F440121A60B4
:101E38001A6842EA07521A60DA6822F4401242EA43
:101E48000152DA6002057FF5DFAE1A6822F440021B
:101E58001A601A6842EA87521A60DA6822F4400265
:101E680042EA8152C604DA607FF5D1AE1A6822F0E0
:101E780040721A601A6842EA07621A60DA6822F049
:101E8800407242EA01628504DA607FF5C3AE1A68DF
:101E980022F040621A601A6842EA87621A60DA68B9
:101EA80022F0406242EA81624404DA607FF5B5AE0E
:101EB8001A6822F040521A601A6842EA07721A60D9
:101EC800DA6822F0405242EA0172DA6002047FF5D1
:101ED800A7AE1A6822F040421A601A6842EA877769
:101EE8001F60DA6822F0404242EA8171D960BDE899
:101EF800F08F00BF002852D0036803F138422DE963
:101F0800F04F920A504DAA5C02F01F0552090124B5
:101F1800022A04FA05F443D0032A00F09080012A2B
:101F280043D001F003077A1E012AC1F3810CC1F3E3
:101F380000188088C1F341113CD9C60700F1888098
:101F4800850700F19480440700F1A280020700F1A0
:101F5800B080C60600F1BE80850600F1CC8044063C
:101F680000F1DA80020600F1E880C60500F1F6808B
:101F7800850500F10481440500F11281020500F194
:101F88002081C60400F12E81850400F13C814404BF
:101F980000F14A81020400F15881BDE8F08F7047D2
:101FA8002A4A95692C439461BBE7284A55692C4312
:101FB8005461B6E7002422464FF0010E4FF00309A2
:101FC80004E00132102A04F10204E6D00EFA02F607
:101FD80036EA0005F5D1D3F808A009FA04F5ED436F
:101FE8000AEA050AC3F808A0D3F808B00CFA04FAFC
:101FF8004AEA0B0AC3F808A0B3F804A01FFA8AFA41
:102008002AEA06069E80B3F804A008FA02F646EA11
:102018000A06B6B29E801E682E401E60D3F800A045
:1020280007FA04F646EA0A061E60D3F80CA001FA7D
:1020380004F605EA0A0A46EA0A05DD60C1E7034A2A
:10204800D5692C43D4616CE7402603080010024090
:102058001A6822F003021A601A683A431A60DA68AA
:1020680022F003020A438507DA607FF56CAF1A682D
:1020780022F00C021A601A6842EA87021A60DA68CB
:1020880022F00C0242EA81024407DA607FF55EAF73
:102098001A6822F030021A601A6842EA07121A60B7
:1020A800DA6822F0300242EA0112DA6002077FF5AC
:1020B80050AF1A6822F0C0021A601A6842EA871202
:1020C8001A60DA6822F0C00242EA8112C606DA60B3
:1020D8007FF542AF1A6822F440721A601A6842EA21
:1020E80007221A60DA6822F4407242EA0122850661
:1020F800DA607FF534AF1A6822F440621A601A6811
:1021080042EA87221A60DA6822F4406242EA8122AF
:102118004406DA607FF526AF1A6822F440521A6046
:102128001A6842EA07321A60DA6822F4405242EA30
:102138000132DA6002067FF518AF1A6822F44042CD
:102148001A601A6842EA87321A60DA6822F4404252
:1021580042EA8132C605DA607FF50AAF1A6822F4CE
:1021680040321A601A6842EA07421A60DA6822F4B2
:10217800403242EA01428505DA607FF5FCAE1A6812
:1021880022F440221A601A6842EA87421A60DA6822
:1021980022F4402242EA81424405DA607FF5EEAE3D
:1021A8001A6822F440121A601A6842EA07521A6042
:1021B800DA6822F4401242EA0152DA6002057FF539
:1021C800E0AE1A6822F440021A601A6842EA87529E
:1021D8001A60DA6822F4400242EA8152C604DA60E0
:1021E8007FF5D2AE1A6822F040721A601A6842EA85
:1021F80007621A60DA6822F0407242EA01628504D6
:10220800DA607FF5C4AE1A6822F040621A601A6874
:1022180042EA87621A60DA6822F0406242EA816222
:102228004404DA607FF5B6AE1A6822F040521A60AC
:102238001A6842EA07721A60DA6822F0405242EAE3
:102248000172DA6002047FF5A8AE1A6822F04042F3
:102258001A601A6842EA87771F60DA6822F04042FB
:1022680042EA8171D960BDE8F08F00BF10B1036800
:1022780082881A85704700BF10B1036882889A6106
:10228800704700BF10B5014600BF074C2368986827
:10229800FFF7ECFF23685868FEF788F8236898680A
:1022A800FFF7EAFF00BF10BDBC57002038B1002976
:1022B8008388026814BF002110218B409361704706
:1022C8000E4B1B8801463BB90D4B0E4A1B78106814
:1022D8000BB981F00101E9E70B4B5A691AB118B93A
:1022E8001A68106058747047084A18681188084AB4
:1022F80092FBF1F2012102605974704744570020A3
:1023080046570020485700204C57002064570020AB
:1023180020A1070010B40A4B0A4A1C780123834005
:10232800234052F8200029B9B3FA83F149095DF82E
:10233800044BBBE7191C18BF01215DF8044BB5E736
:10234800345700203857002030B1036882881B8A30
:102358001A4214BF01200020704700BF38B590F81A
:10236800593003B938BD04461846FFF717FB054630
:10237800FFF7EAFF01460028F4D1D5B12023E87120
:10238800AB712846FFF7B6FD2146104B41F8103FC8
:10239800284620F037FFAB88B3FA83F3C3F11F0355
:1023A8005A1CDFD001229A4009490B6813430B607D
:1023B80038BD2946FFF79EFD2146044B41F8103FE2
:1023C800284620F01FFF0122EEE700BF3109000870
:1023D8000004014070B5044600F11405FFF7BEFF84
:1023E800236E80226B21284698476420FEF7E0FC84
:1023F800236E284603226B219847236E94F85420B5
:102408001921284698470F20FEF7D2FC236E94F82E
:10241800522028461A219847236E284618221B2145
:102428009847236E284618221C219847236E284671
:102438000222372198472846236E01223821BDE819
:1024480070401847F8B5434E0446FFF787FF3778C2
:10245800C7B104F11405A06928F068F994F852206E
:102468001A212846FDF7CCFF0120FEF78BFDA06955
:1024780028F04AF92046FEF711FA94F93E30013364
:102488005FD0F8BD04F11405A06928F04FF9802247
:102498006B212846FDF7B4FF9620FEF789FC03223E
:1024A80068212846FDF7ACFF9620FEF781FC032241
:1024B8006B212846FDF7A4FF0F20FEF763FD1022CD
:1024C8006A212846FDF79CFF0F20FEF75BFD3A4680
:1024D8006C212846FDF794FF0F20FEF753FD94F872
:1024E800542019212846FDF78BFF0F20FEF74AFDDF
:1024F80018221B212846FDF783FF0F20FEF742FD17
:1025080010221C212846FDF77BFF0F20FEF73AFD1D
:10251800102237212846FDF773FF0F20FEF732FD02
:10252800012238212846FDF76BFF0F20FEF72AFD10
:10253800A06928F0E9F80120FEF724FD0123337093
:1025480089E794F93C3001339BD10620BDE8F84077
:1025580003F030B8F81D00202DE9F0410B4E346827
:1025680073691C400FD0DFF828800127B4FA84F380
:10257800C3F11F0307FA03F558F8230003689847C7
:10258800AC437561F2D1BDE8F08100BF00040140A1
:10259800745700202DE9F0410B4E346873691C40D4
:1025A8000FD0DFF828800127B4FA84F3C3F11F03A2
:1025B80007FA03F558F8230003689847AC43756198
:1025C800F2D1BDE8F08100BF00040140745700203B
:1025D8002DE9F0410B4E346873691C400FD0DFF8C9
:1025E80028800127B4FA84F3C3F11F0307FA03F51F
:1025F80058F8230003689847AC437561F2D1BDE8E9
:10260800F08100BF00040140745700202DE9F0411B
:102618000B4E346873691C400FD0DFF828800127FF
:10262800B4FA84F3C3F11F0307FA03F558F823003B
:1026380003689847AC437561F2D1BDE8F08100BFEB
:1026480000040140745700202DE9F0410B4E346816
:1026580073691C400FD0DFF828800127B4FA84F38F
:10266800C3F11F0307FA03F558F8230003689847D6
:10267800AC437561F2D1BDE8F08100BF00040140B0
:10268800745700202DE9F0410B4E346873691C40E3
:102698000FD0DFF828800127B4FA84F3C3F11F03B1
:1026A80007FA03F558F8230003689847AC437561A7
:1026B800F2D1BDE8F08100BF00040140745700204A
:1026C8002DE9F0410B4E346873691C400FD0DFF8D8
:1026D80028800127B4FA84F3C3F11F0307FA03F52E
:1026E80058F8230003689847AC437561F2D1BDE8F8
:1026F800F08100BF0004014074570020084A0948CF
:1027080008B5936943F001039361002140222DF03D
:10271800DCFC054B4FF0FF321A60C3F8032008BDFC
:102728000010024074570020B457002003685B6A09
:10273800184700BF2DE9F041044618460D461646D5
:1027480098462AF013FB2768E6722844A0722946A7
:102758007D69434632462046AC46BDE8F0416047B5
:10276800036810B504461B689847236820469B6891
:102778009847A37B0133A37310BD00BF10B503684E
:1027880004469B689847FF2301226373227310BD98
:10279800427A02B9704710B504460368406804F1EC
:1027A8000A0198470023637210BD00BF437A5A1C80
:1027B8000344D2B242729972037A934200D802B9A2
:1027C800704710B504460368406804F10A01984749
:1027D8000023637210BD00BF30B40B4D002305F118
:1027E800140101E0272B0BD011F8132082424FEA85
:1027F800430403F10103F5D12C44607D30BC7047DC
:10280800002030BC704700BF3C02030870B5448804
:1028180006460D46C4F30B042246002128462DF037
:1028280054FC3369094A934209D3094A934206D2B0
:10283800224628461946BDE870402BF0C5B923B199
:1028480021462846BDE87040184770BD2C6603082D
:102858001D670308064B07498B4202D3002318461D
:1028680070471A88C2F30B029042F8D01433F3E78A
:10287800E06103082C660308024A136823EA000093
:1028880010607047F04E0020F8B5174D2B78A32B39
:1028980028D16B78BE2B25D1022229464FF6FF702E
:1028A800FDF7D0FF114FAC1C22884AB1A618BE42D2
:1028B80018D2052A16D92146FDF7C4FF3446F3E796
:1028C80021460222FDF7BEFF0222A118FDF7BAFF3A
:1028D8000634074B641B1C8041F60F53C31A584239
:1028E8005841F8BD0020F8BD00F0030800000408B6
:1028F800BC3900202DE9F04FDFF848914C4F8BB0E0
:102908000326A7EB09071822002104A82DF0DDFBF8
:10291800484BCDF8109005971A69120604D5464A17
:102928005A6002F188325A6001228DF8242034223C
:10293800DA60424B424C1B88ADF8003002226946EF
:1029480004A8FEF7F5F9022269464FF6FF70FDF775
:1029580079FFDFF8F4A080464FF0000B544536D3DA
:102968000AAC002524F8245D0222214604A8FEF7BB
:10297800DFF9022221464046FDF764FF40BAC04312
:10298800ADF80800022202A904A8FEF7D1F90798B9
:1029980060B106ABC0F10402294618442DF095FB3E
:1029A800069904A8FEF76BF9079508909DF824305E
:1029B800089A23B11F490B6943F080030B61013E5C
:1029C8002DD0002A9FD1FFF75FFF50B32CE0658818
:1029D8008DF80DB0C5F30B05AB1DADF80830238895
:1029E800C3F30B02ADF80A201B0B062202A904A8A8
:1029F8008DF80C30FEF79CF9062202A94046FDF737
:102A080021FF616880462A4604A8FEF791F96168AB
:102A180040462A46FDF716FF143480469EE7002AF2
:102A2800D1D0052002F0C6FD0BB0BDE8F08F00BF85
:102A38000000040800200240230167459E020308A5
:102A4800E061030800F003082C6603080378202BD4
:102A5800024600F10100F9D0092BF7D02D2B2CD01C
:102A68002B2B03BF5378B7EE000A0246B7EE000AD5
:102A7800A3F13001C8B209289FED467A10D8F2EECA
:102A8800046A07EE901AF8EEE77A12F8013FE7EECB
:102A9800267AA3F13001C8B20928B0EE677AF0D9D6
:102AA8002E2B4CD003F0DF03452B0BD0F7EE007A2A
:102AB80067EE276A20EE260A70475378BFEE000AB1
:102AC8000246D5E710B451782D2959D02B290ABFD1
:102AD8009178501C901C0024A1F13003092B53D885
:102AE800002303EB830301EB430310F8011FA1F15B
:102AF8003002092AA3F13003F3D9B3F59A7F28BF2E
:102B08004FF49A73072B42D9DFED236A1A46F7EE82
:102B1800007A083A072A67EEA67AFAD803F007037C
:102B28002BB1F2EE046A013B67EEA67AFBD124B31F
:102B3800C7EE276A5DF8044B20EE260A70475378E3
:102B4800A3F13001C8B2092802F10102AAD8F2EEB5
:102B5800046AF0EE665A07EE901AF8EEE77A12F871
:102B6800013F87EEA66AA3F13001C8B2092866EED4
:102B7800A56A37EE067AEED994E767EE276AD9E7B1
:102B8800901C91780124A7E7F7EE007ACFE7F7EEDB
:102B9800007AC5E70000000020BCBE4CB5EEC00AB4
:102BA800DFED317AF1EE10FACCBF30EE270A30EEC5
:102BB800670ADFED2E7A20EE270A30B5FDEEC07ADF
:102BC80087B017EE904A054684EAE470002303A90B
:102BD800A0EBE4700193009302931AF0A7F8002C7D
:102BE800ACBF20232D2303A88DF800302AF0BEF8AF
:102BF800012803A924D002282DD0032805BF30239B
:102C0800684668468DF801302DF085FA68462AF046
:102C1800ADF80338C4B22246694628462DF0D9FAE1
:102C280000232B5528462AF0A1F82E22431C2A54AB
:102C38000DEB0401E8182DF08BFA284607B030BDDB
:102C4800302368468DF801308DF802308DF8033056
:102C58002DF061FADAE7302368468DF801308DF8F7
:102C680002302DF058FAD1E76F12033A00007A4487
:102C78002DE9F041064615460846B6FBF2F43CB984
:102C880005FB1464124B1B5D00F8013BBDE8F081A5
:102C9800B4FBF2F767B90E4B05FB174705FB146445
:102CA800DA5D00F8012B1B5D00F8013BBDE8F081FF
:102CB800B7FBF2F8B8F1000F02D04046FFF7D8FF93
:102CC80005FB1878024B13F8082000F8012BE3E7FE
:102CD800782E030830B402681146531C036011F8BB
:102CE800024B0160D31C517803609378151D056071
:102CF8001B0443EA0123D078234343EA006030BC35
:102D0800704700BF0368591C1A46016012F8021B7D
:102D18000260587841EA0020704700BF03685A1CD7
:102D280002601878704700BF38B504460068154639
:102D38002AF04AFF22682A44226038BD036810B48A
:102D48000A0A5C1C04601A7003685A1C0260197035
:102D58005DF8044B704700BF03685A1C026010B44A
:102D6800197003680A0A5C1C04601A7003680A0C6C
:102D78005C1C04601A700368090E5A1C0260197002
:102D88005DF8044B704700BF03685A1C0260197055
:102D98000368090A5A1C0260197070472DE9F04748
:102DA800002488B080460F461E46A14605AD531C38
:102DB8000393117839B3252933D1931CCDF810909A
:102DC8000393507830284ED04FF0000AA0F130031A
:102DD800DBB2092B42D96C2819D0642800F0938003
:102DE80024D825281CD063D9582876D063281BD12D
:102DF80031784046B847039A531C03931178043638
:102E080001340029D7D1204608B0BDE8F087039BDC
:102E18005A1C03921B78642B7CD02AD8252B54D1BA
:102E2800252140460134B847039AC0E7732833D0B8
:102E380044D975284FD106F1040E30682B4600227C
:102E48000A217646FDF7F4FB049A00955346394665
:102E58004046FDF72BFC039A0444A8E704AA03A9FB
:102E680019F040FFB7E7D31C039390784FF0010A9D
:102E7800ACE7732B10D05BD9752B3AD0782B96D151
:102E8800A3F15802B2FA82F2306852092B46102197
:102E98000436FDF7CDFBD7E73368049A009339462B
:102EA80000234046FDF702FC04360444039A7EE7FB
:102EB8000028B9D1204608B0BDE8F0876E28B3D104
:102EC800039A336804361C6071E72AD9582BD7D087
:102ED800632B8DD06BE77828A6D1A0F15802B2FAFF
:102EE80082F2306852092B461021FDF7A1FB043607
:102EF800AAE706F1040E30682B4600220A2176461E
:102F0800FDF796FBA0E7331D306829461E46FDF7FE
:102F180061FB99E7331D306829461E46FDF75AFBC9
:102F280092E7002B7FF443AF204608B0BDE8F08756
:102F38006E2BC6D03BE700BF0EB400B584B005AB1E
:102F4800019053F8042B0649039301A8FFF726FFC5
:102F5800019B00221A7004B05DF804EB03B07047BF
:102F6800A90600080FB430B583B006AB0A490B4870
:102F780053F8042B096800680193FFF70FFF084C0A
:102F880005462068FEF75CF90028FAD0284603B009
:102F9800BDE8304004B07047783100207C31002013
:102FA80058610020DFED2B7AB4EEE70AF1EE10FA53
:102FB8004ADDDFED296A9FED297A01E0B0EE670A64
:102FC800B4EEC70AF1EE10FA70EE667AF6DC9FED01
:102FD800247AF4EEC77AF1EE10FA38D5DFED1E6ADE
:102FE8009FED207A01E0F0EE407AF4EEC77AF1EE38
:102FF80010FA37EEA60AF6D4DFED1B7AB4EEE70A2C
:10300800F1EE10FA14DDDFED137A37EEC00A60EE48
:10301800006A9FED166A9FED167ADFED167AA6EE26
:10302800867A20EE266AE6EE877AA6EE270A7047A9
:10303800DFED117AB4EEE70AF1EE10FA44BFDFEDE6
:10304800087A37EEC00AE2E7F0EE407ABFE7B0EE62
:10305800670AD1E7DB0F4940DB0FC940E4CB1641D3
:10306800DB0F49C0E4CB16C1DB0FC93F92E741B97A
:103078009730083C15A82ABEDB0FC9BF09B909E07B
:10308800194690FBF1F301FB13030846002BF7D117
:10309800084670470146FBE710B507EE901A2DED7C
:1030A800028BB8EE678ADFED217A28EE008A0446A3
:1030B80028EE278AB0EE480A2AF046FFF0EE408A4A
:1030C800B0EE480A2AF0A2FEF7EE007A9FED187AD1
:1030D800F0EE675AE8EE875A0023A361B0EE676AFC
:1030E800C7EEA56A63612362E361A8EEC76ABDEC17
:1030F800028B77EEC07AB6EE007AF8EE005A27EE29
:10310800877A20EE250A27EE267A26EE266A67EECB
:10311800A67A20EE260A84ED046AC4ED017A84EDCD
:10312800007A84ED027A84ED030A10BD27D4D236E2
:10313800F304353F10B44C09012250F8243001F053
:103148001F0102FA01F10B4340F824305DF8044BEB
:10315800704700BF4B0901F01F0150F823200123DD
:1031680003FA01F1114214BF18460020704700BF4E
:10317800074A084B10781B78074A834296BFC31A40
:10318800C3F180030020126818441044704700BF40
:10319800007100207D7000202C560020064A074B45
:1031A80010781B7883428ABFC3F18003C01AC01805
:1031B800C0F17F00704700BF007100207D700020C3
:1031C80030B5144C237883B01BB90120237003B0A9
:1031D80030BD052200238DF800208DF8013000BF96
:1031E8000D4D2B689868FFF741F82B6801AA6946CE
:1031F800586827F0D1F92B689868FFF73DF800BFA9
:103208009DF8053003F0010383F00100237003B03B
:1032180030BD00BFCE570020BC57002070B5064C0B
:103228000646256803E023685B1BB34203D8FFF713
:10323800C7FF0028F7D070BD6C5700202DE9F04F6C
:1032480089B0B2F1000A02900491039340F3B08070
:103258000B46002201EB8A0153F8040B8B4202440F
:10326800FAD1039B0592002B00F09A80059B002B56
:103278006AD0544B059A1B68DFF85C91009200995C
:10328800DAB25118B1F5807F8CBFC2F58072009A0E
:1032980001924D4A92689A426DD9190C1A0A4FF058
:1032A800020406208DF81F308DF81E208DF81D10A1
:1032B8008DF81C40FFF7B2FF0620FEF7E3FF434AF4
:1032C8000123137000BFD9F800309868FEF7CEFFCD
:1032D800D9F8003007A95868002227F01BF9002404
:1032E800049D029E019FA34629684FEA8408002294
:1032F8000B46013471B1B9422AD2D9F800003168BD
:103308004068FDF7E3F82A68336813443360BF1A4E
:10331800C5F800B0A24505F1040506F10406E3D19D
:10332800D9F800309868FEF7A7FF00BF254B019930
:1033380000981B68421A0092224A0B441360039AB1
:1033480032B3009A002A9AD1059809B0BDE8F08FE7
:10335800029CD9F8003054F80810586800223B46FF
:10336800FDF7B4F854F808202B683A44DF1B44F8FA
:1033780008202F60D4E70598009C1549154A001BC2
:103388000590059800230B70137009B0BDE8F08F05
:10339800059B009A9B1A0593059809B0BDE8F08F24
:1033A800FFF70EFF00287FF461AF039B0593CBE77F
:1033B800039C1CB9FFF704FF0594C5E70023059398
:1033C800C2E700BF2C560020FC130020CE57002077
:1033D800007100207D700020BC57002070B5104D92
:1033E800104E2B7831788B4284B016D00E4A039257
:1033F8001A4402928CBF0C46CA1A04A98CBFC3F1A6
:1034080080020024012341F8102D02A80222019411
:10341800FFF714FF002333702B7004B070BD00BF9A
:103428007D700020007100208070002070B5194C5C
:10343800194D23782978994284B027D0174A0392E6
:103448001A44029234BF0E46CA1A04A934BFC3F103
:1034580080020026002341F8102D02A802220196BE
:10346800FFF7ECFE23781844C0B203062B7848BF58
:1034780080F080008342207002D0002004B070BD2C
:10348800002301202B70237004B070BD012004B00C
:1034980070BD00BF7D70002000710020807000208A
:1034A80008B545F20820FFF7B9FE0620FEF7EAFE48
:1034B800064B0122C7201A70FEF7E4FE04480549AE
:1034C800054A002303700B70136008BDCE57002017
:1034D800007100207D7000202C5600202DE9F0415D
:1034E80082B00346060C050A032406208DF807302F
:1034F800884617468DF805608DF806508DF804400B
:10350800FFF78CFEC0B100BF0D4C23689868FEF72A
:10351800ADFE236801A95868002226F0FBFF236846
:103528004246002158683B46FCF7D0FF236898685C
:10353800FEF7A2FE00BF384602B0BDE8F08100BF2A
:10354800BC570020F0B5124B9D6885B00DB905B089
:10355800F0BDED0A14D0002704AE7C196410E00217
:1035680010226946FFF7BAFF0F2809DD6B4653F8AA
:10357800042B01320AD1B342F9D12546AF42ECDB24
:10358800FFF72CFF034BED021D60E0E7671CF5E732
:10359800FC1300202C560020B0F1FF3F0AD002286F
:1035A80010B403DC5DF8044BFDF72ABA00205DF87F
:1035B800044B704700207047F0B55B4B5B4A97B0EF
:1035C8001968914200AF00F0A3805949594A002375
:1035D8004FF47000C1F888003B607B60136843F4C7
:1035E8008033136003E03B68B3F5A04F09D013683C
:1035F80003F400337B603B6801333B607B68002B3E
:10360800F1D04C4B1B6813F4003318BF01237B60C7
:103618007B68012B52D0464C464B474AE260474AEA
:10362800596A11605A6A42F080725A625A6942F4C1
:10363800FC025A610025032207F10801012341F623
:10364800FF764FF09040FD60BE603A73BB7318F090
:1036580013F84FF6FF7307F108013948BB6018F0FB
:103668000BF807F108013748374E18F005F807F14D
:103678000801364818F000F807F10801344817F037
:10368800FBFF07F10801334817F0F6FF07F10800C0
:1036980017F002FEBB683049304AA1FB03133049DA
:1036A8009B0CF0204FF0070E5C370B60566084F8D7
:1036B80023009560C2F800E0BD46F0BD294A1D4BC5
:1036C800122111605A685A605A685A605A6842F45E
:1036D80080625A605A6822F47C125A605A6842F42E
:1036E800E8125A601A6842F080721A601A689201E9
:1036F800FCD559680F4A21F003015960596841F017
:1037080002015960536803F00C03082BFAD182E7D1
:1037180000221A6062B6144B1B6883F30888134BA7
:103728001B689847FEE700BFFC9F0020EFBEADDE98
:1037380000ED00E0001002400005FA05883E002078
:1037480000040048000800483F190100000C004828
:10375800001000480014004883DE1B4310E000E01E
:10376800705700200020024000D8FF1F04D8FF1F18
:1037780070B50F4C0F4DC0EBC00004EB80046869B6
:1037880026693043686182B09209667BA160002592
:10379800012101A863618DF804608DF805208DF87A
:1037A80006508DF8071022F043FF02B070BD00BF2D
:1037B8001014002000100240074BC0EBC00030B4CA
:1037C80003EB8000054C056963692B43636101764F
:1037D800427630BC704700BF101400200010024031
:1037E8002DE9F04F5E4C54F8204083B0002C71D086
:1037F800666D984691465B4B7268E264A1602360EF
:1038080004F15A014FF4807304F5AD726161A2614D
:10381800E36023610746307E26F0B6FAF068A8B167
:10382800514B00215A68904203F11C0300F092802A
:1038380001310C29F6D100207A1CD2B20C21FFF7F5
:10384800BBFFE36CF26822632433A364B068D8B189
:10385800454B00215A68904203F11C0378D001318E
:103868000C29F7D100257A1CD2B20B212846FFF784
:10387800A3FF2346F27E3D492846FFF779FFE36C14
:10388800B26862632833636494F85900FEF786F8D7
:10389800054694F85800FEF781F818F0080F82469C
:1038A80096F819B01AD0CDB118F0110F4FF00B03DC
:1038B80007F1010714BF4E213E21EF715A46AB7143
:1038C8002846FEF745F918F0010F45D0236B5BB386
:1038D800636B4BB3204603B0BDE8F08F18F0010FBF
:1038E8000CBF4FF02E084FF04E0819F0020F09D008
:1038F80045B10B227B1CAA71EB7128465A464146FA
:10390800FEF726F919F0010FE0D0BAF1000FDDD06B
:1039180001370C238AF807705A4641468AF8063060
:103928005046FEF715F9D1E7337FB27E8DF80420B3
:103938009B090021012201A88DF805308DF8061099
:103948008DF8072022F074FE204603B0BDE8F08F02
:10395800CDB288E7C8B26FE72846FEF787FCB5E71F
:1039680084310020A0020308101400204509000833
:103978000348D0F83C3113B100F59A7018477047E6
:10398800101400200348D0F8203113B100F58C70D2
:1039980018477047101400200348D0F804310BB1C1
:1039A800FC301847704700BF101400200348D0F8B7
:1039B800E8300BB1E0301847704700BF1014002002
:1039C8000348D0F8CC300BB1C4301847704700BF5B
:1039D800101400200348D0F8B0300BB1A8301847B5
:1039E800704700BF101400200348D0F894300BB182
:1039F8008C301847704700BF101400200248836FAE
:103A08000BB1703018477047101400200248C36D7E
:103A18000BB1543018477047101400200248036C4B
:103A28000BB1383018477047101400200248436A19
:103A38000BB11C30184770471014002002488368E7
:103A480003B11847704700BF101400201749184BDE
:103A5800184A194810B4D1F8884044F47004C1F8E1
:103A680088401C6844F001041C605C6822405A606D
:103A78001A6822F0847222F480321A601A6822F4DA
:103A880080221A605A6822F4FE025A60DA6A22F02A
:103A98000F02DA621A6B002410404FF000621863BC
:103AA8009C608A605DF8044B704700BF00ED00E041
:103AB800001002400CC07FF8CCFC00FF38B50B4C5E
:103AC80023688BB15A68821A002A054604DA0CE08A
:103AD8005A68AA1A002A07DB9A68226018461A68E8
:103AE80090472368002BF3D138BD38BD80490020AA
:103AF8000B4B002210B4027203F1B404042102E05B
:103B0800072A09DC9979890702D519798154013284
:103B18009C4203F11403F3D15DF8044B704700BFD6
:103B28004826030810B40D4C04232146002200E067
:103B38008B7913F0010301F1140106D101320A2A2D
:103B4800F6D103705DF8044B704702EB820204EB78
:103B580082025DF8044B1379037070474826030806
:103B68000123152122224170C270037083707047AF
:103B78002C22022302704370704700BF08B514F06E
:103B880027F9024B024ADA60FEE700BF00ED00E0C9
:103B98000400FA05024A034B1278197816F048BF58
:103BA8003C1E00203D1E00202DE9F0470569C36832
:103BB8001D4028D00F4606464FF000484FF0000938
:103BC800B5FA85F328FA03F2D2431B3B326115405C
:103BD800042B16D8DFE803F03129211903007B6A8A
:103BE800002B32D003F1FF3A1FFA8AFAC7F8249063
:103BF8003C6A34B123682046514698476468002CD3
:103C0800F8D1002DDCD1BDE8F0873868716B036806
:103C180089B29847002DD3D1F5E77868B16B03686E
:103C280089B29847002DCBD1EDE7B868F16B0368EE
:103C380089B29847002DC3D1E5E7F868316C03686D
:103C480089B29847002DBBD1DDE7F36A1FFA83FAE2
:103C5800CEE700BF2DE9F04F2DED028BA0F10A034E
:103C680089B00C46E72B00F25D86DFE813F01C01F3
:103C78005B065B065B065B065B065B065B065B0634
:103C88005B065B065B065B065B065B065B065B0624
:103C98005B065B065B065B065B065B065B067905F7
:103CA8005B065B065B0669055B065B065B065406FE
:103CB8005B06C6055B06AD055B06A1055B069805B8
:103CC8005B062E065B061A065B065B065B0613069A
:103CD8000B065B0641035B065B063A035B061203B1
:103CE8005B065B065B06F6025B065B065B065B062D
:103CF800D7025B06FC005B063D046E015B065B06B3
:103D08005B065B065B065B065B062D015B060F0424
:103D18005B06DB035B0662035B064E035B065B0622
:103D28005B065B061C05E104DA04A904E8005B06EF
:103D38005B065B0236025B06FF01E3015B065B067E
:103D48005B065B06D8015B065B06B7015B065B0694
:103D58005B06A8019101C30281025B065B065B0654
:103D680072025B065B0689045B065B065B065B0604
:103D78005B065B065B065B065B065B065B065B0633
:103D88005B065B065B061C055B065B065B065B0663
:103D98005B065B065B065B065B065B065B065B0613
:103DA8005B065B065B065B065B065B065B065B0603
:103DB8005B065B065B065B065B065B065B065B06F3
:103DC8005B065B065B065B065B065B065B065B06E3
:103DD8005B065B065B065B065B065B065B065B06D3
:103DE8005B065B065B065B065B065B065B065B06C3
:103DF8005B065B065B065B065B065B065B065B06B3
:103E08005B065B065B065B065B065B065B065B06A2
:103E18005B065B065B065B065B065B065B065B0692
:103E28005B065B065B065B065B065B065B065B0682
:103E38005B065B065B065B065B067E045404AC4EC1
:103E4800337853B1AB4F002537F8021F2046FEF7F1
:103E58009BFF33780135AB42F6DC012009B0BDEC9D
:103E6800028BBDE8F08FA24E3378002BF5D0A24F1D
:103E78000025B846236817F81520591C21601A70C8
:103E880098F8011001EB810101EB810101F2EE21AB
:103E980089B22046FEF778FF33780135AB4208F146
:103EA8000208E7DCD9E7954D284628F05FFF00288F
:103EB800D3DD2B460544226813F8011B501C9D4294
:103EC80020601170F7D1C8E716F096FDFF28064666
:103ED80000F0188608A9002501F8125D0DF10D0003
:103EE8008DF80D5016F068FD08A800F8115D16F061
:103EF80057FD08A800F8105D16F046FD08A820F840
:103F0800085D16F035FD23685A1C22601E70236870
:103F18009DF80D20591C21601A7023689DF80E2009
:103F2800591C21601A7023689DF80F20591C2160C4
:103F38001A7023689DF81020591C21601A702046B9
:103F4800BDF81810FEF720FF87E70B686C4E0125B7
:103F58005A1C0A601D700B68B278591921601A70D2
:103F680028F060FD2368674A67495F192760187061
:103F7800B1F90010B2F90000FFF780F823685A1968
:103F88002260187031882046FEF7FEFE284665E755
:103F98000A685E4B5E491878551C256010702268C7
:103FA8005878551C2560107022689B78501C20603A
:103FB80013702046C988FEF7E7FE01204EE7544DEE
:103FC80008462988FEF7E0FE69882046FEF7DCFEF1
:103FD8002046A988FEF7D8FE01203FE74D4D05F1A0
:103FE8006006A9882046FEF7CFFEE9882046FEF73E
:103FF800CBFE29892046FEF7C7FE2368AA7A591CFA
:1040080021601A702368EA7A591C21601A7055F8E1
:104018000C1B2046FEF7A0FEB542E2D11DE73E4943
:1040280052232268501C2060137011F8013F002BA6
:10403800F7D112E7394800232268056803EB4301EA
:10404800561C6D5C26601570026825680A446E1C53
:10405800527826602A70026825680A4401339278EB
:10406800691C0A2B21602A70E6D1F6E62C4D0B68F4
:104078002A68591C127821601A702B68226899786E
:10408800531C2360002311702A6821681A440133E5
:104098005279481C032B20600A70F5D123682A68DE
:1040A800591C127A21601A7023682A68591CD27820
:1040B80021601A7023682A68591C127921601A70C5
:1040C8002B6820465989FEF75FFE2A682368527AD2
:1040D800591C21601A702A6810E100212046FEF759
:1040E8003BFE20460021FEF74FFE0120B6E600BF4A
:1040F800943B00204E6F0020705A0020E0550020AD
:10410800E84E00201471002016710020FC55002094
:104118002C39002058330020C8020308F83A002040
:10412800F46F0020AD4D08462988FEF72DFE6988FA
:104138002046FEF729FEB5F90430A94AD91782FBB3
:104148000323C1EBA301204689B2FEF71DFE01201F
:1041580084E6A44D0846298AFEF716FE698A204699
:10416800FEF712FE2046A98AFEF70EFE012075E62C
:10417800DFF8ACE20027FEB2714600232268501C2B
:10418800206016702268501C20601370226811F895
:10419800010F0133551C062B25601070EED1013735
:1041A800062F0EF1060EE6D18F4900232268501C17
:1041B800206017702268501C20601370226811F864
:1041C800010F0133551C0B2B25601070EED12368AD
:1041D800864A581C07212060197023680021581C42
:1041E80020601970236892F8F020591C2160012082
:1041F8001A7033E60B687E4A7E4910787E4A5D1C49
:104208002560187023688978581C20601970236805
:104218009278591C216001201A701FE60B68774DAF
:10422800591C2A7921601A7023686A79591C2160FF
:104238001A7029882046FEF7A7FD2368AA79591C19
:1042480021601A7069882046FEF79EFD2368EA7986
:10425800591C216001201A7000E6FEF7B1FF23689F
:10426800674D002803F101010CBF022203222160DF
:104278001A7029882046FEF76FFDA9682046FEF7C8
:104288006BFDFEF775FF01462046FEF765FD012030
:10429800E4E50B685B4A5C4D11785C4A581C206069
:1042A800197011682046FEF757FD2368584A591CB3
:1042B800127A21601A7029882046FEF765FDA988C0
:1042C8002046FEF761FD29892046FEF75DFD0021A5
:1042D8002046FEF759FD20460021FEF755FD012036
:1042E800BCE5084608224A49FEF71EFD0120B5E54F
:1042F8000B68484A581C91782060197023685278D6
:10430800591C216001201A70A8E50B68394A4249F6
:10431800D078394A5D1C2560187023684979581C83
:10432800206019702368D278591C216001201A7006
:1043380094E500212046FEF727FD00212046FEF7E0
:1043480023FD00212046FEF71FFD2368334D00267C
:104358005A1C22601E7023682A68591C92F82C2067
:1043680021601A7023682A68591C92F83620216047
:104378001A7023682A68591C92F8372021601A702D
:1043880023685A1C22601E7023685A1C22601E7003
:1043980023685A1C22601E702B682046598FFEF72E
:1043A800F3FC2B682046198FFEF7EEFC23682A6879
:1043B800591C92F82E2021601A7023685A1C22601A
:1043C8001E702B682046598EFEF7DEFC2B682046AF
:1043D800998EFEF7D9FC012040E500BF6C3B002018
:1043E80067666666905D00203751002054500020B3
:1043F800C0600020045600201456002044390020D4
:10440800FC13002044560020B0310020F04E00205C
:104418005C3E002020560020E8530020F83A002097
:1044280013510020B14E0B687279B14D591C2160AF
:104438001A702B682046198CFEF7A6FC2B682046BC
:10444800D98BFEF7A1FC71892046FEF79DFCB18946
:104458002046FEF799FC2B682046598CFEF794FC01
:104468002B682046998CFEF78FFCF1892046FEF7D1
:104478008BFC318A2046FEF787FC2A68236892F86D
:104488002620591C216001201A70E7E4974EF37822
:10449800002B00F029830B680822591C21601A7030
:1044A80023680122991821601A702368914D591CBC
:1044B8002A7921601A702368AA78591C21601A7019
:1044C80029882046FEF760FCE9892046FEF75CFC57
:1044D8002368F279591C21601A702368EA78591CFC
:1044E800216001201A70B9E40B6800255A1C0A6083
:1044F8001D700B685A1C0A601D700B685A1C0A60F4
:10450800204629461D70FEF727FC20462946FEF75F
:1045180023FC0120A2E4784B03F170052268197886
:10452800501C2060117022685978501C206011704E
:1045380022689978501C206011702268D978501C24
:104548002060117022681979501C2060117022684F
:104558005979501C20601170226899790733501CD2
:104568009D4220601170D9D177E4644D0846E989ED
:10457800FEF70AFC2046A989FEF706FC01206DE437
:104588000B685F4F591C3A7821601A703B78002BF2
:104598003FF463AC0025EEB2304625F039F82368C5
:1045A8004278591C216030461A7025F031F801898B
:1045B8002046FEF7E9FB3B780135AB42EBDC4CE4E7
:1045C800504D514E9FED518ADFF86881DFED508ADA
:1045D80005F120070EE0FCEEE77ACDED017ABDF893
:1045E800041020460435FEF7CFFBAF4206F118064B
:1045F8003FF433AC717C0029F3D0464BD5ED007AFB
:104608001B78012BE7D1444B1B68DB0440F1648223
:10461800F5EE407AF1EE10FA40F08D8240F2DC516E
:10462800DFE7084610223D49FEF77EFB012015E42E
:104638003B4B9B8AB3F5006F00F26282B3F5806F43
:1046480000F27782B3F5007F34BF01270227354D8A
:1046580005F10C0655F8041B91FBF7F1204689B2C9
:10466800FEF792FBAE42F5D12F4D304F05F10C0607
:10467800B5EC010AD7ED087A80EE270A29F018FC74
:1046880081B22046FEF780FBAE42F1D1284D05F1FC
:104698000C0655F8041B204689B2FEF775FBAE429E
:1046A800F7D1FFF7DABB00258146DFF88C80DFF809
:1046B8008CB0059504950695079501214FF6FF7A6C
:1046C80005E001350B2D00F04D8118F9011F4F1C35
:1046D8004AFA05F3F5D0DE07F3D5BBF800302B41D5
:1046E800D807EED506A8FEF725FDEAE7C06000204A
:1046F800F83A0020905D00204C3400200456002039
:10470800D961002054540020D05C002000004042B1
:1047180000E08244B45D0020E4600020445400209E
:10472800243B00205C3B0020D8600020306500203E
:10473800A0390020DB9B9141F80203088251002038
:10474800A74D08462988FEF71FFBA9882046FEF7D3
:104758001BFB20462989FEF717FB0120FFF77EBBCC
:10476800A04D05F15006287824F0DEFB2368027A74
:10477800591C21601A7023686A78591C21601A70C4
:104788002368AA78591C21601A702368EA780435CE
:10479800591CAE4221601A70E5D1FFF75EBB0B6869
:1047A800914A591C527D216001201A70FFF756BBAF
:1047B8008E4D05F1800655F8041F2046FEF7CCFA09
:1047C800AE42F8D1FFF749BB894D05F14006B5F86F
:1047D80080102046FEF7D8FA236895F88220591CE5
:1047E80021601A70236895F883200435591CAE425D
:1047F80021601A70EBD1FFF730BB7B4D0B682A7A2A
:10480800591C21601A70A98B2046FEF7BDFA298B26
:104818002046FEF7B9FA698B2046FEF7B5FA2368F9
:10482800EA7C591C21601A70A98C2046FEF7ACFA64
:10483800E98C2046FEF7A8FA2368AA7F591C216054
:104848001A70236895F82020591C21601A70698C09
:104858002046FEF799FA2368EA7A591C21601A70F3
:10486800E9682046FEF778FA23682A7C591C2160FB
:104878001A70236895F82120591C216001201A70AC
:10488800FFF7ECBA0B6801229918216010461A70DC
:10489800FFF7E4BA08460021FEF75EFA0120FFF7A9
:1048A800DDBA544D544E05F1300795F90210534BBB
:1048B80093F906208A4203F1080336D09E42F7D1C5
:1048C8000835BD42F1D1FFF7C8BA4D4B03F15A057F
:1048D80022685979501C2060117022681978501C80
:1048E8002060117022685978501C2060117022686D
:1048F8009978501C206011702268D978501C20606B
:104908001170226819790633501C9D42206011707D
:10491800DED1FFF7A2BA0B683A4A581C117820601A
:104928001970EBE40020FFF799BA23685A1C22603B
:10493800197029882046FEF727FA2368EA78591C57
:1049480021601A7023682A79591C21601A7023681B
:10495800AA79591C21601A7023686A79591C216048
:104968001A70ADE7DFF8A8A000254FF00808013558
:10497800C5F1200208FA02F2A5F120032AFA05F689
:10498800164328FA03F31E43252D06F001024FF0C3
:1049980000030BD01343EAD0E8B227F0C1F900288E
:1049A800E5D0294606A8FEF7C5FBE0E7164B1B78BD
:1049B800DA0700F1AE800025144E2F4602E00135DB
:1049C800252D27D029463046FEF7C4FB0028F6D00F
:1049D800294606A8FEF7BEFB002878D10137EEE786
:1049E800B0310020485600205C3E00205050002086
:1049F80054500020B45A0020383E0020083E0020C1
:104A080064370020445600204D3C0020D06100202F
:104A180090E33FF4664B674DB3F850102046FEF71D
:104A2800B3F9654B1988204689B2FEF7ADF9634B97
:104A380019684B0103F02002C1F340031343C1F38B
:104A4800800243EA4203C1F3C00243EA8203C1F38E
:104A5800401243EAC20301F0100119432046FEF751
:104A680093F904A904222046FEF75EF92368297801
:104A7800534A581C2060197011886429A8BF642102
:104A88002046FEF781F9B9F1960F47D0002120465C
:104A9800FEF77AF92168B7F1190348BFA7F11203A5
:104AA800A3F3C4034A1C226020461A460B7005A9CA
:104AB800FEF73AF92368434A581C10212060197000
:104AC80020461188FEF748F90120FFF7C7B9394693
:104AD80004A8FEF72FFB81E7F4EEC87AF1EE10FA8E
:104AE80045DA4FF47A717CE50B68B178364A581C80
:104AF8002060197023681278591C21601A70D4E458
:104B08000827A4E523685A1C226001201E70FFF7BD
:104B1800A5B9069B43F0010306934CE723680322DB
:104B2800591C21601A7023686A78591C21601A7010
:104B3800B0E704278BE5F4EEC87AF1EE10FA3FF5FA
:104B48006DADF4EEE87AFDEEE77AF1EE10FA17EEC5
:104B5800901A1ED86FF4F973303903FB01F140F253
:104B6800E73391FBF3F101F2DB5189B239E5FDEE50
:104B7800E77A40F2E73217EE903A303B02FB03F354
:104B880088FB0312D917C1EB622101F2E93189B21E
:104B980027E540F2F313A1F5836103FB01F140F22D
:104BA800E73391FBF3F101F2DD5189B219E500BF5A
:104BB8000C100020EC3A0020FC640020203B002070
:104BC800BE390020C0510020F855002008B5012149
:104BD8000220FDF79FFB094B1B7803F00503052B0B
:104BE80008D000210120FDF795FB00210846FDF7BC
:104BF80091FBFEE713F07EF9F3E700BF8031002058
:104C0800022828BF022010B4084C094B207000EB82
:104C18008002C0EBC20207495DF8044B013003EB88
:104C28004203C0B20B600DF079BA00BFEC3A002025
:104C3800CC4D0020F83A002008B51AF037FAFDF7F5
:104C480059FEBDE808401AF019BA00BF38B5434B01
:104C58005A899989914224BF00225A81198ADA898E
:104C6800914224BF0022DA81DA788AB3072A2FD04A
:104C78003B493C4D91F85700012400210A282C702B
:104C88009C70D9713DD00C2865D0DFED377A8ABB8E
:104C9800364C9FED370AA278002918BFF0EE407A0B
:104CA800062A04D8334901EB820191ED0F0A2179D4
:104CB80059B3013A032A4DD8F7EE007A87EE800AF5
:104CC80029F0F6F82388984228BF1846208038BD76
:104CD800D97921B198780428B8BF04209870204861
:104CE80090F857000A280CD00C28CED1DFED227A94
:104CF800002ACDD0072ACBD00A282CD1DFED1F7A85
:104D0800C6E70A20DFED1E7AC1E79B78154A07EE51
:104D1800103A1178B8EEC77A27EE277A07EE901A7C
:104D2800F8EEE77A67EE877AB4EEE70AF1EE10FA62
:104D380010DDC0EE077AFDEEE77A17EE903A102BF9
:104D4800A8BF1023012BB8BF0123DBB28B4238BFA9
:104D58000B46137038BDDFED0B7A99E7C060002071
:104D680030650020F85500206F120339905D00204F
:104D78006F120338C80203080AD7A3390F506E3AD6
:104D88005304E9386F12833AF8B50F4C0F4DAC4213
:104D980006D2616820461434FDF738FDAC42F8D3DA
:104DA8000B4A0C4B0C4C0D4D0D4E15600125002285
:104DB80004270C4925701A705A700B48B770BDE863
:104DC800F840086015F09EBBE06103082C660308F4
:104DD800F83A0020EC3A0020F8550020CC4D00208D
:104DE800C0600020F46F0020FC3A002008B5FFF7EF
:104DF800CBFF1AF05BF9FDF77DFDBDE808401AF01E
:104E08003DB900BFF0B50C292BD8DFE801F06F2AB7
:104E18002A2A4C2A2A2A2B2A2A2A0700046AB2F8A4
:104E28000CE097881668674D24F480540462036A7E
:104E38004468C16923F4005343EA0E3321F4E64180
:104E4800A84243EA073341EA062100F0B58005F598
:104E58000065A84200F0B08092684460C1610264B5
:104E68000362F0BD046A96899588D2F800E0554F30
:104E780024F480740462036A4468C16923F40073EB
:104E880043EA062321F07301B84243EA052341EAC5
:104E98000E017ED04C4DA8427BD092684460C1611F
:104EA800C2630362F0BD046A96899588D2F800E06F
:104EB800444F24F010040462036A4468816923F0B3
:104EC800200321F0807143EA061321F4E641B84239
:104ED80043EA051341EA0E2148D03B4DA84245D08C
:104EE80092684460816182630362F0BD046A9389B9
:104EF800B2F804E01768334E24F001040462056A2E
:104F08004468816943EA0E0321F4803125F00205E3
:104F18009BB221F07301B04243EA050341EA07015D
:104F280014D0294DA84211D005F54065A8420DD0EE
:104F380005F58065A84209D005F58065A84205D029
:104F480092684460816142630362F0BDD689158A24
:104F5800578A23F0080333433D43D68824F440742A
:104F680023F00403ADB233432C43E9E7D589178A0C
:104F7800D68823F0800343EA051324F44064558A55
:104F880023F0400344EA870443EA061344EA85040D
:104F9800A6E7D589178AD68823F4006343EA052350
:104FA80024F44054558A23F4806344EA071443EAFE
:104FB800062344EA051470E7158A24F4804444EA79
:104FC800851449E7002C0140003401402DE9F04FD9
:104FD800C822002183B07848784CDFF80492784DD5
:104FE800784E794FDFF8FC812BF06FF877487849D5
:104FF800DFF8F4E1DFF8F4C100221359834200F02E
:10500800C180B3F1804F00F0C980AB4200F0C88086
:10501800B34200F0C780BB4200F0C680734500F081
:10502800C580634500F0C480434500F0C380DFF8C5
:10503800C0A153457ED00AF5806A534508BF0923AD
:1050480079D01432C82AD8D15C4C624D624E604F78
:1050580004F1C80802E01434A04568D0A379002BF5
:10506800F9D023794FEA131909F1FF39B9F1020F81
:1050780003F00F03EFD835F8190040FA03F2D2070E
:10508800E9D54FF0010A0AFA03F3013B184028F06A
:1050980017FB16F809305149184411EBC002DAD051
:1050A80051F83000DFF84CE1217A00F138439B0ACF
:1050B8001EF8033003F01F0E5B09022B0AFA0EFAE2
:1050C80062D0032B65D0012B03D17B694AEA030325
:1050D8007B6193880093B3FA83F3C3F11F039BB2F8
:1050E800DA0800EB820203F00703D2F820E09B0005
:1050F8004FF00F0C0CFA03FC2EEA0C0EC2F820E05D
:10510800D2F820E001FA03F343EA0E03136269467A
:105118000023022214348DF804208DF805308DF810
:1051280006308DF8073016F0A7FAA04596D103B0DF
:10513800BDE8F08F082309EBC3034FF0010B93F888
:105148005CA00AF01F034FEA5A1ABAF1020F0BFAD1
:1051580003F30BD0BAF1030F0ED0DA457FF471AF29
:10516800D1F814A043EA0A034B616AE7D1F818A002
:1051780043EA0A038B6164E7D1F81CA043EA0A03F7
:10518800CB615EE70023D6E7BB694AEA0303BB614C
:105198009FE7FB694AEA0303FB619AE70123CAE731
:1051A8000223C8E70323C6E70423C4E70523C2E7AD
:1051B8000623C0E70723BEE7D05700204826030888
:1051C800000400400008004000100040002C01408E
:1051D80000100240342403083C240308B85B002074
:1051E800C802030800400140001400400034014098
:1051F800004401404026030801490248FEF7D4BC98
:10520800705800200048014001490248FEF7CCBC14
:10521800485800200040014001490248FEF7C4BC3C
:10522800205800200004004002494FF08040FEF75B
:10523800BBBC00BFF857002001490248FEF7B4BCC8
:10524800D0570020002C014001490248FEF7ACBCB1
:10525800D0570020002C01402DE9F04104684A4D48
:10526800A30AAB4272D009D8B3F5801F6AD04A3D71
:10527800AB425AD14FF0700E022608E0434DAB42C4
:1052880068D00235AB4252D14FF0C00E04264779A0
:105298004FEA970C002961D0B000634685190227B0
:1052A800D4F80C809F400CEB4503BFB2384D03F196
:1052B800040C47EA080745F8231045F82C20E76056
:1052C800EFF31181502282F31288821905EBC20292
:1052D800136973B313620433821905EBC202576969
:1052E80017B11F6053690433821905EBC20297692D
:1052F80017B11F6093690433821905EBC202D7699D
:1053080017B11F60D36904330027CAB21F6082F344
:105318001188304405EBC000036A6BB9E3684FF6A7
:10532800FE721340E360BDE8F081BDE8F081BDE89E
:10533800F08105EB0E03CFE7E36843F00103E36078
:10534800BDE8F0814FF0480E0126A0E74FF0200E8F
:1053580000269CE74FF0980E032698E7BF08022323
:1053680006FA03F0BB40DB43E768094D9BB23B40BC
:1053780087190CEB470CE3600CF1040345F82C107B
:1053880045F823209CE700BF4B0010005000100098
:10539800D057002030B503685C4D18885C4CB4FBCE
:1053A800F2F20139013AAB4294B283B089B282B2C7
:1053B80066D05848834263D0B3F1804F60D0A0F5DF
:1053C800983083425CD000F58060834258D05248C0
:1053D80083425BD000F5806083427DD022F4407226
:1053E80000F58C3092B283421A80D9621C850ED0A7
:1053F800484A93420BD002F54062934207D002F527
:105408008062934203D002F58062934201D1002268
:105418001A8601225A611A883C4992B242F0010266
:105428008B421A8062D0B3F1804F61D03B4A9342DD
:1054380060D002F5806293425ED002F5006293422A
:105448005CD002F5806293425AD002F590329342C2
:1054580058D002F54062934256D002F580629342DA
:105468001ED002F58062934208BF092219D002A813
:105478004FF0012340F8043D21F0DAF803B030BDC5
:10548800254822F07002834292B2A3D101201A80EB
:10549800D9621C8558611A8892B202431A80C5E7FE
:1054A80008221F4B03EBC20301A893F85D408DF857
:1054B8000440012300228DF805308DF807308DF85F
:1054C800062021F0B5F81B2CD8D1164B019301A862
:1054D80021F0AEF803B030BD01201A80D9621C85D6
:1054E80058611A8892B202431A809CE70022D8E7D2
:1054F8000122D6E70222D4E70322D2E70422D0E72A
:105508000522CEE70622CCE70722CAE7002C014095
:1055180000A24A040034014000100040000400408A
:10552800C802030819010001204B98422DD0B0F1A0
:10553800804F2CD0A3F5943398422AD003F580638A
:10554800984228D003F50063984226D003F580637B
:10555800984224D003F59033984222D003F5406353
:10556800984220D003F58063984207D003F5806302
:10557800984208BF092202D00020704708220C4B2D
:1055880003EBC20393F85C0070470022F7E701229F
:10559800F5E70222F3E70322F1E70422EFE7052209
:1055A800EDE70622EBE70722E9E700BF002C014000
:1055B800C80203082DE9F04F013085B0C3B2039348
:1055C8008E4D8F4F8F4C904E0A230293DFF84092F6
:1055D8001DF03AFC4FF4FA7A4FF0100C4FF47A7041
:1055E800D9F80430C3F30803002B40F0C880EFF368
:1055F8001183002B40F0C3802968A26800BF2B6884
:105608009942F9D1D7F800E000FB0EF39B1AB3FBDF
:10561800FEF300FB01314FF0010E0191D9F804307F
:10562800C3F30803002B40F08E80EFF31183002BA7
:1056380040F089802B68A16800BF2A689342F9D19D
:10564800D7F800B000FB0BF2521AB2FBFBF200FBDA
:105658000323019A9B1AB3F57A7FDFD3BAF1010AC3
:10566800BED1039B002B40F0C4804FF47A7ADFF858
:10567800A09150464FF0100CD9F80430C3F308033A
:10568800002B40F09980EFF31183002B40F09480B9
:105698002968A26800BF2B689942F9D1D7F800E0C1
:1056A80000FB0EF39B1AB3FBFEF300FB01314FF036
:1056B800010E0191D9F80430C3F308033BBBEFF3A3
:1056C800118323BB2B68A16800BF2A689342F9D1D4
:1056D800D7F800B000FB0BF2521AB2FBFBF200FB4A
:1056E8000323019A9B1AB3F57A7FE3D3BAF1010A2F
:1056F800C2D1029B013B02937FF468AF4349444BFC
:105708004448454A0860DA6005B0BDE8F08FEFF319
:1057180011888CF31288A1682368DB0344BFC6F89C
:1057280000E0A1682B6832685FFA88F888F311886E
:10573800D7F800801A4400FB08F35B1AB3FBF8F3B0
:1057480000FB0233CDE7EFF311888CF31288A168D0
:105758002368DB0344BFC6F800E0A1682B68326801
:105768005FFA88F888F31188D7F800801A4400FB9C
:1057780008F35B1AB3FBF8F300FB023369E7EFF3B6
:1057880011828CF31288D4F808E02368D90303D572
:1057980001233360D4F808E02B683168D2B282F371
:1057A80011883A68194400FB02F3A3EB0E03B3FB1C
:1057B800F2F300FB01312EE7EFF311828CF312882C
:1057C800D4F808E02368D90303D501233360D4F85B
:1057D80008E02B683168D2B282F311883A6819441C
:1057E80000FB02F3A3EB0E03B3FBF2F300FB013162
:1057F8005DE718461DF0B0F937E700BF6C57002089
:105808007057002010E000E068570020FC9F00203F
:1058180000ED00E0EFBEADDE0400FA052DE9F0472B
:10582800AF4FB04E19F042FCBE421ED2DFF83C83A7
:10583800DFF83C934446258862197DB14A450DD26C
:10584800052D0BD933886188C3F30B03994200F007
:10585800F680144625886219002DEFD1716830460C
:105868001436FCF7D3FFBE42E4D39F4A1378A3F162
:10587800170102290FD99D4911F83300002840F07B
:105888000081D8000144497829B1994911F8333089
:10589800002B00F01E81974C6378022B84BF0023F5
:1058A80063702378022B84BF00232370924B9A786D
:1058B800042A00F0058132B91A88B2F5F07F84BF56
:1058C8004FF4F0721A808D4D8D4A2B681A40002AC9
:1058D80000F00281D80700F1EE80590400F1E6805B
:1058E8001A0700F1DE809B0400F1D480854D2B68F7
:1058F8005A8C998C914224BF00225A84FFF7A6F94A
:1059080016F084FD10B980480BF05CF98020FCF794
:10591800B3FF4FF40070FCF7AFFF4FF48020FCF7A3
:10592800ABFF4FF40010FCF7A7FF4FF00070FCF737
:10593800A3FF4FF08060FCF79FFF6378022B06D827
:10594800724A734903EB430302EB83030B6023782A
:10595800022B07D803EB83016E4AC3EBC10302EBAA
:1059680043032B6026F054FA002130226A482AF0BB
:10597800ACFB286810F00EFF684B2E6803F150014D
:1059880002E0043399427AD01A78002AF9D19C7837
:10599800D8788442F5D26249624B91F804E06248B3
:1059A800624D5C6B624B2860C827642111FB0E7145
:1059B800DFF8C0E159605F4F30F8061C5E4DAEF865
:1059C800001000219960D960196159619961D96104
:1059D80083F8201083F821103A702E600CB119F06A
:1059E800AFF9564B9FED565A1B88564A9FED566A9B
:1059F8005579564C56495748086006EE903AF8EEE5
:105A0800E66A1388C5EE265A07EE103A53881279CB
:105A1800C4ED005A07EE903AB8EEC77A4E4BF8EE4E
:105A2800E77A1D725A7227EE067A67EE867ABDE823
:105A3800F04783ED017AC3ED007A19F01FBB637953
:105A48009B077FF406AF716894F804A03046FCF712
:105A5800DDFE3388BAEB133F04D01436BE42FFF4A0
:105A6800E9AE02E773887068AA1FC3F30B039A4272
:105A780004F10601A8BF1A4628F0A6F8EDE70122AE
:105A880089E7D8000C186468002C7FF4FBAE172453
:105A98001470F7E63148FCF7EFFE4020FCF7ECFE07
:105AA80024E72F48FCF7E8FE2B681CE72D48FCF795
:105AB800E3FE2B6814E72C48FCF7DEFE2B680CE7A6
:105AC8009A8AB2F57A7FBFF4FEAE4FF47A729A8260
:105AD800F9E618231370DEE643F400532B60F9E669
:105AE8002C660308E0610308445600205C2A03087A
:105AF800840C0308EC3A0020905D0020F04E002052
:105B080009600002F83A0020B45A0020FC3A00204C
:105B1800F46F0020CC4D0020D023002048560020F0
:105B280044390020243B00200A560020A8610020A8
:105B38009C510020221C0020042400201C2200204C
:105B4800C0C9FB482C1E002017B7D13820220020DE
:105B5800303700203661023D0C3700200940000232
:105B680001600002092000020860000202F0030838
:105B7800000004083C4D002008B519F097FAFCF71E
:105B8800B9FE19F07BFAFFF749FE0120BDE808408D
:105B98000CF0C4BA2DE9F04F013085B0C3B20393BD
:105BA8000B4602918B4C8C4E002B00F099808B4D4C
:105BB8008B4FDFF830921DF047F94FF4FA7A4FF027
:105BC800100C4FF47A70D9F80430C3F30803002B93
:105BD80040F0DE80EFF31183002B40F0D980296874
:105BE800A26800BF2B689942F9D1D7F800E000FB02
:105BF8000EF39B1AB3FBFEF300FB01314FF0010ECD
:105C08000191D9F80430C3F30803002B40F08780D2
:105C1800EFF31183002B40F082802B68A16800BF4E
:105C28002A689342F9D1D7F800B000FB0BF2521A58
:105C3800B2FBFBF200FB0323019A9B1AB3F57A7FB0
:105C4800DFD3BAF1010ABED1039B002B40F0BD801F
:105C58004FF47A7ADFF88C9150464FF0100CD9F84F
:105C68000430C3F30803002B75D1EFF31183002B25
:105C780071D12968A26800BF2B689942F9D1D7F879
:105C880000E000FB0EF39B1AB3FBFEF300FB0131AF
:105C98004FF0010E0191D9F80430C3F3080313BB88
:105CA800EFF31183FBB92B68A16800BF2A68934200
:105CB800F9D1D7F800B000FB0BF2521AB2FBFBF295
:105CC80000FB0323019A9B1AB3F57A7FE3D3BAF159
:105CD800010AC4D1029B013B0293002B7FF467AFFA
:105CE80005B0BDE8F08FEFF311888CF31288A16836
:105CF8002368DB0344BFC6F800E0A1682B6832685C
:105D08005FFA88F888F31188D7F800801A4400FBF6
:105D180008F35B1AB3FBF8F300FB0233D2E7EFF3A7
:105D280011888CF31288A1682368DB0344BFC6F886
:105D380000E0A1682B6832685FFA88F888F3118858
:105D4800D7F800801A4400FB08F35B1AB3FBF8F39A
:105D580000FB023370E7EFF311828CF31288D4F85A
:105D680008E02368D90303D501233360D4F808E099
:105D78002B683168D2B282F311883A68194400FB63
:105D880002F3A3EB0E03B3FBF2F300FB01317FE751
:105D9800EFF311828CF31288D4F808E02368D90352
:105DA80003D501233360D4F808E02B683168D2B2F8
:105DB80082F311883A68194400FB02F3A3EB0E033F
:105DC800B3FBF2F300FB013118E718461CF0C4FEE0
:105DD8003EE700BF10E000E0685700206C57002045
:105DE8007057002000ED00E02DE9F04F95B0B0F9B4
:105DF80008500D81EDB2442D00AF0C46904600F0DE
:105E08004384064643D9812D00F07B8300F29880B5
:105E1800542D00F0CC8040F2D6806E2D00F0028424
:105E2800802D40F0D380764B93F800A00AF1020A47
:105E38001AF0FF0A00F09780724BDFF8F481724E77
:105E4800DFF8F0B19A4403F101090A2516E0322D72
:105E580001F0E882A5F13C00C0B2132841F2E982C2
:105E680000232268511C216015702268D14502F177
:105E780001012160137076D019F8015B0A2DE6D173
:105E8800BBF80030FF2BA8BFFF23DBB2E9E7052DE5
:105E980000F0E88320D8022D00F0818040F21083C2
:105EA800032D00F0B583042D40F09080574920461B
:105EB8002A46FCF739FF00212046FCF765FF2268D7
:105EC8000021531C0125236028462B4654371170A6
:105ED8006381BD46BDE8F08F242D5ED040F2A682D6
:105EE800282D00F05783382D70D10A68484B0125BA
:105EF800511C21601570226805215019206011700D
:105F080022680A2150192060117022680021501956
:105F18002060117022681978501920601170226869
:105F280059785019206011702268997853192360A4
:105F38002B461170284654376381BD46BDE8F08F63
:105F4800A02D18D040F29182B82D00F05F83FE2D6D
:105F58003CD1304D05F1080635F8021B2046FCF708
:105F680013FFB542F8D101252B46284654376381E3
:105F7800BD46BDE8F08F284B08461968FCF7ECFED3
:105F8800264B20461968FCF7E7FE254B1968204682
:105F98000125FCF7E1FE2B46E7E7224BF6E7042252
:105FA800214920460125FCF7BFFE2B46C2E70B68B6
:105FB80000215A1C22601970226801255319236098
:105FC8002B461170B6E7522D3FF479AF214628468B
:105FD800FDF740FE03460028C5D1742D00F08382EA
:105FE800772D29D13268716891421EBF531C3360E6
:105FF80011780E4A08BF1946204622F041FFB2E741
:10600800D96100207003030860240020F13A0020C1
:10601800B74D0020FC610020ACF7FF1FB0F7FF1F51
:10602800B4F7FF1FF04E0020A02E0308618102087C
:106038006766666688240020F52D01F0A782472D43
:1060480000F04E83292D336801F06082392D01F06C
:106058004A82212D01F0278271680B3DCA1AEF2D63
:1060680000F2698401A050F825F000BFC37200084F
:106078003F6900083F6900083F6900083F69000858
:106088003F6900083F6900083F6900083F69000848
:106098003F6900083F6900083F6900083F69000838
:1060A8003F6900083F6900083F6900083F69000828
:1060B8003F6900083F6900083F6900083F69000818
:1060C8003F6900083F6900083F6900086F720008CF
:1060D8003F6900084D7200083F69000823720008F4
:1060E8003F6900083F6900083F690008C973000854
:1060F8003F690008537300083F69000821730008CE
:106108003F690008FB7200083F6900081172000827
:106118003F690008B97100083F6900086571000807
:106128003F6900083F6900083F6900083F690008A7
:106138006F5F00083F690008497100083F6900085F
:106148003F6900082F7100083F690008D5700008F2
:106158003F6900083F6900083F6900083F69000877
:10616800957000083F6900083F6900083F6900080A
:10617800557000083F690008077000083F6900086B
:106188003F690008C96F00083F6900083F690008B7
:106198003F6900083F6900083F6900083F69000837
:1061A8003F690008F56E00083F690008736E000833
:1061B8003F690008916D00083F690008B96C000844
:1061C8003F6900084B6E00089B6C00083F69000897
:1061D8003F6900083F6900083F6900083F690008F7
:1061E8003F6900083F6900083F6900083F690008E7
:1061F8003F6900083F6900083F6900083F690008D7
:106208003F6900083F6900083F6900083F690008C6
:106218003F6900083F6900083F6900083F690008B6
:106228003F6900083F6900083F6900083F690008A6
:106238003F6900083F6900083F6900083F69000896
:106248003F6900083F6900083F6900083F69000886
:106258003F6900083F6900083F6900083F69000876
:106268003F6900083F6900083F6900083F69000866
:106278003F6900083F6900083F6900083F69000856
:106288003F6900083F6900083F6900083F69000846
:106298003F6900083F6900083F6900083F69000836
:1062A8003F6900083F6900083F6900083F69000826
:1062B8003F6900083F6900083F6900083F69000816
:1062C8003F6900083F6900083F6900083F69000806
:1062D8003F6900083F6900083F6900083F690008F6
:1062E8003F6900083F6900083F6900083F690008E6
:1062F8003F6900083F6900083F6900083F690008D6
:106308003F6900083F6900083F6900083F690008C5
:106318003F6900083F6900083F690008716C000880
:106328003F690008556C00083F6900083F6900088C
:106338003F6900083F6900083F6900083F69000895
:106348003F6900083F6900083F6900083F69000885
:106358003F6900083F6900083F6900083F69000875
:10636800F76B00083F690008BF6B00083F69000829
:10637800016B0008E76A0008A36B00083F69000882
:10638800CD6A00083F690008A56A00083F6900084F
:10639800456A00083F690008DD6900083F69000890
:1063A8003F690008B36900085D6900084969000889
:1063B8008B69000821690008F76800083F69000830
:1063C8003F6900083F6900083F6900083F69000805
:1063D8003F6900083F6900083F6900083F690008F5
:1063E8003F6900083F6900083F6900083F690008E5
:1063F8003F6900083F6900083F690008D76800083E
:106408003F6900083F6900087F6800083F69000885
:106418003F6900083F6900083F6900083F690008B4
:106428003F6900083F69000867680008202D7FF46D
:10643800CDAD0B68984D591C6A7821601A70236895
:106448002A78591C21601A702368AA78591C21607F
:106458001A7029892046FCF797FC23686A79591C29
:1064680021601A702268A9792BE5822D7FF4AEADE0
:106478000B688A4A8A4D1178874A581C206019701F
:1064880011892046FCF780FC864B22681B88FF2B6D
:1064980002F10101A8BFFF2321601370A96881F3ED
:1064A800100189B22046FCF76FFC296801F30F013F
:1064B80089B22046FCF768FC7B4B2268197800E516
:1064C800012D7FF483AD0B680022591C21601A70DE
:1064D80023685A1C22601D7022682421531C2360E3
:1064E8002B46117026E53268716891421EBF531C15
:1064F800336011786D4A08BF1946204622F0C0FC67
:1065080031E56B4B1E78033616F0FF063FF42BADD2
:10651800684BDFF8C4811E4403F1010A4FF00A09F1
:1065280020E0B9F1500F00F05F87B9F1320F00F0A9
:106538009687A9F13C00C0B2132840F29487002541
:10654800294623685A1C2260204683F80090FCF7ED
:106558001BFC29462046FCF717FC56453FF403ADC3
:106568001AF8019BB9F10A0FDBD1534B9D681968E2
:1065780005EB85054FF6FF736D009D42A8BF1D46CC
:106588009942A8BF194625EAE57521EAE171ADB23D
:1065980089B2D6E70B68DFF84491484E591C0222AD
:1065A80021601A7023684FF006085A1C226083F88D
:1065B800008023680A22591C21601A70236801256B
:1065C8005A1922601D70B9F800102046FCF7DCFB50
:1065D800B9F802102046FCF7D7FB23685A19226045
:1065E80083F8008023685022591921601A702368A3
:1065F8000022591921601A7031882046FCF7C4FB23
:1066080071882046FCF7C0FB2B4693E42C4BBDE475
:106618000B685A1C0A601D700B680222591C216005
:106628001A704CE41F4B0A681B881D4DFF2BA8BF2E
:10663800FF23511C21601370A96881F3100189B2EE
:106648002046FCF7A1FB1F4B20461988FCF79CFB52
:10665800296801F30F0189B220460125FCF794FB54
:106668002B4667E40B2218492046FCF75DFB0822FD
:1066780016492046FCF758FB0125072214492046F5
:10668800FCF752FB2B4655E4002A3FF46CAC114B47
:10669800136001252B464DE48C510020CE6200206A
:1066A8007C6200208862002086510020418D02080B
:1066B800D961002080030308142400204824002006
:1066C8005837002080510020A82E0308B42E030854
:1066D800C02E0308853B000858240020F4550020EC
:1066E800726835687B623046551BFCF7F3FA052D56
:1066F80038627B6A00F2C9878026B346012594E890
:106708000600521A103A9642C8BF1FFA82FBBD4AC9
:10671800396A92683A61521A9345396A7B6220460F
:10672800FA6088BF1FFA82FBFCF716FB7B6A002B16
:1067380000F08987002D40F002872368C7F800D051
:106748005D71C0B00533C7F808D0FB61BBF1000F1D
:1067580001F022803B6A3A69934281F02280AA467E
:106768003E6A7D627C6080255446FB681C1BA54BF5
:10677800B4F5807F28BF4FF480749B6832199A4221
:1067880088BF9C1BFCF72AFE2246BC68304621467F
:10679800FCF7A4FEF969B86104EB000C0B787B6187
:1067A800644530D2DFF884920CF1FF3C04F1FF3EDF
:1067B8001EF8013F09EB830219F823405688FCB103
:1067C80000234FF4004204F1FF3816424FEA520208
:1067D80002D00878284308706D0806D10AF1010A2A
:1067E8004D701FFA8AFA01318025D34505D8F44542
:1067F80000F250864345C0F24D8601339C42E4D1F5
:10680800E645D5D1F9617B6ABA6913449BB2D34591
:106818007B6206D97B6A3A6A1C46D6183B699E4257
:10682800A3D37C68802D1CBF0AF101031FFA83FAE9
:106838000AF1020189B22046FCF7A6FA2368796AB0
:1068480001255A19226020461D70FCF79DFA23681D
:10685800534423602B46D7F800D0FFF76BBB6A4B35
:106868001B78DB0767D40125FEF7E6F9FEF7D6FFAC
:106878002B46FFF75FBB5A1C32601A780F2A5AD88A
:10688800991C3160C2EBC202604958788854D81C00
:1068980030600A4499785170191D3160D978917027
:1068A800591D31601979D170991D3160597911716B
:1068B800D91D31609979517103F108013160DB7993
:1068C800937101250FF020FD2B46FFF733BB3046AF
:1068D800FCF718FADFF84C81A8F80E003046FCF7F0
:1068E80011FA0125A8F80C002B46FFF723BB304608
:1068F800FCF708FADFF83881A8F810003046FCF7F2
:1069080001FAA8F812003046FCF7FCF90125A8F8AE
:1069180014002B46FFF70EBB1A46591C316012F8BB
:10692800020B3260DA1C597832609A781AF0ECFE61
:1069380000287FF418AB4FF0FF352B46FFF7FABA63
:10694800334B344918684E22012527F03DF92B4670
:10695800FFF7F0BA19465A1C32602F4A11F8020B99
:106968001070316059785170D91C31609B789370E0
:106978003046FCF7C7F9294B0125D8802B46FFF78D
:10698800D9BA1A46591C3160254912F8020B087009
:10699800326024495A788A70DA1C3260224A9B781D
:1069A800937001252B46FFF7C5BA3046FCF7AAF9C4
:1069B800DFF86880A8F800003046FCF7A3F9A8F8CB
:1069C80002003046FCF79EF90125A8F804002B4682
:1069D800FFF7B0BADFF85C9099F80030002B3FF46D
:1069E800C2AADFF8548000253046FCF78BF911F075
:1069F8006DF999F80030A8EC010A01359D42F3DBE6
:106A0800FFF7B1BAFC1300204D3C00204C340020A5
:106A1800F83A0020F40D0308FC5500202C3900201A
:106A2800C06000200456002014560020900303087C
:106A3800905D0020D9610020843800200D2A7FF461
:106A48007AAF5A1C32601D78072D3FF674AFDFF815
:106A58002C9330464FF00C08FCF754F908FB05F866
:106A680009EB0805A8803046FCF74CF9E880304669
:106A7800FCF748F9336828811A46591C316012F826
:106A8800021BA97232605B78EB723046FCF722F980
:106A9800012549F808002B46FFF74CBA5A1C32600A
:106AA8001878060600F1B986AD4B1B78DD073FF56F
:106AB8005AAA032828BF00200125FEF7A1F82B4673
:106AC800FFF738BAA64B1B78D8073FF54CAA012523
:106AD800FEF78CF9FEF7A2FE2B46FFF72BBAA04B68
:106AE8001B78D9073FF53FAA9E4B4FF4C872012582
:106AF8001A802B46FFF71EBA092A7FF71CAFDFF86A
:106B080080821A46591CD8F80050316012F8021BCE
:106B1800297032605A78AA70DA1C32609A78642A2E
:106B280003F10401A8BF64226A713160DA78642A2B
:106B380003F10501A8BF6422AA7131601A79EA71CC
:106B48009A1D32605A79642A03F10701A8BF6422AA
:106B58002A7231609A79EA7003F108023260DB79AF
:106B68002B713046FCF7CEF8726833686881D11A09
:106B780000290CDD591CD8F800003160521A002A8F
:106B88001978417203DD9A1C32605B7843700125E5
:106B980025F03EF92B46FFF7CDB9714B1B78DA0784
:106BA8003FF5E1A9704A1378012543F004031370F7
:106BB8002B46FFF7BFB96D4A1068DA1C014621332E
:106BC800951E356012F8035C0D70551E356012F87D
:106BD800025C4D70326012F8015C8D700332934292
:106BE80001F10301ECD110F0FBFEFFF7BCB9C2F3D1
:106BF8004705122D3FF69FAEC5B107F1500307F1C7
:106C08002A0903EB450AC846AAF1260A3046FCF7CA
:106C180079F828F8020FC245F8D1554B39F8022FF8
:106C280023F8022FC845F9D1112D09D8514A6B0014
:106C3800023B13440021223223F8021F9A42FBD15F
:106C48004D4A01231D461370FFF774B9DFF83481EC
:106C580000233046C8F80030FCF73CF80125C8F896
:106C680000002B46FFF766B91A46591C316012F826
:106C7800025B3260DA1C587832609978002D00F097
:106C88001486012D7FF46FA90CF078FA2B46FFF7D4
:106C980051B9334A127812F001017FF44CAE5A1CF4
:106CA8003260187801250CF0B9F92B46FFF742B984
:106CB8003046FCF727F83046FCF724F83046FCF756
:106CC80021F83046FCF72AF83368284D1946581C35
:106CD8002A68306011F8020B82F82C00316059786C
:106CE80082F83610D91C31609B7882F837303046EC
:106CF800FCF714F83046FCF711F83046FCF70EF8AC
:106D08003046D5F80080FBF7FDFFA8F83A0030467A
:106D1800D5F80080FBF7F6FF33687268A8F83800EA
:106D2800D11A01290ADD591C2A6831601B7882F8BA
:106D38002E303046FBF7F2FF33687268D31A032B04
:106D48000BDD3046D5F80080FBF7DCFFA8F83200F1
:106D580030462E68FBF7D6FFB086286843E700BFA9
:106D68004D3C0020127000201C540020F83A0020EE
:106D7800A6580020A8580020CC58002058330020DE
:106D8800F46F0020583700205A1C3260C24DDFF8DB
:106D980034831B7888F805303046D5F80090FBF727
:106DA800B1FFA9F820003046D5F80090FBF7AAFFFC
:106DB80072683368A9F81E00D11A072919DD304610
:106DC800FBF7A0FFA8F80A003046FBF79BFFA8F8DE
:106DD8000C003046D5F80090FBF794FFA9F8220084
:106DE8003046D5F80090FBF78DFF33687268A9F834
:106DF8002400D11A03290BDD3046FBF783FFA8F8DE
:106E08000E003046FBF77EFF33687268A8F8100062
:106E1800D21A002A05DD591C2A6831601B7882F8CD
:106E28002630FDF713FF20F0CDFE9C4B1B68002B8E
:106E380000F0FE84286801250FF0FAFA2B46FFF7C8
:106E480079B81A46591C3160954912F8020BC87076
:106E5800326094495A784A71DA1C3260924A9B78B7
:106E6800D37001252B46FFF765B81A46591C3160C7
:106E7800DFF8508212F8021B88F8021032608B4942
:106E88005A780A70DA1C3260894D9A782A711A1D6C
:106E98003260DB78092BA8BF09233046AB70FBF7BB
:106EA80031FF336872682880D11A012905DD304620
:106EB800FBF728FF33687268E8819A4207D05A1CAA
:106EC80032601B78003318BF012388F80730FDF7BC
:106ED800BDFE336872689A423FF445A85A1C326076
:106EE8001B78EB7001252B46FFF724B83046FBF7DB
:106EF80009FF054613F080FDFF283FF434A83F2D15
:106F080000F2A18407F15008002308F8243D4FEA55
:106F1800D509414607F12B0087F82B3009F1010903
:106F280013F04AFD97F82B305FFA89F905F0070549
:106F38004B4505F1010503D197F82C30AB4203D03E
:106F48002946484613F044FD33687268D21A012A6C
:106F58007FF709A85A1C07F15000326000221D78FB
:106F680000F8252D13F01CFD97F82B30AB420AD002
:106F7800504B1B683BB19A79AA4204D31B681B6922
:106F88000BB12846984733685A1C326040460022A5
:106F98001D7887F82C2013F0F7FC97F82C30AB42BB
:106FA8003EF4E1AF434B1B68002B3EF4DCAF1B689B
:106FB8005B69002B3EF4D7AF28469847FEF7D3BF4E
:106FC8003D4A1278012A3EF6CEAF18465A1C326066
:106FD800DFF8F48010F8022B88F80220DA1C891AEE
:106FE800306001295878326040F344843046FBF71A
:106FF80089FE0125A8F800002B46FEF79BBF5A1C06
:10700800326093F80080B8F1110F3FF694AC9A1CE7
:1070180032602A4D5B7805F818303046FBF772FE6F
:1070280040F6CA039842A8BF184640F2EE23984299
:1070380005EB4801B8BF18460125A0F2EE222B4601
:10704800192092FBF0F24A70FEF774BF1A46591CD9
:107058001B4D316012F8021B297132605B786B712D
:107068003046FBF74FFE336828805A1C32601B7885
:10707800AB713046FBF746FE336868805A1C3260B5
:107088001B78EB7101252B46FEF754BF0125FCF751
:1070980007FA2B46FEF74EBFF83A00202856002084
:1070A80004560020E853002014560020F85500200C
:1070B800905D0020A03B0020E54E0020705A002083
:1070C80044390020C0600020E84E00205A1C32607D
:1070D800C74A1B78DFF8488313700023C8F80030CC
:1070E8003046FBF7F7FD3368D8F80020C149C24D98
:1070F80010435A1CC8F8000032601B780B723046E7
:10710800FBF700FE28603046FBF7FCFD6860304660
:10711800FBF7F8FDA8603046FBF7F4FD3046FBF7B7
:10712800F1FDFEF720BFB54A03F1080101333360D2
:1071380013F8010C02F8010F8B42F7D1FEF713BFC9
:10714800591C1A463160AE4912F8020B8870326039
:107158005B784B7001252B46FEF7ECBE0721B2FB8E
:10716800F1F1C1EBC105521B7FF4E5ABC9B201F1E6
:10717800FF395FFA89F900293EF4F5AEDFF884A2F9
:1071880009F1010915465A1C326093F900109D4B0C
:107198004FF0000893F902208A4203F1080300F037
:1071A800A18208F10108B8F1060FF3D1FFF7C3BBBC
:1071B8005A1C32601A780E2A3FF6BDAB991C316012
:1071C8005D78032D3FF6B7AB8F48062101FB02F12E
:1071D800421803F1030E5571C6F800E09D78455436
:1071E800191D3160D9785170591D31601979917024
:1071F800991D31605979D170D91D31609B7913710E
:1072080001252B46FEF796BE5A1C3260794A1B7838
:10721800537501252B46FEF78DBE3046FBF772FDF0
:10722800DFF8D481C8F800003046FBF76BFDC8F8DA
:1072380004003046FBF766FD0125C8F808002B4618
:10724800FEF778BEDFF8D8810023C8F80030304652
:10725800FBF740FDD8F8003001250343C8F800309B
:107268002B46FEF767BE5A1C32601D78132D3FF679
:1072780062AB9A1C326058787B6221F03BFE002892
:107288003FF459AB7B6A614A017802F82510D91C92
:10729800316002EB850299785170191D3160D878F8
:1072A8009070581D30605A491B79D37008680125C1
:1072B80024F03CFD2B46FEF73DBE5649102A1346E6
:1072C8004FF0000228BF10230A604A608A60CA6033
:1072D8000A74002B3EF447AE326801391344013278
:1072E800326012F8010C01F8010F9A42F7D1FEF74B
:1072F8003ABE591C31601D781F2D3FF61CAB052A7C
:107308007FF419AB3046FBF7E5FC434B43F8250007
:1073180013F0F8F8FEF727BE3F4D05F14008304658
:10732800FBF7F0FC3368A5F88000591C1A46316059
:1073380012F8021B85F8821032605B7885F883307A
:107348000435A845EBD1FEF70EBE5A1C3260294D14
:107358001B782B723046FBF7D5FCA8833046FBF729
:10736800D1FC28833046FBF7CDFC32686883531C78
:1073780033601278EA747268D31A032B00F32E82F2
:107388003368D11A05290EDD5A1C32601B78EB725E
:107398003046FBF79FFC3368E8605A1C32601B7864
:1073A8002B7433687268D21A002A7EF7DCAD5A1C37
:1073B80032601B7885F8213001252B46FEF7BABDCF
:1073C800581C30600A4A1D781570091A00297EF782
:1073D800CAAD991C31605B78003318BF01230125C1
:1073E80053702B46FEF7A6BD0C4BFFF7BFB800BF86
:1073F800445600205C3E0020B03100205B3E002057
:1074080020560020B45A0020643700204856002037
:10741800F83A0020E0550020545000204C24002069
:10742800F04E00203388FF2BA8BFFF23DBB2FEF706
:1074380018BD22F0EDF800283EF412AD03780A2BAF
:107448002FD8B0F9023088FB0312DB17C3EBA20375
:107458009BB2FF2BA8BFFF23DBB2FEF702BD98E863
:107468002200FFF785B822F0D3F800283FF467A878
:1074780003780A2B3FF663A8B0F90430B0F9061078
:1074880003EB830383F3500521EAE171ADB289B2BE
:10749800FFF757B8FB697C681A463B7D1370FFF706
:1074A800C1B90023D8E71A46591C3160BF4D12F8FC
:1074B800021B697032605A782A70DA1C32609B7835
:1074C800AB703046FBF71EFC33682881591C1A46FE
:1074D800316012F8021B697132605B78AB7101256B
:1074E8002B46FEF727BD5A1C32601A780A2A00F08C
:1074F800DF803046FBF712FC3046FBF70FFC012516
:107508003046FBF70BFC2B46FEF714BD5A1C3260C5
:107518001B780A2B00F0C680502B7FF4FCAD304658
:10752800FBF7F0FBDFF8A882A8F800003046FBF76D
:10753800E9FB0125A8F802002B46FEF7FBBC9C4B93
:107548003A6A9B68D4F800905A449A4240F2BF8045
:107558003A6AA3EB0208FBF741FF42464946386AFC
:10756800FBF7BCFF236803442360002D3EF4FBAC0B
:1075780086427EF7F8AC002100E0236801305A1CEF
:10758800864222601970F8D1FEF7EDBC3368726844
:107598009A4240F0D680874BFF221A704FF0000ABB
:1075A800854D0BF06DFB51462022844885F800A0DC
:1075B80028F08BFD87F82CA097F82C30072B00F2C9
:1075C800E980DFF810927D4E524697F82C3003EB95
:1075D800430309EBC3035B7CE3B197F82C3003EB5F
:1075E800430309EBC30320215B699BB197F82C3057
:1075F80003EB430309EBC303586946F82200FAF783
:1076080079FC2B7856F82300FAF736FE2A780132EF
:10761800D2B22A7097F82C300133DBB287F82C30BD
:1076280097F82C30072BD0D92368591C21601A7081
:10763800B8F1000F3EF497AC614BC8F80030012553
:107648002B46FEF777BC002D7FF479AF59462046CC
:10765800FBF79AFB23685A1C22601D70544B26685E
:107668009D683B6A0BEB0302AA4200F21081FBF70C
:10767800B5FE5A463146386AFBF730FF23680125C4
:10768800034423602B46FEF755BC3046FBF73AFB14
:10769800326871687B6A9142834648D106461D4626
:1076A800FFF72DB83046FBF72DFBDFF82C813BE7C1
:1076B8009A1C3260434A59781170D91C3160997804
:1076C8005170191D3160DB789370FEF74CBCFBF7E5
:1076D80085FE5A464946386AFBF700FF236803448B
:1076E800236045E70AEBC80B30468BF80210FBF71E
:1076F80009FB32682AF838001346511C316013F828
:10770800021B8BF80310336053788BF80430D31CBA
:10771800336093788BF80630131D33600135D278C7
:107728008BF805204D457FF42EADFEF71CBC511C8F
:10773800316012781D46131C064618BF0123FEF758
:10774800DEBF5A1C194632601A4811F8022B027023
:1077580031605B784370042A03D9FF2A7EF4AFAB0B
:107768001CE719490978994205D8022A7EF4A7AB83
:10777800FF2B7EF4A4AB236801255A1922601D70E3
:10778800B8F1000F3EF4EFAB104BC8F800302B46B1
:10779800FEF7D0BB524647E7DA46C7F824B0FFF7F2
:1077A80047B87D62AA46FFF743B800BF8C51002056
:1077B800FC1300203C1E002033320020A459002076
:1077C80045550108B74D0020D96100209D3B0008B0
:1077D80048240020D05C0020F45500203046FBF7F8
:1077E80091FAA8843046FBF78DFA33687268E8840A
:1077F800D11A03297FF7C5AD1A46591C316012F812
:10780800021BA97732605B7885F820303046FBF799
:1078180079FA336872686884B3E500F07F0003285A
:1078280028BF002001250BF0C5FC2B46FEF782BBC4
:1078380021482249224A234B036001250B6013602B
:107848002B46FEF777BB07F12C08404613F090F85B
:10785800BB8DAB423FF478AB1B4B1B68002B3FF44E
:1078680073AB1B689B69002B3FF46EAB28469847A7
:10787800FFF76ABB154A99781288012512FB00F2B6
:107888002B4692FBF1F2A8F80020FEF753BB3B6AA7
:10789800ED1AFBF7A3FD2A463146386AFBF71EFEB0
:1078A800236803442360FEF75EBB01250EF056FFF4
:1078B8002B46FEF73FBB00BFC4340020183500201C
:1078C8008035002049080008A03B002014710020E2
:1078D8002DE9F04F2DED028B93B0834619F0C2FBD2
:1078E800B64B1D7825B113B0BDEC028BBDE8F08F07
:1078F800B34B1B685B05F6D5B24FB34E3B68002B04
:1079080057D0B24C3168D4F810218A1A7C2A50D941
:1079180094F81421DFF800839FEDAD8AC4F81011A4
:10792800013284F814214FF0240A5E20984750460B
:107938003B689847A74BF8EC016A9B8A07EE103A18
:10794800F8EEE66AB8EEC77A0AF1010AC6EE877A57
:107958005FFA8AFA67EE887AFDEEE77ACDED027A69
:10796800BDF908905FFA89F022F0ECF9C9F3072015
:1079780022F0E8F9BAF1270F3B68D6D15E20984784
:107988003B6830209847002022F0DCF9002022F0E4
:10799800D9F93B685E20984794F8143113F003082E
:1079A80000F0868113F0070801F03782282B01F0D8
:1079B8002183894B1B78002B72D0844C874AD4F8DA
:1079C8001831ABEB0303934200F27C8794F82091C3
:1079D800B9F1000F35D1DFF84482D8F80000F9F783
:1079E8003BFCC0B201280FD902287D4F41F08183AA
:1079F8003B78002B41F0FF85D4F82431ABEB03032F
:107A0800B3F57A6F81F07087D4F82831002B47D00E
:107A180094F82031C3B9734B1B689B7801211E3B36
:107A280000228B4284F8201184F8342141F2038724
:107A3800D8F800000221043022F0FAF894F82C312A
:107A480011E0D4F828315BB3D4F8303140F6B732BE
:107A5800ABEB0303934223D994F82C31002B01F0AC
:107A6800B282DFF8B881013BDBB284F82C31002BFD
:107A780000F08387D4F8287194F8342117F8011B93
:107A880094F83531D8F80000C4F828710A44013355
:107A980084F8342184F83531F9F7E2FBC4F830B1C1
:107AA800514BD6F800801B7843B1504F386828B145
:107AB8004F4B1B78013B012B40F26F874D4B1B78D6
:107AC80063B14D4F3B684BB1404CD6F80090D4F8A9
:107AD8004C31A9EB0303632B00F21D81DFF84081D1
:107AE80098F80030022B01F036823D4F97F8743039
:107AF800032B00F02C87414B1B7873B1404D2B684A
:107B08005BB1324CF9F7F2F9D4F85831029044F6E7
:107B18001F62C31A934200F259813A4B1B78002B1B
:107B280040F08080384B1B7843B1284CD4F8A832F9
:107B380003F5C333A0339B4580F07286334B1B7823
:107B4800002B3FF4D0AE214E314C324D06F2C927FE
:107B58002068F9F781FB00283FF4C5AE2068F9F7E3
:107B680073FB2B7880465A1E33B120682A70F9F7C8
:107B780073FB0028F2D1B6E603223946781E28F0B6
:107B88008AFA96F8C83296F8C92286F8CB8283F426
:107B98007F4383F0FF039B1A1FFA88F89BB2B8EB68
:107BA800132FD5D196F8CA22DBB29A42D0D1781ECB
:107BB80021F0A8FD2B7818442870C9E7E73A00207F
:107BC800E4600020946400206C570020401E0020D0
:107BD80000007A44243B00205E5200203F0D030041
:107BE8000000002090640020605200207462002091
:107BF80068520020705200201C4700207852002054
:107C08007C520020BC520020CD520020825200201D
:107C1800885200208C5200205C3B00208C6400209D
:107C28009A5900205B4C2278A2B15B4B9B7A53B1E6
:107C3800F9F75CF9594B1B68C31AA3F57A73B3F5C6
:107C4800FA6F07D82278564B56491868F9F7D4FACC
:107C580000232370544CD4F8A03203F5C333A03367
:107C68009B45FFF45FAF514DC4F8A0B22B78002BB1
:107C780041F004834E4D2B78002B41F00B824D4987
:107C880094F8A4228D5CE90701F1BB84AA0701F1ED
:107C980075846B0701F16D83474A94F8A432117813
:107CA800013393FBF1F201FB123384F8A43239E774
:107CB800D4F8102141F288339A4201F2F2813B68EC
:107CC8005E2098473B68142098473C4B3C4AB3F9E0
:107CD800043082FB03124FEAE378C8EBA2080FFADC
:107CE80088F85FFA88F022F02DF8C8F3072022F010
:107CF80029F83B685E2098473B681C20984700207D
:107D080022F020F8002022F01DF83B685E209847FA
:107D180094F8143146E6DFF8A4A0DFF8A4804120E7
:107D280021F034FFBAF9023088FB0320DB17C3EBDC
:107D3800A00080B221F010FFBAF9003088FB0320C0
:107D4800DB17C3EBA00080B221F006FFBAF90430BC
:107D580088FB0320DB17C3EBA00080B221F0FCFEF8
:107D6800184B38681978F9F77BFA94F8503113F002
:107D7800010801F0CF81144AC4F84C910133DBB2F9
:107D8800A2FB0312D20802EB8202A3EB420384F89F
:107D98005031A3E6505200205C3E0020B849002034
:107DA800C052002010520020401E0020C452002063
:107DB800C5520020C8520020CC5200206C3B002045
:107DC8006766666681470020CDCCCCCC94F85E31DE
:107DD800002B41F05A81DB4B1A6802F00803002B94
:107DE80048F603414AF60B404BF60F4349F607475E
:107DF80004BF03460F4612F0040F4FF0190118BFD5
:107E08001F46920684F85E1103D547F4804747F071
:107E18002007CD4B5A79C7F30909002A41F091850B
:107E28009B79002B41F07786984664204FF0FF3A03
:107E38004FF0000C0A970B97ADF834C0CDF83AC054
:107E4800CDF83EC0CDF842C0CDF83090ADF83680C0
:107E5800ADF838A08DF846000AAF0FCFDFF800E381
:107E680084F805C0AEE80F0097E80F00AEE80700F9
:107E78002EF8023B71464FF0010C1B0CFE271F2009
:107E8800C82201F81E39A770A27184F807C0E070F3
:107E980094F86E01207180F0F10383EA0313DAB2DB
:107EA800130983F0E70343EA022383EAC2031BB200
:107EB80083EA0312D2B2C3F3072383EA121343EA15
:107EC800022383EAC2031BB283F0C80282EA0212C9
:107ED800D2B2C3F3072383EA121343EA022383EAE5
:107EE800C2031BB283EA0C0787EA0717FFB2C3F382
:107EF800072282EA171242EA072200EB0C0382EA01
:107F0800C7070EEB0C0084F86E31278011F8013B8F
:107F18007B4083EA0313DBB21A0982EA172242EA9A
:107F2800032282EAC3031BB29FB281422780EDD1AC
:107F380083F07C0383EA0313DBB24FEA131E8EEA55
:107F4800172E8EEA032E8EEAC30E0FFA8EFE1FFA44
:107F58008EFADFF810C2A4F800A05FFA8EFE4FEA8E
:107F68001A2A84F828A084F827E00CF5CB7804F1C5
:107F78002209DCF80000DCF80410DCF80820DCF842
:107F88000C3047460FC70CF1100CCC45B846F0D161
:107F9800DCF8000038606D4F9CF8043088F8043035
:107FA80007F1270884F8BDE184F8BEA117F8011F7E
:107FB8002868F9F755F9B845F8D194F85F31002BDE
:107FC80041F05E806249326809780A2084F85F01CE
:107FD800002901F0C4815F4F01293888069041F2D9
:107FE800A8850229B7F802E001F0C684B888059090
:107FF800032901F09785F8880490042901F0AE85DB
:108008000529388901F0A5850629B7F80A9001F0F5
:108018009C850729B7F80C8001F09485FB890393A8
:1080280094F86E110A920B4683F0300282EA02122B
:10803800D2B217094849079387F07A0747EA022717
:108048000988237187EAC202444FC1EB012187FBEB
:10805800013A069B4FF0000C63F30F0C059B6EF37F
:108068001F4C4FF0000E63F30F0E049BCDF82CC08D
:1080780012B28A440027C91763F31F4EC1EB6A2A5C
:10808800039BCDF830E082EA021160F30F0700206D
:10809800C9B268F30F00C2F3072269F31F4782EAE7
:1080A800111263F31F404FF000090D978DF83DA0A2
:1080B8000E908DF83C9042EA01220DF1280C82EADC
:1080C800C107BCE80F003FB287F0C80888EA081863
:1080D800DFF88CE084F805905FFA88F8C7F3072783
:1080E800AEE80F0087EA181747EA08239CE8030060
:1080F80083EAC8031BB283F023024EF8040B82EA1A
:108108000212D2B2C3F30723079F83EA1213704601
:1081180043EA022383EAC20207F1010C20F814198A
:108128004FF023081621FE27C82384F86EC1228049
:1081380084F807800EF1020EA770E170A371114652
:1081480012E000BF203B00208C510020D71F0020E8
:10815800943B0020506F00208051002003082080AD
:10816800481E0020421E002010F8013B4B4083EAC5
:108178000313DBB21A0982EA112242EA032282EAD5
:10818800C3031BB299B270452180EDD183F0F4038B
:1081980083EA0313DBB24FEA131E8EEA112E8EEA2E
:1081A800032E8EEAC30E0FFA8EFE1FFA8EF8E64FE4
:1081B800A4F800804FEA182C5FFA8EFE84F81EE0BF
:1081C80084F81FC07968BA683868FB6807F5CB7807
:1081D800A8E80F0038697969BA6904F29717A8E81E
:1081E800070004F2B51884F8B5C184F8B4E117F8AB
:1081F800011F2868F9F734F8B845F8D194F866C132
:10820800BCF1000F40F03687D04B94F86E71B3F98B
:108218000010B3F90220B3F904309FEDCD6ADFF8FE
:1082280040E384F805C007EE103A33680A9387F0F4
:108238006A0383EA031306EE901AD9B20B0983F096
:10824800D50343EA012383EAC1031BB283EA03117E
:108258005242C9B207EE902AC3F3072383EA1113E7
:1082680043EA0123F8EEE77AF8EEE66AB8EEC77A51
:1082780083EAC1031BB267EE867A66EE866A27EE4A
:10828800067A002083F0C808CDED0C7ACDED0B6A94
:108298008DED0D7A0E900F90109088EA08160DF16A
:1082A8002809F6B2C3F30728B9E80F0088EA1618B8
:1082B80048EA062888EAC6080FFA88F8AEE80F00E8
:1082C80088F01E0699E8070086EA0616F6B2C8F393
:1082D800072383EA161343EA06238EE8070083EA96
:1082E800C6061C20C8214FF005084FF01E0CFE23BF
:1082F8007A1CE070A17184F8668184F807C0A370C5
:10830800AEF1100127710EF10C00268084F86E2161
:1083180011F8013B734083EA0313DBB21A0982EABE
:10832800162242EA032282EAC3031BB29EB28142AA
:108338002680EDD183F0270383EA0313DBB24FEAEB
:10834800131E8EEA162E8EEA032E8EEAC30E0FFA3D
:108358008EFE1FFA8EFC7C4FA4F800C05FFA8EFEDA
:108368004FEA1C2C84F825C084F824E007F5CB7864
:1083780004F1220938687968BA68FB6846460FC66E
:1083880010374F45B046F5D1724E3B88A8F80030FB
:1083980006F1240784F8BAE184F8BBC116F8011F76
:1083A8002868F8F75DFFB742F8D194F867A1BAF1E9
:1083B800000F40F0598694F86E81644B664AB3F911
:1083C8000410B2F90620654EDFF898E1644F84F88E
:1083D80005A088F0220080EA0010C0B2030983F0EB
:1083E800590343EA002383EAC0031BB2B2F5FA6FCC
:1083F80083EA0310C0B2A8BF4FF4FA62C3F307239D
:10840800B2F57A7F83EA101343EA0023B8BF4FF42A
:108418007A7283EAC000A2F57A72642303FB02F23F
:108428008EFB023ED31786FB0162C9174FF0000C82
:10843800C3EBAE13C1EBA201CDF828C006B2CDF84C
:108448002CC0CDF830C0CDF834C0ADF83A30ADF816
:1084580038100DF1280CBCE80F0086F0C80E8EEA23
:108468000E1E5FFA8EFEC6F3072686EA1E1646EA39
:108478000E260FC786EACE0636B286F04A0383EA8E
:108488000313DBB2C6F3072181EA13113A46DCF87D
:1084980000E042F810E941EA032108F1010681EA07
:1084A800C30305204A214FF0FE0C84F86E614FF09B
:1084B800C80E142684F8670184F8048023800437E2
:1084C800E17184F802C0E67084F806E0184612F8F4
:1084D800011B414081EA0111C9B20B0983EA10234B
:1084E80043EA012383EAC10109B288B2BA42208073
:1084F800EDD181F0140181EA0111C9B24FEA111ED0
:108508008EEA102E8EEA012E8EEAC10E0FFA8EFE2A
:108518001FFA8EF60C4F26804FEA16295FFA8EFE58
:1085280084F81D9084F81CE079683868BA68FB689C
:10853800B7F8188007F5CB7CACE80F003869796983
:10854800ACE8030010E000BF421E00206C3B002096
:1085580088C3E43AD71F0020506F0020676666661C
:10856800481E0020D34D621004F29716ACF8008024
:1085780084F8B391B04684F8B2E104F2B31918F85C
:10858800011F2868F8F76CFEC145F8D1C44BC54AED
:108598001B781278013B12F00100DBB214BFC02136
:1085A8004021172B03D8C04A134493F830A0BF4B7F
:1085B8001A8893071ABF002341F01001012312F40F
:1085C800027F18BF022312F0100F18BF062312F003
:1085D800200F18BF1023002841F060814FF0030CD2
:1085E80094F86E910A9389F0460383EA0313DAB28A
:1085F800130983F0920343EA022383EAC2031BB2FE
:1086080083EA0310C0B2C3F3072282EA101242EAD7
:10861800002282EAC00212B282F0C80E8EEA0E1E52
:108628005FFA8EFEC2F30722002382EA1E1203209D
:108638008DF82CA08DF82FC08DF82D3042EA0E2C25
:108648008DF82E108DF830000AAA07CA8CEACE0ED3
:108658000FFA8EFEDFF868A2E3718EEA0E1CAAE814
:1086680003005FFA8CFCCEF3072E8EEA1C1E4EEA3E
:108678000C2181EACC0C94F808E08AF800200FFA63
:108688008CFC8EEA0C0E8EEA0E1E5FFA8EFECCF380
:10869800072282EA1E1242EA0E22607AA17A94F830
:1086A8000BC0637182EACE0212B2504080EA001E0B
:1086B8005FFA8EFEC2F3072080EA1E1040EA0E2001
:1086C80080EACE0000B2414081EA0111C9B2C0F38C
:1086D800072282EA111242EA012282EAC10212B298
:1086E8008CEA020C8CEA0C1C5FFA8CFCC2F30722A1
:1086F80082EA1C1242EA0C2294F80CE0607BA17B0F
:1087080094F8108084F8049082EACC0212B28EEABF
:10871800020E8EEA0E1E5FFA8EFEC2F3072282EA6E
:108728001E1242EA0E2282EACE0212B2504080EABB
:108738000010C0B2C2F3072282EA101242EA0022F5
:1087480082EAC00212B2514081EA0111C9B2C2F3F1
:10875800072282EA111242EA012282EAC102E17B7F
:1087680013B281EA030282EA0212D2B2C3F30723E8
:1087780083EA121343EA022383EAC2031BB288EA9C
:10878800030282EA0212D2B2C3F3072383EA121366
:1087980043EA022383EAC2031BB283F0320282EA6D
:1087A8000212D2B2C3F3072383EA121343EA022365
:1087B80083EAC2031BB29AB24FF0FE0C4FF0090EC7
:1087C800C82009F10101DBB284F802C084F803E093
:1087D8004FEA122CA07184F86E11228084F812C01E
:1087E800637438687968BA68B7F80C900AF5C47E7B
:1087F800AEE807000AF5CC7A8EF80280AEF8009051
:1088080084F8A8C184F8A73116F8011F2868F8F77A
:1088180027FDB245F8D1029BC4F85831FFF77DB95E
:1088280094F8AC32204AC4F8A8B202EB8302926CE6
:1088380042B312AD04F2B3231D4E45F8203D00218A
:1088480004F2C52331800B9380211523A52784F8D2
:10885800B232284684F8B11284F8B072904728469C
:108868003188FAF791FA0A9D124804F52C716D1AAD
:10887800152DA8BF15252A4625F0A6F90E4A94F805
:10888800AC3215700D4A013382FB0312A2EBE3727E
:1088980002EB42029B1A84F8AC32FFF74FB900BFD3
:1088A800445600204D3C00209407030882510020C4
:1088B800CC5100204C4800206148002056555555A1
:1088C800481E0020D34AD44B92F80BE03168D4F804
:1088D8001C211B88D148891A4FF47A72DFB202FB37
:1088E8000EF21B0A8777077591424FF00007C3778E
:1088F80043758770077180F0EE83C94BC9491A68C0
:108908009B68C4F818B181FB02E7D21781FB03E129
:10891800C2EBA702DB17C3EBA10311124FEA232C0A
:108928004FF0F40E02770127417780F8203030218C
:108938007522782380F821C080F81AE0C77680F87D
:10894800221080F8232080F82430FFF73FB8DFF8A2
:10895800F492D9F80000F8F773FC00283FF4CBA88C
:10896800D9F800000121F8F767FC0222002387F8F4
:10897800742088F80030FFF7BEB894F8341194F8E2
:108988003531D8F800004A1C013384F8342184F8C2
:108998003531F8F765FCFFF781B8A34CDFF8A892EA
:1089A8004FF0000A0AE01B2B00F002830D2B00F0A9
:1089B80012824FF0010389F801303868F8F74CFC4F
:1089C800002838D03868F8F73FFC83B27E2B32682D
:1089D8002AD099F801100029EFD194F83621002AFD
:1089E800E1D07D2B00F00C8294F844E1BEF1000F39
:1089F80004D080F02003DBB284F84411511CC9B2C2
:108A08002244092984F8361182F8383100F0EC81C3
:108A18000829D2D8B4F84221134403EB132303F0F6
:108A2800FF03A4F84231C8E784F836A184F837A1D7
:108A380089F801A0C1E794F8453133B194F8393188
:108A480084F84501302B00F01D8794F83721774BC7
:108A5800DFF8F8C1DFF8F8E1DFF8F8A101271046E0
:108A680000283FF42BA83268A2EB0802012A00F282
:108A7800AD8194F84691B9F1000F40F0B08294F8B6
:108A8800471133F8112012B984F84771E8E701312A
:108A9800B2F5826F84F8471100F002811FD9B2F550
:108AA800E26F00F09A8034D9B2F5046F00F0A48028
:108AB800B2F5116F00F04781B2F5E46FD0D11046DE
:108AC8005B4A176C918A642303FB07F393FBF1F16C
:108AD80021F094F8002384F83731FEF7EFBFB2F5A0
:108AE800007F00F0B9802CD8B2F5807F00F0458176
:108AF800B2F5887FB4D1DCF800205207B0D5002148
:108B08004FF4887021F07AF8002384F83731FEF7A3
:108B1800D5BFB2F5C06F00F0B380B2F5E06F9FD15A
:108B2800434A906B918A642303FB00F34FF4E0609F
:108B380093FBF1F121F062F8002384F83731FEF756
:108B4800BDBFB2F5047F00F02781B2F5806F87D1F1
:108B580094F848310133DBB2032B00F2588142F21A
:108B6800107184F8483101FB03F1324B1B88002B4C
:108B780040F04B810131304B1B78DF072F4B1B88AE
:108B880048BF0431D80748BF0A319A0748BF143193
:108B98001F0648BF2831D80548BF28315A0748BFA3
:108BA80064311F0748BFC831980548BF01F5C8712F
:108BB8009A0648BF01F57A71DF0648BF01F5FA61E8
:108BC800580648BF01F57A614FF4806021F016F825
:108BD800002384F83731FEF771BF1046144AD76B6B
:108BE800918A642303FB07F393FBF1F121F006F864
:108BF80084F83791FEF762BF114BB3F9041001EB0B
:108C080081011046490020F0F9FF84F83791FEF7FA
:108C180055BF00BFC062002088620020905200202B
:108C28007C62002067666666401E00209407030881
:108C3800243B0020C05100204D3C002082510020E0
:108C48006C3B0020205A002000000020203B002020
:108C58008C510020CE6200209EF8061000293FF4B7
:108C6800FFAEC84BC8491B68104681FB0321DB17C0
:108C7800C3EBA10120F0C2FF84F83791FEF71EBFB5
:108C88009EF80620002A3FF4EBAEBE4B4FF4C060BE
:108C9800996820F0B3FF002384F83731FEF70EBF40
:108CA800DCF8002012F020097FF4DAAEB74A116828
:108CB800090600F1C985B64A127B002A3FF4D0AEF6
:108CC80094F84911032900F26686DFE801F032289A
:108CD8001902B04B1B6859799A79DB7901F1407117
:108CE80001EB022101EB0341002384F849314FF4E1
:108CF800826020F083FF002384F83731FEF7DEBE60
:108D0800A54B1A68137A507992781B0403EB002359
:108D180013444A1C84F8492103EB0161E7E79E4BA1
:108D28001A68D379107952781B0403EB0023134493
:108D3800EFE7994B1A689379D07812781B0403EB04
:108D480000231344E5E79EF80520002A3FF488AE87
:108D58009AF8001000293FF483AE904B1B8803EB70
:108D680083035B004FF4116093FBF1F120F046FFA1
:108D7800002384F83731FEF7A1BEDCF80020510744
:108D88007FF56EAE00214FF4807020F037FF00238E
:108D980084F83731FEF792BE9EF80520002A3FF48A
:108DA8005FAE9AF8001000293FF45AAE784B5B7B0F
:108DB800002B00F06F85794B1B8893FBF1F101EBD9
:108DC800810149004FF4047020F018FF002384F853
:108DD8003731FEF773BE4FF0010184F8361184F87D
:108DE8003831A4F84221E8E5B4F84221C2F1FF0283
:108DF80093427FF4DEAD4FF0010384F84531D8E5A6
:108E08004FF0010384F84431D7E50231B3E601237A
:108E180084F8483142F21071A7E63B685E20984713
:108E28003B6802209847FF2020F0F2FB0378FF2BD5
:108E380000F0258590F901304FEAE3785FFA88F869
:108E4800D8B220F07FFF404620F07CFF3B685E20D0
:108E580098473B6803209847FF2020F0D9FB037808
:108E6800FF2B00F00785B0F90830D8B2C3F3072903
:108E7800DFF8348120F066FF484620F063FF98F859
:108E88000530002B40F0A7820AA9454820F01EFFB4
:108E98003B685E2098473B6813209847BDF92880B7
:108EA8005FFA88F020F04EFFC8F3072020F04AFF51
:108EB8003B685E2098473B681B209847BDF92A808D
:108EC8005FFA88F020F03EFFC8F3072020F03AFF51
:108ED8003B685E2098473B68232098474E2020F047
:108EE80031FF002020F02EFF0AA92D4820F0EEFEC9
:108EF8003B685E2098473B6812209847BDF9288058
:108F08005FFA88F020F01EFFC8F3072020F01AFF50
:108F18003B685E2098473B681A209847BDF92A802D
:108F28005FFA88F020F00EFFC8F3072020F00AFF50
:108F38003B685E2098473B6822209847452020F0F0
:108F480001FF002020F0FEFE3B685E20984794F861
:108F58001431FEF72BBDF7F7C9FF124B1B68C01A77
:108F680040F6B833984200F2CA80DFF840A09AF879
:108F780004303A2B00F08F83002388F80030FEF786
:108F8800BABD00BF7C62002067666666E4600020A8
:108F9800C0620020F46F0020F83A002088620020A8
:108FA80080969800A05900208C51002088590020F4
:108FB8003868F8F751F900287FF4FBAC4FF001034B
:108FC80084F83731F9E4C4F8283184F82031DFF81F
:108FD800A48220F061FE94F82C31FEF744BD974935
:108FE800062020F015FC002384F8460184F8373168
:108FF800FEF764BD4FF000093B6884F814915E20C9
:109008003468DFF8748298473B68172098474846C9
:1090180020F098FE8A4BA3FB04239B0BA8FB0312AA
:109028005209C2EB0212A3EB8203D8B220F08AFEE7
:109038003B685E2098473B6818209847814BA3FB04
:1090480004239B09A8FB03125209C2EB0212A3EBEB
:109058008203D8B220F076FE484620F073FE3B68C3
:109068005E209847FEF7A5BC0AF1FF3A84F867A18D
:10907800FFF7D1BB0CF1FF3C84F866C1FFF795B947
:10908800013B84F85F31FFF7B9B8013B84F85E31E2
:10909800FEF793BF6C493A2020F0BAFB2870FEF720
:1090A80041BD3B685E2098473B6810209847404682
:1090B80020F048FE404620F045FE3B685E20984779
:1090C8003B6821209847404620F03CFE404620F06F
:1090D80039FEFEF7F4BD5D4B32681B78C4F81C21DD
:1090E800013B012B3FF609AC102202238270037169
:1090F80003E420F0C1FD01233B70FEF785BC544A10
:10910800B2F8523100210133A2F8523188F8001028
:10911800FEF7F1BC4F4B1B88DA0515D4D80600F1D1
:109128002784990600F133845A0600F13F84180712
:1091380000F14984D90700F1E38413F0020F0CBF52
:109148004FF004084FF00C08434B444A1B78D27880
:1091580003F001030AB143F002035320029320F005
:1091680015FD3F4A128802EB820202EB8202900050
:1091780080B220F0F1FC002020F0EEFC394A3A4998
:1091880012883868C2EBC212520081FB02311144C6
:109198004FEAE27ACAEB612A5FFA8AFA5146F8F78F
:1091A8005FF8324B38681A78029B48EA03082F4B5D
:1091B8008AEA020A002183F800A0F8F751F841462C
:1091C8003868F8F74DF8294B284A1B78386888EA38
:1091D8000303DBB219461370F8F742F894F85031DC
:1091E800002B7EF4C8AD4F2020F0D0FC14F06AF9B3
:1091F80014F068F914F066F901213868F8F730F8C6
:109208001B4A1A4B92F800801B78184A386808F0F5
:10921800010883F0010341461370F8F721F8134B56
:10922800124A1B78386888EA030319461370F8F75E
:1092380017F894F85031FEF79EBD00BFFD9B020859
:1092480073B2E745D34D6210ED0F02088651002036
:10925800401E0020825100204D3C00209C510020DF
:109268008862002080510020030820808147002068
:109278001C5400208C64002089888888AE4EAF4B2F
:1092880000930024A6F13F01AD4BAE4A089106F8C1
:10929800404CAD4909960AA8F9F74EFE089E731C82
:1092A80008933470089B2922591C08911A70089B4E
:1092B800EA22591C08911A70089BC822591C089167
:1092C8000AA81A7023F052FD471C0AA93A460898C2
:1092D80024F07AFC089AD31901330893D455089BD3
:1092E8005A1C08921C70089B5A1C08921C70089BF8
:1092F8005A1C08921C70089B5A1C08921C70089BE8
:109308005A1C08921C70089B5A1C08921C70089BD7
:109318005A1C08921C70089B5A1C08921C70089BC7
:109328005A1C08921C70089B5A1C08921C70089BB7
:109338005A1C08921C70089BFF22591C08911A702D
:10934800089B0122991812A808911A7050F8283D14
:109358009B1B337017F016FE2C70FEF7E3BB884694
:1093680089460846049105918E4606910391FEF7B9
:1093780057BE764A704B12680B93A3F14005002044
:109388002121D70003F8400CA97040F1CE82704922
:109398000326704B1B88580500F1C482DA0700F1D8
:1093A800F38203F002036C4A002B1CBF032611460C
:1093B8006A4F3246384624F007FCF31912A80133E5
:1093C800B91E40F8203D00225B1AF2556B7017F069
:1093D800D9FDFEF761BC624B93F800A0BAF1000F0B
:1093E8003FF452AD5F4AB4F816E111883B68029227
:1093F8004FEA0E1E64201FFA8EFE00FB01A14FEA01
:109408004A00B1FBF0F14EEA012E1FFA8EFEC1F3BD
:1094180003215E204EEA010998473B6806209847D9
:109428005FFA89F020F08EFC4FEA192020F08AFCC0
:10943800B4F81631029A4C49B2F800904A7A0133CE
:109448009BB2012A93FBFAF00AFB1033A4F81631F9
:1094580000F0BD826E2345484A7B03FB09F380FB7D
:1094680003014FEAE379C9EBA1092AB13C4B1FFA82
:1094780089F91B7899FBF3F93B68DFF8FCA05E20BB
:1094880098471FFA89F93B683A209847AAFB093A96
:109498004FEA5A1A1FFA8AF3D8B2029320F052FC04
:1094A800029B180A20F04EFC3B685E2098473B68F8
:1094B8003B209847642303FB1A939BB22C4805333F
:1094C80080FB0320DB17C3EBA000C0B220F03AFCFE
:1094D800002020F037FC3B68DFF898A0DFF8909078
:1094E8005E2098473B6828209847DAF8003089FBC7
:1094F8000329DB17C3EBA9095FFA89F020F022FCE6
:10950800C9F3072020F01EFC3B685E2098473B68A3
:1095180004209847B8F80830002B40F04B82DAF85E
:10952800083083F310085FFA88F020F00BFCC8F3CA
:10953800072020F007FCA7E410520020F13A002091
:10954800E82E0308F02E0308FC2E0308145400200C
:10955800D42E030882510020E42E0308D3510020A2
:10956800CE62002088620020C0620020310CC33027
:10957800676666667C6200201F85EB51CC4ACD4B3E
:109588000B9212AEA2F13D0046F8200D1988CA4F81
:10959800A2F1400300204FF00A0E02F8400C082206
:1095A80083F801E030469A70F9F7C8FB3B68C34975
:1095B800DA1781FB0313C2EBA30399B23046F9F71C
:1095C800BDFB07F08FFBBF680A9B3A0C591C0A9138
:1095D8001A700A9B3A0A591C0A911A700A9B5A1C5B
:1095E8000A921F700A9B5A1C0A921870304617F08C
:1095F800C9FCFEF74EBBC4F824B187F80090FEF70B
:1096080003BAAF4F9FEDAF8AB7F90220A8480B9075
:1096180007EE902AF8EEE77A12AE67EE887AA0F1A4
:109628003D01FDEEE77A46F8201D00F8403C08238E
:10963800CDED027A00F83F3C1E23BDF8081000F873
:109648003E3C3046F9F77AFBB7F9003007EE903A1E
:10965800F8EEE77A304667EE887AFDEEE77ACDEDE8
:10966800027ABDF80810F9F769FBB7F9043007EE7C
:10967800903AF8EEE77A304667EE887AFDEEE77AB8
:10968800CDED027ABDF80810F9F758FB304617F00F
:1096980079FCFEF7FBBA9AF80240C4B1013CE4B287
:1096A800013454445146002211F8013B534083EAE7
:1096B8000313DBB2120ADF0042EA03228C4287EA74
:1096C800131382EA0302EFD1002A7FF455AC794ADA
:1096D8007D4F794B12887D4CFA61DFF804921A6845
:1096E800FA629B68B4F85221F8660021FB64D9F845
:1096F8000000F963FA65F6F7FFFD029000287EF492
:10970800F5A90221D9F80000F7F796FD94F854312D
:109718009AF803200392642B4FF0040287F8742010
:1097280040F0648194F85531072B04BF9DF8083048
:1097380084F8553194F85531069307EB031ADAF893
:1097480004100291084623F011FBDAF8081005917D
:109758005FFA80FA084623F009FBC0B204900AEBCE
:109768000002069B5A48029902900832C27123F0FF
:109778000F0286468272049803F00F0300EBCA00BA
:109788008EF80D3052468EF80E000EF10F0024F0C0
:109798001BFA504B049A05990AF10900184424F061
:1097A80013FA0298C37903F1010ACBB1013B5FFABE
:1097B80083FC0CF1080CDFF82CE18444002307300B
:1097C80010F8011B59408B00CA0883EA410302F0D4
:1097D80018024B404EFA02F253408445DBB2EFD1F7
:1097E8003C4A03980AF8023013F03AFE94F85531CF
:1097F8000022013384F8553184F85421029BDDF8A6
:1098080008A09B785BB11AF80510D9F80000F7F7A3
:1098180027FD01359AF80230EDB2AB42F3D894F83F
:1098280054310322013384F8543187F8742088F8BE
:109838000020FFF78EB80221D8F80000F7F7FCFCEB
:1098480094F82C31FEF70FB91023042218460AA900
:109858008DF82A908DF82B908DF82C908DF82D90FE
:109868008DF828308DF8292020F0A8F984F8379150
:10987800FEF724B94FF000094846FFF7F9BA404609
:10988800FFF7DFBA1449881F20F066F884F846010C
:10989800FFF7DBB8074B1988FFF791BA0F4AD27860
:1098A800002A0CBF4FF0040C4FF0050CFEF798BED1
:1098B80010520020886200207C620020676666667D
:1098C8006C3B002058A08B4100000020401E002067
:1098D800F4460020FA460020801F00209C510020FA
:1098E800205A00200007090E0123D8F800003B7019
:1098F800F7F7AAFC0746D8F80000F7F7A5FC7F069B
:109908007EF482A88E287EF47FA894F82031002B5C
:109918007EF497A8944BC4F828312D2384F82C3171
:10992800FEF779B80326914942E5914B914A1B68A5
:10993800914903F48003834216BF11460426032687
:1099480027E58E499A790B8803EB830303EB83039E
:109958004FEA83081FFA88F8002A00F0D580884B60
:109968001B680FFA83FA07F0BDF940B2FEF760BA38
:109978004FF03408FFF7E8BB984699461846049319
:1099880005930393FEF74CBB7E49042610E54FF080
:109998002408FFF7D9BB4B1CDBB2042B84F84931F0
:1099A8004FEA01617FF4A3A9FFF79EB94FF01008B1
:1099B800FFF7CABB07F096F920F0C4F9002020F0A1
:1099C800C1F9FFF761BA4FF02008FFF7BDBB3B684C
:1099D8005E2098473B68392098475FFA89F020F065
:1099E800B1F94FEA192020F0ADF974E597F875A0A0
:1099F800654904951AF00F0F04BF0AF1010A5FFACE
:109A08008AFABAF1070F28BF4FF0010A4FEA0A1C79
:109A180007EB0C03187C5D4B02930A18002392F89D
:109A280024105A4A93725FFA8CF31A46584B96469A
:109A380007EB0C024EEA000001291870D26803F106
:109A480001000CD90239C9B28D1C1D44034603F824
:109A5800012BAB424FEA1222F9D101310844BC4430
:109A680022F060030AF1010A9CF811205FFA8AFAD1
:109A78001343BAF1080F037000F1010347D04FEA0E
:109A88000A1C07EB0C01424A087C3F4901449A1A18
:109A980091F8241055180EF1100E132D5FFA8EFE52
:109AA800C6DD049D0298DFF8F0E0D1B28B1DDBB271
:109AB80043F04002C27103F1010CCBB14B1DDBB284
:109AC8000833C31804930EF10100002310F8011B9A
:109AD80059408B0083EA4103CA084B402D4902F0E4
:109AE800180241FA02F25340049A8242DBB2EDD1E5
:109AF80003980CF80E3087F875A013F0B1FC7DE6DA
:109B08004FF00808FFF720BB4FF0FF3329E7204A42
:109B1800049D9A1AC6E71A4B9046B3F900A0642030
:109B2800FEF786B998469946184604930393FEF7BC
:109B380077BA984699461846049305939E46039328
:109B4800FEF76EBA0393FEF76BBA98460393FEF7D7
:109B580067BA984699460393FEF762BA98469946BB
:109B680018460393FEF75CBA90520020D82E0308DB
:109B7800E4600020D42E0308CC2E0308886200205D
:109B88007C620020DC2E030894070308F4460020BA
:109B9800014700200007090EFA4600202DE9F04F82
:109BA8002DED0C8B3C4B1B7895B0012B099001F0E7
:109BB8006D863A4C94F80021002A41F0C180072BA9
:109BC800374D01F05E86002305936B68344898474B
:109BD800002800F06981B5F8B470002285F8552096
:109BE800002F40F04387B5F93E00AA6AB5F93C60FA
:109BF800696AB5F94030DFF8B4B0821AE86A6A6376
:109C0800711A1B1A2963274895F85610AB6315F08B
:109C180019F8DBF80030990040F1F080D5ED0D5AC5
:109C2800D5ED0C7A204A94ED656AD4ED666A94ED18
:109C3800677AD4F8A0311268B8EEE58AD5ED0E5AE5
:109C4800F8EEE77AF8EEE58A013377EE867A38EEB1
:109C5800268A78EE878A9342C4ED657A84ED668A0F
:109C6800C4ED678AC4F8A03101F0D0830A4B1F788D
:109C7800142F02F011870023D4F8A8610693062E4A
:109C880000F2AF80DFE816F0D81535156A149D1676
:109C980014004915CE1400BFF86100200C210020E3
:109CA8003065002060650020044A0020E460002040
:109CB800D84B1A78D4F8ACE1DFF8D0C39FEDD67A48
:109CC8004FEACE000CEB000383ED007A002A7DD02A
:109CD800D249B0EE476AF0EE476A0023F1EC017A08
:109CE800013367EEA77A05EE903AB4EEE77AF1EE23
:109CF80010FAF8EEE55AB8BFB0EE677A934276EEFE
:109D0800A76AA7EEA56AE9D1F5EEC06A0CEB0003D5
:109D1800F1EE10FA83ED007A58DDC6EE265AC04BF4
:109D2800C04A1288F7EE007A75EEE75AD3ED007A4A
:109D380065EEA77AFDEEE77A17EE903A812B43F3AA
:109D48001C859342A8BF134607EE903AF8EEE77ACF
:109D5800B54B00EB0E0103EB810393ED057AD3EDD0
:109D6800003A93ED066A93ED014AD3ED046AD3ED08
:109D7800034A93ED025AA3EEA77AA4EE276A66EE89
:109D8800C76AA7EE646ABDEEC77AE5EE276A17EEE2
:109D9800101A812983ED056AC3ED066A43F3EA8444
:109DA8008A42A8BF0A4607EE902AF8EEE77AFCEE48
:109DB800E77ACDED077ABDF81C300CEB00029380F2
:109DC800BEF1000F02D1132F04F05181152F42F07C
:109DD8001A846044DFF8B882838828F81E30D4F8E3
:109DE800A861924B013683FB06239A19F317C3EB3C
:109DF800A203C3EBC303F61AC4F8A8618C4B1B7803
:109E0800002B01F0A3808B4EDFF88892DFF880A248
:109E180006F5BC780027884BD5ED087A1B78172BF8
:109E280001F08E8396ED007AB8EEC78A082B28EEEB
:109E3800278A07D1B0EE480A069324F039F8069B22
:109E48002AF81700DBF8002092000BD5002F04F049
:109E58001F84B0EE480AD5F8143208F1700098470C
:109E6800B0EE408AB0EE480AD5F83431A8F1700057
:109E78009847D5F8A431404698476F4B1B78032B79
:109E8800B0EE408A01F05683D6F8F800D5F8B8301D
:109E9800B0EE480A98470137032F08F12408A9ECC7
:109EA800010A06F10406B6D1634B93F80090B9F1A4
:109EB800070F00F0988694F8B831002B40F0A08680
:109EC8005E4B5B79002B40F0CB8501235A4A84F81E
:109ED800B8311278072A02F0238000230B93584BDD
:109EE80094ED709A93ED007A564BD4ED6FCAD3F87F
:109EF80000A0554B0693F7EE007A37EEC9CA534BCC
:109F080008932CEE07CA524B0A93B4EEE7CA514B9A
:109F180007930025F1EE10FA4F4BDFF87C91DFF83C
:109F28007CB1DFED4E8A9FED4EAADFED3BBADFED47
:109F38004D9A9FED4DBADFED4DAADFF864814C4F85
:109F4800059388BFB0EE67CA2E464A4B99ED008A42
:109F58002B44D3ED007AF5EE407AF1EE10FA17D0E3
:109F6800454B2B44D3ED006A38EE667AB0EEC76AEB
:109F7800F4EEC67AF1EE10FA08D5B5EEC07AF1EE35
:109F880010FACCBF37EEA68A36EEE78A83ED008A50
:109F9800069B1A88930700F08580022E00F08280C5
:109FA8009AF82E10354B07EE901A2B4493ED007A51
:109FB8004B42F8EEE76A07EE903A26EE877AF8EE1B
:109FC800E77AB4EEE77AF1EE10FA0AD407EE901ABF
:109FD800F8EE677AF4EEC77AF1EE10FA88BFF0EE81
:109FE800477A274B274903EB460331F91600B3F9A3
:109FF8000C30C01A07EE100AB8EEC77AD007E7EEA1
:10A00800687A40F10586204B93ED008A27EE888A0E
:10A0180048E000BF0A4A0020000000000C21002090
:10A028000C4A0020084A0020404C00209324499202
:10A03800014A002060650020F8610020C06000200F
:10A04800D4350020F83A0020825100207800002002
:10A058004D3C0020D460002020540020CDCCCC3DC5
:10A06800AE47813F0000C84200003443610BB63B55
:10A078002C540020C8350020D0220020782200204F
:10A08800045600206C3B0020B0350020284C0020EE
:10A09800FC610020D860002010220020C03400207D
:10A0A80038540020079B94F8D0212B44D3ED01DAD3
:10A0B80038EE6DDA002A3DD0D24BD4F8D421099974
:10A0C8001B688A1A9A4235DD9AF84830022B01F04B
:10A0D8009B87022E04F08782CB4B1B68990740F1BF
:10A0E8001C87CA4BCA49DFF890E331F916C09EEDC8
:10A0F800008ADFF888E3C7ED00BA03EB460028EED4
:10A10800288AB0F90C00A0EB0C0007EE900AF8EED4
:10A11800E77ADEF8000027EE888A904238EE6DDA9A
:10A12800C1F22681F7EE007AB4EEE79AF1EE10FA62
:10A1380001F1F580B74B2B4493ED000A059B2CEEFB
:10A14800800A022E20EE0D0AA3EC010A059304F002
:10A158001182089B9BED007AD3ED007AAE4BD7EDC8
:10A16800006A93ED006AAD4B67EE277A2B4427EE21
:10A178008C7AD3ED007A67EE277AF0EE665AEDEE28
:10A18800275AB1EE467AB4EEE57AF1EE10FA08DC19
:10A19800F4EEC65AF1EE10FA8CBFB0EE467AB0EE85
:10A1A800657A94ED706AF7EE007AB4EEE76AF1EE3C
:10A1B80010FAACBF0123002343B1F0EEE66AF0EEDB
:10A1C800C77AF4EEE67AF1EE10FA01D587ED007A57
:10A1D800022E04F09081924A924B52F826001B6896
:10A1E800B0EE6D0A9847904A904B52F826001B68CB
:10A1F80098479AF8373023B1069B1B88002B00F04C
:10A208006B85B0EE6B8A8A4B9BED007A38EE400A7C
:10A218002B4493ED008A83ED000A9AF8483030EE1B
:10A22800480AC0EE077A2BB30A9B1B78DB0721D5B7
:10A23800B7EE007AB4EEC79AF1EE10FA04DB94F8A0
:10A24800D031002B00F05587D4F8D431099AD31AAD
:10A258006C4A12689A420DDD764B93ED007AB0EEA7
:10A26800CDDAB4EEC7DAF1EE10FA41F19D800023A1
:10A2780084F8D031704B94F8E0212B4493ED007AA8
:10A288002CEE877A67EE277AC8ED007A32B9059BFB
:10A29800C7ED00BA43ED01BAC8ED00BA0136032E86
:10A2A80009F1040908F1040807F1040705F1040598
:10A2B8007FF44BAE614B1B78072B01F03383012BE6
:10A2C80001F01B86002794F8E831002B40F0EF8559
:10A2D8005B4A5C4B10681B6810F4805A93F82C306A
:10A2E80040F05E86584A594992ED006A498B584AAF
:10A2F80084ED7E6A92ED007A564A84ED7F7A07EE05
:10A30800901AF8EEE76AD2ED037A534A84ED7C6A34
:10A3180037EE467A77EEE67AD2ED006A84ED7B7AFC
:10A32800012284F80022C7EEA65A4C494C4A91ED06
:10A33800005A4C499FED4C6A91ED004A4B49DFEDBC
:10A348004C6AD1ED004A92ED007A35EE045AF7EEE8
:10A35800007AF4EEE75A35EE245AF1EE10FA88BF87
:10A36800F0EE675A25EE065AF4EEE65AB1EE476A61
:10A37800F1EE10FAB4EEC65AB8BFF0EE665AF1EE36
:10A3880010FAC4ED815A01F1CE80B4EEC75AF1EE4D
:10A3980010FA88BFB0EE475A304ADFED336AD2ED83
:10A3A800017A304A92ED014A304A77EE847AD2ED4A
:10A3B800014A77EEA47A67EEA67AB4EEE76AF1EE80
:10A3C80010FA08DCB4EEE77AF1EE10FA8CBFB0EEC2
:10A3D800676AB0EE476A214ADFED236AD2ED027A56
:10A3E800204AD2ED024A234A77EEA47A92ED007A07
:10A3F80067EEA67AB1EE473AF4EEC37AF1EE10FAB8
:10A4080047D43DE0DC350020203B002004560020E6
:10A418006C3B002084350020F83500209035002062
:10A42800C8340020C43400201C3500201835002012
:10A43800E4220020E83500209C350020F861002047
:10A44800E4600020F83A00207C5400205C3E0020A4
:10A45800D4550020D0620020343900202054002038
:10A46800FC3500202C5400206F12833A3854002009
:10A478000000000000360020B0350020D83500204C
:10A48800F4EEC77AF1EE10FA8CBFB0EE473AB0EEB0
:10A49800673AF04A52780AB9B1EE433A002B41F0D4
:10A4A8006283F7EE003AEC4D2A78002A02F05486CF
:10A4B800EA4BDFEDEB6AD3ED024A93ED017AD3ED77
:10A4C800037A66EE244AE5EE074AE3EE274A63EE8E
:10A4D800A44AF4EEE64AF1EE10FAB4BFB0EE664ACA
:10A4E800B0EE644A98BFF0EE646A012ACDED0C4ADA
:10A4F80002F0578693ED067AD3ED052AD3ED077A55
:10A5080026EE077AA5EE227AA3EE277A23EE877A3B
:10A51800B4EEE67AF1EE10FAB4EEC47A8CBFF0EE3F
:10A52800667AF0EE477AF1EE10FA98BFF0EE676AB5
:10A53800B4BFF0EE447AF0EE477A022A8DED0D7A38
:10A5480000F0DE8093ED0A7AD3ED092A93ED0B4AE9
:10A5580026EE077AA5EE227AA3EE047A23EE877A0E
:10A56800B4EEE67AF1EE10FAB4EEE77A8CBFB0EE0C
:10A57800664AB0EE474AF1EE10FA98BFF0EE446A28
:10A58800A8BFF0EE477A032A8DED0E7A00F0B88066
:10A5980093ED0E7AD3ED0D2A93ED0F4A26EE077A46
:10A5A800A5EE227AA3EE047A23EE877AB4EEE67A51
:10A5B800F1EE10FAB4EEE77A8CBFB0EE664AB0EE70
:10A5C800474AF1EE10FA98BFF0EE446AA8BFF0EEE1
:10A5D800477A042A8DED0F7A00F0928093ED124AA3
:10A5E800D3ED112A93ED137A26EE044AA5EE224AFA
:10A5F800A3EE074A23EE844AB4EEE64AF1EE10FAD7
:10A60800B4EEE74A8CBFB0EE667AB0EE447AF1EE6B
:10A6180010FA98BFF0EE476AA8BFF0EE447A052A10
:10A628008DED104A6CD093ED164AD3ED152A93EDB3
:10A63800177A26EE044AA5EE224AA3EE074A23EE2D
:10A64800844AB4EEE64AF1EE10FAB4EEE74A8CBF5B
:10A65800B0EE667AB0EE447AF1EE10FA98BFF0EEFA
:10A66800476AA8BFF0EE447A062A8DED114A47D012
:10A6780093ED1A4AD3ED192A93ED1B7A26EE044A74
:10A68800A5EE224AA3EE074A23EE844AB4EEE64A30
:10A69800F1EE10FAB4EEE74A8CBFB0EE667AB0EE8F
:10A6A800447AF1EE10FA98BFF0EE476AA8BFF0EED0
:10A6B800447A072A8DED124A22D093ED1E7AD3ED03
:10A6C8001D2A93ED1F4A26EE077AA5EE227AA4EEFC
:10A6D800037A27EE237AB4EEE67AF1EE10FAB4EEB6
:10A6E800E77A8CBFB0EE666AB0EE476AF1EE10FA10
:10A6F8008DED137A98BFF0EE466AA8BFF0EE477A60
:10A7080077EEE67AF7EE006AF4EEE67AF1EE10FA02
:10A71800C4ED707A43F3908486EEA77A022ADDEDC1
:10A728000D7A67EE244A67EE877ACDED0C4ACDEDB7
:10A738000D7A2DD0DDED0E7A67EE877A032ACDEDFE
:10A748000E7A25D0DDED0F7A67EE877A042ACDEDF3
:10A758000F7A1DD0DDED107A67EE877A052ACDEDE8
:10A76800107A15D0DDED117A67EE877A062ACDEDDD
:10A77800117A0DD0DDED127A67EE877A072ACDEDD2
:10A78800127A05D0DDED137A27EE877A8DED137AEC
:10A79800344B1E6816F0805601F09180F6EE005A90
:10A7A800C4ED815A002A02F0CC842F4BD4ED7F4AA5
:10A7B80093F8038094F900320A99D4ED7E6A91F8EF
:10A7C80000E0DFF8B0C02949DFF8AC90B1F9061015
:10A7D8009CED007A059106EE103AFDEEE44A244B12
:10A7E80099F80090B3F81AB094ED7B5AD4ED7C7ABE
:10A7F80014EE903AFDEEE64A00F0100C00F48000EA
:10A808000EF0010EB8EEC66A14EE901A0690B8F172
:10A81800000F41F0EB81DFF84480BCF1000F41F0FC
:10A82800968098ED007ADDED0C6ADFF850C025EED1
:10A83800877AA6EE267AF0EE676AE5EE076ABDEE3D
:10A84800E67A17EE106A17EE100A9E42A8BF18465D
:10A8580016E000BF44560020D9610020A43800202B
:10A8680000000000145400209C510020506F00206C
:10A878005C3E002080380020B45D00205454002045
:10A88800B142C8BF084607EE100AB8EEC77A012AD7
:10A898008CED007A00F0DC8098ED047ADDED0D6A2D
:10A8A80025EE877AA6EE267AF0EE676AE5EE076A65
:10A8B800BDEEE67A17EE106A17EE100A9E42A8BFA0
:10A8C8001846B142C8BF084607EE100AB8EEC77A64
:10A8D800022A8CED017A00F0BB8098ED087ADDED54
:10A8E8000E6A25EE877AA6EE267AF0EE676AE5EE1E
:10A8F800076ABDEEE67A17EE106A17EE100A9E4256
:10A90800A8BF1846B142C8BF084607EE100AB8EEFD
:10A91800C77A032A8CED027A00F09A8098ED0C7AB7
:10A92800DDED0F6A25EE877AA6EE867AF0EE676A85
:10A93800E7EE056ABDEEE67A17EE106A17EE100A22
:10A948009E42A8BF1846B142C8BF084607EE100A83
:10A95800B8EEC77A042A8CED037A79D098ED107A8C
:10A96800DDED106A25EE877AA6EE867AF0EE676A44
:10A97800E7EE056ABDEEE67A17EE106A17EE100AE2
:10A988009E42A8BF1846B142C8BF084607EE100A43
:10A99800B8EEC77A052A8CED047A59D098ED147A66
:10A9A800DDED116A25EE877AA6EE867AF0EE676A03
:10A9B800E7EE056ABDEEE67A17EE106A17EE100AA2
:10A9C8009E42A8BF1846B142C8BF084607EE100A03
:10A9D800B8EEC77A062A8CED057A39D098ED187A40
:10A9E800DDED126A25EE877AA6EE867AF0EE676AC2
:10A9F800E7EE056ABDEEE67A17EE106A17EE100A62
:10AA08009E42A8BF1846B142C8BF084607EE100AC2
:10AA1800B8EEC77A072A8CED067A19D098ED1C7A19
:10AA2800DDED136A65EE875AE6EE265AE5EE257ADD
:10AA3800FDEEE77A17EE900A8342A8BF03468142EB
:10AA4800C8BF0B4607EE903AF8EEE77ACCED077AE6
:10AA5800BEF1000F40F03882002A40F0308233E225
:10AA6800AB4B1B78013BDBB2FFF730BAA94B07931E
:10AA78004FF47A761B68B6FBF3F3C3EB4316A6498B
:10AA8800DFF8B88291F801A0A449B8F9060091F856
:10AA9800009003EB8603DE00B6B2B74202F0E48012
:10AAA800D5F88810B5F93CE0EB6E4A1C07EE90EA41
:10AAB8007344012AC5F88820EB66F8EEE77A02F0BD
:10AAC800DE80D5ED1E5AD5ED206A07EE102A37EE46
:10AAD800E56AB8EEC75A012F86EE057A37EE257A71
:10AAE80077EEC77A85ED1F7AE7EE866A85ED1E7ADE
:10AAF800F0EE667AC5ED216AC5ED206A02F094840D
:10AB0800D5F89C10B5F93EE02B6F4A1C07EE90EA89
:10AB18007344012AC5F89C202B67F8EEE77A02F007
:10AB2800C780D5ED235AD5ED256A07EE102A37EEF2
:10AB3800E56AB8EEC75A012F86EE057A37EE257A10
:10AB480077EEC77A85ED247AE7EE866A85ED237A73
:10AB5800F0EE667AC5ED266AC5ED256A02F098849E
:10AB6800D5F8B010B5F940E06B6F4A1C07EE90EAD3
:10AB78007344012AC5F8B0206B67F8EEE77A02F053
:10AB8800B080D5ED285AD5ED2A6A07EE102A37EE9F
:10AB9800E56AB8EEC75A012F86EE057A37EE257AB0
:10ABA80077EEC77A85ED297AE6EE276A85ED287A69
:10ABB800F0EE667AC5ED2B6AC5ED2A6A02F05C8470
:10ABC800A8F80600B5F8B430544A013B92F8009052
:10ABD800A5F8B43007990023B9F1070F4B608B60D3
:10ABE800CB607FF468A9F6F781F9059BDFF84C8103
:10ABF800C01A94F8B831A8F80000002B3FF460A9F7
:10AC0800013B84F8B83115B0BDEC0C8BBDE8F08F72
:10AC180094ED5E7AB1F90000D4ED5F6AB1F902E013
:10AC28003F4AF4EEC76A80EAE0738EEAEE71A3EB5E
:10AC3800E073F1EE10FAA1EBEE71B8BFF0EE476ADF
:10AC48008B42B8BF0B4607EE103A1378B8EEC77AB6
:10AC580027EE287A002B40F01D82324B93ED006AD4
:10AC6800B4EECA6AF1EE10FA41F1DC80F7EE005A50
:10AC780075EEC65A3BEE477A65EEAA5A2A4BA7EEFE
:10AC8800256A93ED007A26EE076AB5EEC06AF1EE02
:10AC980010FA40F21086C9EE865AB7EE007AB0EE86
:10ACA800476AA6EEE56AF0EE466AF4EEC76AF1EE88
:10ACB80010FA88BFF0EE476AF5EEC06AF1EE10FAB6
:10ACC800B8BFF0EE6B6A194B93ED007A67EE877A9E
:10ACD800A7EEA68AFFF7E6B9154B164A2B4493ED63
:10ACE800007AD2ED007A144B67EE277AF7EE006A05
:10ACF800F4EEE67AF1EE10FA93ED007A88BFF0EE02
:10AD0800667A67EE877A27EE888AFFF77CBA00BFF3
:10AD1800F8550020D4600020C0600020F8610020B1
:10AD2800BC350020C4350020B8350020B4350020DB
:10AD380084220020AC350020A8350020FC610020CA
:10AD4800072B02F029820026DFF83CB3B64DDBF86A
:10AD58000030590501F16B80B44B1B78002B40F093
:10AD6800F381B34F94F8123123B1B24A1288920793
:10AD780042F0A88194F81821002A41F06280BB7F34
:10AD8800002B00F0F383022B02F01680032B01F056
:10AD9800BE82A94B5B88F97F0231C9B2002A01F053
:10ADA800FC87002B01F0F987A4480068B3FBF0F397
:10ADB8000FFA83F9A4F84891002903F0458107EEBA
:10ADC800909AF8EEE77AF7EE006A86EEA77A9C4B3F
:10ADD8000129D4ED576AD3ED007A77EEE67A67EE6B
:10ADE800877AC4ED537A21D0D3ED017AD4ED586A2D
:10ADF80077EEE67A022967EE877AC4ED547A15D0A1
:10AE0800D3ED027AD4ED596A77EEE67A032967EE34
:10AE1800877AC4ED557A09D0D3ED037AD4ED5A6A0E
:10AE280077EEE67A67EE877AC4ED567A8548007839
:10AE3800092803F02D81B9F1000F40F39E8391B3E7
:10AE480094ED577AD4ED537A77EE877A0129C4EDD9
:10AE5800577AC3ED007A21D094ED587AD4ED547A1C
:10AE680077EE877A0229C4ED587AC3ED017A15D0B6
:10AE780094ED597AD4ED557A77EE877A0329C4EDA3
:10AE8800597AC3ED027A09D0D4ED5A7A94ED567AFC
:10AE980077EE877AC4ED5A7AC3ED037A013902292D
:10AEA800B8BF0221C9B2002A18BF022166E30A9B73
:10AEB800654D1B78DE0700F163812A7822B1920084
:10AEC8006249634822F080FE624B1B68002B40F009
:10AED8002E83614B1B789BB1287870B1DFF87081A5
:10AEE800DFF8A8910026F0B2D9F80030B8EC010AD2
:10AEF8009847287801368642F5DB584B1B689847F7
:10AF0800504B1B78072B00F0DF84012384F80031B5
:10AF180015B0BDEC0C8BBDE8F08F514BC7ED00BAF6
:10AF28001B689342BFF6FEA84E4B1A88002384F88C
:10AF3800D031002A41F08E864B4A4C4B1178186864
:10AF480081F00101F7F7B2F9FFF7F4B8484EDFF8DE
:10AF5800409106F5F47806F51577F6EC017A95ED4B
:10AF6800080AD5F81432F8EEE77A404627EE800A48
:10AF78009847A8F1E000D5F834319847A8F1700057
:10AF8800D5F8A4319847D6F8F400D5F8B8309847E2
:10AF980008F124084745A9EC010ADED1FEF784BF71
:10AFA8000A9A1278D50703D4214A128BA4F8F421FF
:10AFB800304A2349128891ED037A07EE902AF8EE79
:10AFC800E77AB4EEE77AF1EE10FA41F281802A4985
:10AFD800098807EE901AF8EEE77AB4EEE77AF1EE10
:10AFE80010FAC0F2E7872549254AD1ED006A92EDAB
:10AFF800006A2449C4ED7E6ABCEEC75A76EE665AEA
:10B0080015EE102AC4ED7C6AC4ED7B5A84ED7F6A84
:10B01800A4F8F4210122D1ED006A84F8002277EE29
:10B02800677AFFF780B900BF30650020221C002036
:10B038005C3E002082510020943B002028560020CE
:10B04800D0620020F8610020D961002084380020F7
:10B0580054540020BC340020BC600020B05D0020A7
:10B06800D835002044570020465700204857002074
:10B0780060650020383900203A3900202439002042
:10B08800D455002040390020E4600020A85D00204D
:10B09800D8600020CC4B93ED005AB5EEC05AF1EEC3
:10B0A80010FA40F30884C94BD3ED004AF5EEC04AC4
:10B0B800F1EE10FA40F3FF8334EEC77A66EEE95AF0
:10B0C80087EE246AC5EE856AB7EE007AB4EEC76AE1
:10B0D800F1EE10FA88BFB0EE476AB5EEC06AF1EE3D
:10B0E80010FA76EE876AB8BFB0EE6B6A66EE266A2B
:10B0F800DBE5B74A92ED007AF0EEE76AF4EEC76A4C
:10B10800F1EE10FA7FF7A0A8B24A92ED007AF0EEBD
:10B11800CD6AF4EEC76AF1EE10FA7FF795A8AE4A49
:10B1280099ED007AD2ED006AB0EEC77AB4EEE67A0D
:10B13800F1EE10FA7FF588A801220999C4F8D41114
:10B1480084F8D021FFF784B8A44BA54FB3F90620A3
:10B158007B8B9A423FF706AEA24B1B78012B01F07E
:10B168000786192B01F004860E2B3FF4FBAD082B44
:10B178003FF4F8AD9C4B00229A60C4F80C21F1E52D
:10B188002B78002B3FF4A0AED4ED5F3A94ED5E6AC5
:10B19800D4ED7C7A954A94ED7B7AD2ED005A94ED01
:10B1A8005C4AD4ED5B4ADFF85C82DFF85CC2F4EEFF
:10B1B800C63AF3EE046AF1EE10FA37EEA65A00F139
:10B1C800F78798ED026A26EE446AF0EE674AE6EEE3
:10B1D800074AF4EEC54A34EEE66AF1EE10FA48BFC3
:10B1E800B0EE656A012B8CED006A3FF46DAE98ED08
:10B1F800066A26EE446AF0EE674AE6EE074AB4EEBF
:10B20800E45A34EEE66AF1EE10FA88BFB0EE656AE9
:10B21800022B8CED016A3FF457AE98ED0A6A26EED0
:10B22800446AF0EE674AE6EE074AF4EEC54A34EEA1
:10B23800E66AF1EE10FA48BFB0EE656A032B8CEDB2
:10B24800026A3FF441AE98ED0E6A26EE446AF0EECB
:10B25800674AE6EE074AB4EEE45A34EEE66AF1EEDF
:10B2680010FAC8BFB0EE656A042B8CED036A3FF490
:10B278002BAE98ED126A26EE446AF0EE674AE6EEC7
:10B28800074AB4EEE45A34EEE66AF1EE10FAC8BFA3
:10B29800B0EE656A052B8CED046A3FF415AE98EDA7
:10B2A800166A26EE446AF0EE674AE6EE074AF4EEBE
:10B2B800C54A74EEE66AF1EE10FAB8BFF0EE656AB8
:10B2C800062BCCED056A3FF4FFADD8ED1A6A66EEA1
:10B2D800C46AF0EE674AE6EE874AB3EE046AB4EE53
:10B2E800E45A74EEC66AF1EE10FAC8BFF0EE656A69
:10B2F800072BCCED066A3FF4E7ADD8ED1E6A26EEC3
:10B30800C44AE4EE077AB4EEE75A77EEC67AF1EE6D
:10B3180010FAC8BFF0EE657ACCED077AD4E5079944
:10B32800334BD1ED017A93ED007AF0EEE77AF4EE43
:10B33800C77AF1EE10FA7EF5FDAED1ED027AF0EEA5
:10B34800E77AB4EEE77AF1EE10FA7EF7F3AED1EDD4
:10B35800037AF0EEE77AB4EEE77AF1EE10FA7EF7C8
:10B36800E9AE244B1B689A077FF5DEAD2249234BD3
:10B37800B3F90C20B1F900E02148AEEB020E0068E9
:10B388008EEAEE72A2EBEE728242BEF6D3AEB3F94B
:10B398000E30B1F90220D21A82EAE273A3EBE2730B
:10B3A80098427EF7C7AEBFE50B4B99ED007AD3ED17
:10B3B800006AB0EEC77AB4EEE67AF1EE10FA7EF7DC
:10B3C80059AFFEF754BF00BFB8350020C035002084
:10B3D800EC350020E8350020F0350020506F0020C3
:10B3E8005C3E002044560020D062002080380020B7
:10B3F800E4350020203B00206C3B00200456002050
:10B40800E0350020A43800205454002007EE103AFC
:10B41800524BDFF854811B78C4F8A071B8EEC77A94
:10B42800F7EE006A132B86EE879AB8F90400B4F891
:10B43800A47195ED080A01F07583494B494A93EDCB
:10B44800001A93ED053A93ED122A93ED176AD3ED9E
:10B45800091A93ED0E4AD3ED015AD3ED063A93ED4E
:10B468000A7A93ED0F5AD3ED132AD3ED186AD3ED68
:10B47800044AD3ED030A67EE897A69EE288A29EE31
:10B48800088AA1EE273A02EB87060021A2EE286A75
:10B49800C4F89411C4F89811A1EE884AE5EEA73AC9
:10B4A800A7EE085A93ED167AD3ED0D5A93ED021ACA
:10B4B800D3ED0C1A86ED003AE2EEA86A64EEC34AB0
:10B4C80027EE467A93ED0B2AD3ED152A86ED204A0E
:10B4D800E0EEC33A65EEC45A93ED143AC3ED053A6B
:10B4E800E1EE274AF0EE477AA1EEC45AE2EE085A96
:10B4F800E2EEC66AE3EE287AC3ED064A83ED0E5AF9
:10B50800C3ED0F5A86ED406AC3ED176AC3ED187A8A
:10B51800C4F89C117B1C03F01F03A4F8A431A8F8FD
:10B528000400FEF7A3BBB0EE465AFEF735BF0AF09B
:10B538003BFBCEE422F0BCFC2AF81700FEF7A4BCC3
:10B5480096ED007A05EB4702B8EEC78A928F2AF883
:10B55800172028EE278AFEF775BC00BFF861002087
:10B56800AC4C0020284A0020FC610020A4F8483197
:10B578009946002A00F07281D74B0221D74ADFEDA5
:10B58800D86A1068D74A90F802C092F800E00278AA
:10B5980007EE902AF8EEE77AB0EE007A67EEA67A20
:10B5A800F4EEC77AF1EE10FA40F30E8337EEC77A5D
:10B5B800DFEDCD6AB0EE676AA7EE266AB0EE467A8E
:10B5C8009FEDCA6AD3ED006A66EE866AB0EEE66A57
:10B5D800C4ED5B6A84ED5E6ABCF1000F13D005EE22
:10B5E80090CAB8EEE55ADFEDBE5A66EEA64A25EED9
:10B5F800255AF7EE005A75EEC55A64EE864AE4EE0F
:10B60800855A66EEA56ADFEDBA5A427927EE257AA1
:10B6180027EE267ACAB1DFEDB26ADFEDB65A26EE1A
:10B62800266A06EE902AF8EEE66A26EE266AB4EE58
:10B63800E56AF1EE10FA00F37285F7EE005A35EE7E
:10B64800C66AC5EE866A27EE267ABEF10C0F9FED14
:10B65800AA8ADFEDAA6A00F01385B4EEC87AF1EE83
:10B6680010FA98BFB0EE478AB4EEE68AF1EE10FA07
:10B67800B8BFB0EE668A84ED418A002900F0E28006
:10B68800B0EE007AF4EEC77AF1EE10FA05DD37EE87
:10B69800C77ADFED956AE7EE267A93ED017ADFED5A
:10B6A800936A27EE267AB0EEC76A84ED5C7A84ED59
:10B6B8005F6ABCF1000F13D006EE90CADFED885A1E
:10B6C800F8EEE66A27EE075A66EEA56AF7EE005A24
:10B6D80075EEE65A25EE065AE5EE265A27EE257A45
:10B6E800DFED836A827967EEA67A67EE877AAAB178
:10B6F80007EE102AB8EEC77ADFED795ADFED7D6ADA
:10B7080027EE067A27EE257AB4EEE67AF1EE10FAFD
:10B7180040F30985DFED7A6A67EEA67ABEF10C0F71
:10B7280000F08D84DFED746A9FED747AF4EEE67AAA
:10B73800F1EE10FA88BFF0EE667AF4EEC77AF1EE11
:10B7480010FAB8BFF0EE477A0129C4ED427A79DDE4
:10B758004278DFED636A07EE902AF8EEE77AB0EEFA
:10B76800007A67EEA67A427AF4EEC77AF1EE10FA1A
:10B7780005DD37EEC77ADFED5C6AE7EE267A93EDF2
:10B78800027ADFED5A6A27EE267AB0EEC76A84EDB0
:10B798005D7A84ED606A9AB106EE902ADFED505A20
:10B7A800F8EEE66A27EE075A66EEA56AF7EE005A43
:10B7B80075EEE65A25EE065AE6EE855A27EE257A04
:10B7C800DFED4B6AC37967EEA67A67EE877A0BB32B
:10B7D80007EE103AB8EEC77ADFED415ADFED456A59
:10B7E80027EE067A27EE257AB4EEE67AF1EE10FA1D
:10B7F8000CDCB5EEC07AF1EE10FA01F1C082B7EEBA
:10B80800006A36EE477AC6EE076A01E0DFED3C6A69
:10B8180067EEA67ABEF10C0F00F00784DFED366AFA
:10B828009FED367AF4EEE67AF1EE10FA88BFF0EE84
:10B83800667AF4EEC77AF1EE10FAB8BFF0EE477AFE
:10B84800C4ED437ABEF1090F00F0D38397F8217055
:10B85800002F40F06A83002384F81831294B1B78A5
:10B8680023B9294FBB78002B41F0AD821D4B1B78C3
:10B87800072B00F022840022072B84F800217EF495
:10B88800A2A9F5F733FB0590FEF79FB91F4B204C93
:10B898001A68204BDFF8888094F80001D2691B8869
:10B8A800A8F80020A8F8023000287FF44CAA0590D8
:10B8B800194DFEF78AB9DFED196AFFF704BA41029C
:10B8C8003EF56CAFFEF76EBFF5F710FB144BC01BCF
:10B8D800D880FFF71ABB00BFD0620020F46F0020A9
:10B8E8000AD7233CF8610020D7A368416F12033BB5
:10B8F80000004843A4707D3F00C0F94400C0F9C46B
:10B908000000C842E73A0020E84E0020FC5300201F
:10B918000C210020BE390020306500200000000006
:10B92800FC610020F5F7E2FAA94B0B9A1B78DFF8C7
:10B93800B482801A012BA8F8020000F0E082072BDD
:10B948007EF4C0ACF5F7D2FA0746FEF7BCBCBEF1F0
:10B95800000F41F05B8498ED007ADDED0C6ADFF8AA
:10B9680088C225EE877AA6EE867AF0EE676AE7EE59
:10B97800056ABDEEE67A17EE106A17EE100A9E42C7
:10B98800A8BF1846B142C8BF084607EE100AB8EE6D
:10B99800C77A012A8CED007A3FF491AA98ED047ACF
:10B9A800DDED0D6A25EE877AA6EE867AF0EE676AF7
:10B9B800E7EE056ABDEEE67A17EE106A17EE100A92
:10B9C8009E42A8BF1846B142C8BF084607EE100AF3
:10B9D800B8EEC77A022A8CED017A3FF470AA98ED86
:10B9E800087ADDED0E6A25EE877AA6EE867AF0EE05
:10B9F800676AE7EE056ABDEEE67A17EE106A17EE9B
:10BA0800100A9E42A8BF1846B142C8BF084607EEB2
:10BA1800100AB8EEC77A032A8CED027A3FF44FAACF
:10BA280098ED0C7ADDED0F6A25EE877AA6EE867A18
:10BA3800F0EE676AE7EE056ABDEEE67A17EE106A81
:10BA480017EE100A9E42A8BF1846B142C8BF084662
:10BA580007EE100AB8EEC77A042A8CED037A3FF491
:10BA68002EAA98ED107ADDED106A25EE877AA6EEFB
:10BA7800867AF0EE676AE7EE056ABDEEE67A17EEBB
:10BA8800106A17EE100A9E42A8BF1846B142C8BFF6
:10BA9800084607EE100AB8EEC77A052A8CED047A34
:10BAA8003FF40DAA98ED147ADDED116A25EE877A38
:10BAB800A6EE867AF0EE676AE7EE056ABDEEE67AEC
:10BAC80017EE106A17EE100A9E42A8BF1846B14238
:10BAD800C8BF084607EE100AB8EEC77A062A8CEDEA
:10BAE800057A3FF4ECA998ED187ADDED126A25EE97
:10BAF800877AA6EE867AF0EE676AE7EE056ABDEE0B
:10BB0800E67A17EE106A17EE100A9E42A8BF18468A
:10BB1800B142C8BF084607EE100AB8EEC77A072A2E
:10BB28008CED067A3FF4CBA998ED1C7ADDED136A0B
:10BB380065EE875AE6EE265AE5EE257AFDEEE77AB7
:10BB480017EE900A8342A8BF03468142C8BF0B463E
:10BB580007EE903AF8EEE77ACCED077A002A7FF400
:10BB6800AEA9FFF7B1B91B4B5A79002A3EF499AC3C
:10BB7800194A1278002A3EF494AC1B78DFED174A74
:10BB880007EE903A164BB8EE677A1B8807EE902AB4
:10BB980006EE903AF8EEE77AF8EE666A67EE277AEC
:10BBA800B7EE007AC7EEA63AF4EEE43AF1EE10FAF0
:10BBB80088BFF0EE643AF4EEC73AF1EE10FAB8BF77
:10BBC800F0EE473AFEF76FBCB0EE677AF8E400BFD4
:10BBD800F86100208C510020CE620020713DAA3F00
:10BBE80088620020FC61002054540020BCF1000F42
:10BBF80000F09783BEF1000F41F0A287DFF8A4851B
:10BC0800B9F1000F41F0E185D8ED006ADDED0C4A8D
:10BC1800DFF894C565EEA66ABDEEC77A17EE101A6E
:10BC2800B0EE667AA4EE867AF0EE676AE7EE056A09
:10BC3800BDEEE67A17EE106A17EE100A9E42A8BF0C
:10BC48001846B142C8BF084607EE100AB8EEC77AD0
:10BC5800012A8CED007A3FF432A998ED047ADDEDE3
:10BC68000D6A25EE877AA6EE867AF0EE676AE7EE29
:10BC7800056ABDEEE67A17EE106A17EE100A9E42C4
:10BC8800A8BF18468E42B8BF084607EE100AB8EE9D
:10BC9800C77A022A8CED017A3FF411A998ED087A47
:10BCA800DDED0E6A25EE877AA6EE867AF0EE676AF3
:10BCB800E7EE056ABDEEE67A17EE106A17EE100A8F
:10BCC8009E42A8BF18468E42B8BF084607EE100A23
:10BCD800B8EEC77A032A8CED027A3FF4F0A898ED03
:10BCE8000C7ADDED0F6A25EE877AA6EE867AF0EEFD
:10BCF800676AE7EE056ABDEEE67A17EE106A17EE98
:10BD0800100A9E42A8BF18468E42B8BF084607EEE2
:10BD1800100AB8EEC77A042A8CED037A3FF4CFA84C
:10BD280098ED107ADDED106A25EE877AA6EE867A10
:10BD3800F0EE676AE7EE056ABDEEE67A17EE106A7E
:10BD480017EE100A9E42A8BF18468E42B8BF084692
:10BD580007EE100AB8EEC77A052A8CED047A3FF48C
:10BD6800AEA898ED147ADDED116A25EE877AA6EE75
:10BD7800867AF0EE676AE7EE056ABDEEE67A17EEB8
:10BD8800106A17EE100A9E42A8BF18468E42B8BF26
:10BD9800084607EE100AB8EEC77A062A8CED057A2F
:10BDA8003FF48DA898ED187ADDED126A25EE877AB2
:10BDB800A6EE867AF0EE676AE7EE056ABDEEE67AE9
:10BDC80017EE106A17EE100A9E42A8BF18468E4258
:10BDD800B8BF084607EE100AB8EEC77A072A8CEDF6
:10BDE800067A3FF46CA898ED1C7ADDED136A65EECF
:10BDF800875AE6EE265AE5EE257AFDEEE77A17EE43
:10BE0800900A8342A8BF03468142D8BF194607EE6D
:10BE1800901AF8EEE77ACCED077A002A7FF44FA85B
:10BE2800FFF752B8C74B93ED006AFEF72EBFAB6819
:10BE3800002B3EF491AF05F1500128469847FEF7D4
:10BE48008BBFC14BC149D3F8EC30086844F6206178
:10BE58008B42A8BF0B46B3F57A7FB8BF4FF47A730D
:10BE680099B2C006A4F81A11DBF8003041F1D78264
:10BE7800DB0400F16B83B64BD3F800C0BCF932E0A9
:10BE8800B44BB548D3ED037AD4F81C31A0FB0101BB
:10BE98008809642191FBF0F11429BDEEE77A04EBDF
:10BEA8004308A8BF142101339942C4F81C3117EE86
:10BEB800109ADCBF0023C4F81C3104EB4303A8F834
:10BEC8002091B3F9203107EE103AB8EEC77A77EE31
:10BED800C77AFDEEE77ACDED057ABDF9141081EA4F
:10BEE800E173A3EBE173734502F397809B4B19460B
:10BEF8004FF07E530B60FEF742BFDFF8B082F4F7D5
:10BF0800F5FF974AD4F8E4311268C4F8E401C31A7B
:10BF18009A1A0746A8F80430A8F80620FEF7D3B9FD
:10BF2800F4F7E4FF0B90FDF7DABF1E218748F7F717
:10BF380011F900283FF48FAC8A4B1B885A063FF54D
:10BF48008AAC94F88431BB4242F0C880834BD4ED6C
:10BF5800627A93ED010AD4ED435A9FED836ADFEDCF
:10BF6800836A27EEE57A68EE277AA8EE007AE5EE8E
:10BF7800807AB4EEC67AF1EE10FA88BFB0EE467A4F
:10BF8800B4EEE67AF1EE10FAF4EEC67AB8BFB0EE87
:10BF9800667AF1EE10FA88BFF0EE467AF4EEE67AA9
:10BFA800F1EE10FAB8BFF0EE667A84ED417AC4ED8E
:10BFB800437A50E4B4F8F411914240F282856C4916
:10BFC8006C4AD1ED007A92ED007A6B49C4ED7E7A25
:10BFD80077EE676AC4ED7C7A0122C4ED7B6A84ED52
:10BFE8007F7AD1ED006ADFED657A84F80022FEF7EA
:10BFF8009AB9FDEEC87ADFF8B48117EE903AA8F83E
:10C008000490A8F8063021E45D4B1B88002B40F013
:10C0180077855C4A5C4B11781868F6F747F9D4F8CD
:10C02800D421099B9A1AFEF754B8BDEEE77ADFF8D7
:10C038007C8117EE103AA8F80430FFF7EFBB9FEDAC
:10C048004A7ADFED4A6ADFF86481F4EEC77AF1EEE6
:10C0580010FA98BFB0EE677AFDEEE77AB4EEE67AAA
:10C06800F1EE10FA17EE902AB8BFB0EE667A012901
:10C0780084ED427AA8F802203FF76AABFFF7E6BBE7
:10C08800B4EEC87AF1EE10FA98BFB0EE478ABDEE6A
:10C09800C77AB4EEE68ADFF81481F1EE10FA17EEEB
:10C0A800102AB8BFB0EE668A84ED418AA8F800204D
:10C0B80000297FF4E5AAFFF7C9BBF4F717FFDFF8FB
:10C0C800EC80324B801B1B78A8F80400FFF7D3BB29
:10C0D8002F4A3049D2ED006A2F4A91ED006A127852
:10C0E800C4ED7E6A84ED7F6A002A40F0E68476EE2D
:10C0F800C65AF0EE466ABCEEC76A2849C4ED7B5AB8
:10C1080016EE102AC4ED7C6AA4F8F421FF22D1EDC2
:10C11800006A84F8002277EEC77AFEF704B9DFEDEB
:10C12800206AFFF790BAB5EEC07AF1EE10FA00F186
:10C138002A86B7EE006A36EE477AC6EE076AFFF738
:10C14800EBBA00BFB83500200C10002014540020B2
:10C15800F83A0020D0620020D34D62107800002009
:10C16800285600208251002000C0F94400C0F9C4BC
:10C1780024390020D4550020403900200000000058
:10C18800445700204657002048570020F8610020F7
:10C198007C54002028390020B45D00203C39002060
:10C1A8000000C842A438002054540020FC6100203C
:10C1B80098ED016A26EE646AB0EE674AA6EE074A71
:10C1C800B4EEC45A34EE666AF1EE10FAC8BFB0EEA7
:10C1D800656A012B8CED006A3EF476AE98ED056A2F
:10C1E80026EE646AB0EE674AA6EE074AB4EEC45A71
:10C1F80034EE666AF1EE10FAC8BFB0EE656A022B3B
:10C208008CED016A3EF460AE98ED096A26EE646A28
:10C21800B0EE674AA6EE074AB4EEC45A34EE666A30
:10C22800F1EE10FAC8BFB0EE656A032B8CED026A16
:10C238003EF44AAE98ED0D6A26EE646AB0EE674A9F
:10C24800A6EE074AB4EEC45A34EE666AF1EE10FA66
:10C25800C8BFB0EE656A042B8CED036A3EF434AEB9
:10C2680098ED116A26EE646AB0EE674AA6EE074AB0
:10C27800B4EEC45A34EE666AF1EE10FAC8BFB0EEF6
:10C28800656A052B8CED046A3EF41EAE98ED156ABE
:10C2980026EE646AB0EE674AA6EE074AB4EEC45AC0
:10C2A80074EE666AF1EE10FAC8BFF0EE656A062B06
:10C2B800CCED056A3EF408AED8ED196A66EEE46A7C
:10C2C800B0EE674AA6EE874AB3EE046AB4EEC45AE3
:10C2D80074EE466AF1EE10FAC8BFF0EE656A072BF5
:10C2E800CCED066A3EF4F0ADD8ED1D6A66EEE44A80
:10C2F800E4EE877AF4EEC57A77EEC67AF1EE10FAB4
:10C30800B8BFF0EE657ACCED077AFEF7DDBD97F899
:10C318002030C3EB431103EB8103DB009BB2FEF734
:10C328003ABDDFF80485B9F1000F41F0E480D8ED9B
:10C33800006ADDED0C4ADFF8F4C465EEA66ABDEECE
:10C34800C77A17EE101AB0EE667AA4EE867AF0EE87
:10C35800676AE7EE056ABDEEE67A17EE106A17EE31
:10C36800100A9E42A8BF1846B142C8BF084607EE49
:10C37800100AB8EEC77A012A8CED007A3EF468AB51
:10C3880098ED047ADDED0D6A25EE877AA6EE867AB9
:10C39800F0EE676AE7EE056ABDEEE67A17EE106A18
:10C3A80017EE100A9E42A8BF18468E42B8BF08462C
:10C3B80007EE100AB8EEC77A022A8CED017A3EF42D
:10C3C80047AB98ED087ADDED0E6A25EE877AA6EE82
:10C3D800867AF0EE676AE7EE056ABDEEE67A17EE52
:10C3E800106A17EE100A9E42A8BF18468E42B8BFC0
:10C3F800084607EE100AB8EEC77A032A8CED027ACF
:10C408003EF426AB98ED0C7ADDED0F6A25EE877ABF
:10C41800A6EE867AF0EE676AE7EE056ABDEEE67A82
:10C4280017EE106A17EE100A9E42A8BF18468E42F1
:10C43800B8BF084607EE100AB8EEC77A042A8CED92
:10C44800037A3EF405AB98ED107ADDED106A25EE1F
:10C45800877AA6EE867AF0EE676AE7EE056ABDEEA1
:10C46800E67A17EE106A17EE100A9E42A8BF184621
:10C478008E42B8BF084607EE100AB8EEC77A052AFA
:10C488008CED047A3EF4E4AA98ED147ADDED116A95
:10C4980025EE877AA6EE867AF0EE676AE7EE056AF9
:10C4A800BDEEE67A17EE106A17EE100A9E42A8BF94
:10C4B80018468E42B8BF084607EE100AB8EEC77A8B
:10C4C800062A8CED057A3EF4C3AA98ED187ADDEDBC
:10C4D800126A25EE877AA6EE867AF0EE676AE7EEAC
:10C4E800056ABDEEE67A17EE106A17EE100A9E424C
:10C4F800A8BF18468E42B8BF084607EE100AB8EE25
:10C50800C77A072A8CED067A3EF4A2AA98ED1C7A1F
:10C51800DDED136A65EE875AE6EE265AE5EE257AD2
:10C52800FDEEE77A17EE900A8342A8BF03468142E0
:10C53800D8BF194607EE901AF8EEE77ACCED077ADD
:10C54800BEF1000F7EF4C0ACFEF786BAAA4BD3F852
:10C5580000C0BCF832E04FEA5E0E91E4DFF8D092FA
:10C56800D4ED017A94ED006AB9F80000D9F81430D6
:10C5780077EEA77AF0EE006AB0EE677AA6EE267A32
:10C58800013804EBC002D6EE267A083A1033F6EEEC
:10C59800003A27EE237A67EEA37A84ED207AC4ED79
:10C5A800217A964CA64604F1800192ED027A92ED2A
:10C5B800036ADEED036ADEED027A53ED014A13EDFC
:10C5C800025A37EE674A76EEC65A77EE277AE4EED5
:10C5D800845A0138A2F10802E5EE047A0EF1080E39
:10C5E80003F1080336EE267A01F10801E4EE877AB2
:10C5F800E5EE475A67EEA37A25EEA37AC1ED007AF5
:10C6080081ED017AD1D1142F7DF4EBABF4F76EFCF8
:10C61800069BDFF82082C01AA8F80200D4F8A861A7
:10C62800FDF7DFBBD4F8AC81B4F8A4A1744BCAF110
:10C6380020095FFA89F90AEB481E03EB8E0E5FEAC0
:10C64800990301F0F185013318016E496E4A0EEB2A
:10C65800000C0EF1100313ED024A13ED035A13ED0B
:10C66800016A13ED047A51ED024A51ED035A51ED76
:10C67800016A51ED047A64EE244A65EE255A66EEA5
:10C68800266A67EE277A10339C4542ED024A42ED4E
:10C69800035A42ED016A42ED047A01F1100102F1F8
:10C6A8001002D8D15949A0F11002964401EB020CAE
:10C6B800224419F0030309D0BEEC017AFCEC017A9C
:10C6C80067EE277A013BE2EC017AF5D1BAF1000F67
:10C6D80041F0D481142F7DF484ABF4F707FC069B5A
:10C6E800DFF85081D4F8A861C01AA8F80200FDF755
:10C6F80078BBDFF83C914148D9F80820B9F80C100C
:10C7080020F0D4FA424B1F78142F01F0A185D4F8F9
:10C71800A8610136C4F8A86122E7D4F8AC913D4B72
:10C728003D4ADFED3E7AD2ED008A3D4A4FEAC90123
:10C738000B44F8EE688A9B8809EE103A643BC82BD4
:10C74800A8BFC82368EEA78AF8EE497A782BB8BF45
:10C75800782368EEA78A07EE903A4944B0EE680A53
:10C7680002EB8108B8EEE78A21F0EEFBB8EEC99A31
:10C77800F0EE409AB0EE680A21F048FB38EE097AEC
:10C7880079EE487A28EE098A67EE877AB7EE006A6A
:10C7980088EE277A142FF8EE007A77EE076A60EEB3
:10C7A800277A89EEA67A77EE065A36EE477AC6EEEB
:10C7B800256A67EEA67A27EE267AC8ED006A88ED24
:10C7C800047AC8ED026AC8ED017AC8ED037A01F06F
:10C7D8009185144B0E4A09F1010983FB0938A8EB2E
:10C7E800E97808EB48080136A9EB08081778C4F877
:10C7F800A861C4F8AC8117E7F83A00200C210020A2
:10C80800284A0020B84B00201C210020A84B0020FB
:10C81800F8610020284C0020D460002027D4D236AC
:10C828004867002056555555A43800205454002018
:10C83800104A0020FC610020DFF80494B9F800E0F9
:10C84800D9F804C04FEA5E084FEA880204EB8E0666
:10C858005FEADE0E04EB020300F0A08010320EF156
:10C86800010EEB4803EB0E1E324410330CF1100797
:10C8780006F1100151ED032A51ED043A10ED043A86
:10C8880010ED032A51ED026A11ED016A10ED020A5A
:10C8980010ED018A12ED044A12ED035A53ED044AD1
:10C8A80053ED035A13ED027A53ED017A52ED020A61
:10C8B80012ED011A73EE238A72EE221A40ED048AF1
:10C8C80040ED031A70EE268A78EE061A40ED028AC9
:10C8D80040ED011A74EE848A75EE851A43ED048AD8
:10C8E80043ED031A77EE208A77EE811A43ED028A28
:10C8F80043ED011A73EE633A75EE655A17ED035A64
:10C9080032EE623A74EE644A65EE631A17ED044A31
:10C9180023EE052A64EE652AE3EE041A10339E45D9
:10C9280024EE843AA3EE842A00F1100007F11007E0
:10C93800A5EE853A01F1100102F11002E4EE852A14
:10C9480041ED071A01ED082A02ED073A42ED082ADF
:10C9580057ED055A17ED065A70EE666A38EE466AC4
:10C9680030EEC77A71EE677A26EE253A65EEE63A3A
:10C9780025EE674A67EE054AE6EE053AA6EE853AE1
:10C98800A7EE254AE7EEA54A01ED063A41ED053A3C
:10C9980002ED064A42ED054A7FF46CAF1FFA88F8AB
:10C9A800624641469B4816F09BFD4146D9F8042053
:10C9B800304616F095FD984B1B78142B7FF42EAE5D
:10C9C80024E6DFF8809299F80020900801F0148599
:10C9D800DFF874C200F101084FEA48180CEB080EA2
:10C9E8000CF12003ACF1700113ED076A53ED056AF1
:10C9F80013ED037A53ED017A53ED025A13ED084A09
:10CA080053ED064A13ED045A26EE066A66EEA66A48
:10CA180027EE077A67EEA77AA4EE046A20339E45CC
:10CA2800E4EEA46A01F11001A5EE057AE5EEA57A17
:10CA3800F1EEC65AB1EEE66AF1EEC76AB1EEE77AF0
:10CA480041ED085A01ED076A41ED066A01ED057AE4
:10CA5800CAD1A8F12008C44404EB001012F0030363
:10CA680018BF0CF1080C0FD05CED017A1CED027AAE
:10CA780067EEA77A013BE7EE077A0CF1080CB1EEF6
:10CA8800E77AA0EC017AEFD1142F01F05C8401362B
:10CA9800C4F8A861FDF70EB9F4F728FA5E4B0690C2
:10CAA8001F78142F05BFDFF8A481D4F8A861D4F843
:10CAB800A861A8F80060FDF7E2B876EE665AFFF7BD
:10CAC8001ABB564A5649D2ED007A564A91ED007A79
:10CAD8001278C4ED7E7A84ED7F7A002A01F097827D
:10CAE80077EE676A5049C4ED7C7AC4ED7B6AFF2211
:10CAF800D1ED006ADFED4D7A84F80022FDF713BC12
:10CB08004B494B69002B3DF4E4AA4A484A4B00883C
:10CB180093FBF0F00B684FF0010E186081F811E0FC
:10CB2800FDF7D7BA454EDFF8289196ED004A96ED05
:10CB3800057AD6ED014A96ED066AD6ED046A96EDB9
:10CB4800035AD6ED025A67EE897A09EB8703A4EEF9
:10CB5800277AA4EEA76A66EEC76AA5EE476AE5EEED
:10CB6800A76A20EE070A86ED056AC6ED066A83ED18
:10CB7800007A29EE088A21F09BF969EE288AD6ED19
:10CB88000E5AD6ED176A96ED091AD6ED121A96EDD9
:10CB98000F5A96ED187A96ED0A2AD6ED132A96EDD5
:10CBA8000D6AD6ED167A96ED0C3AD6ED0B3A96ED5F
:10CBB800154AD6ED144AE1EE085A002209EB87031C
:10CBC800E8EEA16A00B2C4F89421A2EE085AC4F8AB
:10CBD8009821C4F89C21A8EEA27A26EE656A67EE31
:10CBE800E67AA3EE655AA3EE886AA6EEC47AE8EE62
:10CBF800A47A86ED0E5AC3ED205A86ED0F6AC3ED6E
:10CC0800406A86ED177AC6ED187AFEF783BC00BF36
:10CC18001C2100200C210020F86100207C540020F9
:10CC280028390020B45D00203C39002000000000B5
:10CC38004C5700206457002020A10700AC4C00206E
:10CC4800104A00200A4A00208C210020FC610020A4
:10CC5800284A0020B3494A69002A3DF46BAA0A68A9
:10CC680013604B74FDF766BAB5F93C306A6207EE9B
:10CC7800903A0122F8EEE77AEB66C5F8882000239F
:10CC8800012FC5ED1F7AC5ED1E7AC5F8803001F079
:10CC9800E681B7427DF434AFB5F93E302B6707EE35
:10CCA800903A00220123F8EEE77AAA62C5F89C3090
:10CCB8000023012FC5ED247AC5ED237AC5F89430F9
:10CCC80001F0D181B7427DF44BAFB5F940306B67C5
:10CCD80007EE903A00220123F8EEE77AEA62C5F8F7
:10CCE800B0300023012FC5ED297AC5ED287AC5F8A3
:10CCF800A8307DF465AF9FED8C8AB9F1030F46D05B
:10CD0800BAF1000F09D007EE90AAF8EEE77AF4EE30
:10CD1800C87AF1EE10FA01F17483844A6B6F1268D5
:10CD280094F8B011A8F8060003EB560393FBF6F647
:10CD38000023EE6293621363D36231B17C4B1B888C
:10CD480023F40063002B7DF43DAF7A4B1B6813F48A
:10CD5800003341F07C8178491A46C85C012803F108
:10CD68000C0300F00E850132152AF6D1FDF72ABF13
:10CD7800724B9B7B002B3EF4FDA9FDF7F3BFF7EE4A
:10CD8800006AFEF745BDF7EE006AFEF7C5BCB0EED7
:10CD9800480A21F08DF800B2B2E7B4F8489109F1D9
:10CDA800FF390FFA89F9B9F1000FA4F848917EF715
:10CDB800E0AB634BFEF743B8B4F81A3103F57A7366
:10CDC8009BB2FDF7E8BFDFF88C8198F80020013AA4
:10CDD8000D2A18D8DFE812F097006A011901FC0043
:10CDE80017001700E5005501C00080006C006000C6
:10CDF80055000E001F2005931EF092FF059B10B9E9
:10CE0800012288F80020012B00F01E86FA78002AFB
:10CE18003EF42CAD4B4A1278D00706D405930BF09C
:10CE2800FBFB059B002841F07382474FD4F8901113
:10CE38003A68914201F2738298F80030012B3EF46F
:10CE480015AD94F88C21002A3EF410AD0B2B0DD8AB
:10CE580001229A4040F6030112EA01090CD112F4AA
:10CE6800C06F03D0093B012B41F25384374B3A681A
:10CE78005A600B2388F80030002384F88C31FEF7C1
:10CE8800F5BC012B01F022830E23132088F8003013
:10CE980005F064F8BB78B6E7012B01D1F6F700FB83
:10CEA8000D23132088F8003005F058F8BB78AAE75E
:10CEB800264A254952680968C8328A4204D320F0B4
:10CEC80049FEBB7800289ED0032B01F01B83012369
:10CED80088F80030BB7896E71D4B1B78002B01F0D3
:10CEE80086821A201EF01CFF002841F0808294F8E8
:10CEF8008C31002B41F07B82092388F8003015F033
:10CF08002BF8BB787FE70F4B1B78DB0701F1E98231
:10CF18001F201EF005FF0028BCD00C2388F8003025
:10CF2800B8E700BF4C57002000000000FC53002069
:10CF3800C0510020583700205C100308E85A002030
:10CF4800D06200204D3C00206C570020D8550020AE
:10CF580098560020E54E00201A201EF0E1FE002819
:10CF6800CDD0994B1B88002BC9D1984B4520D3F8BD
:10CF780000901FF0E3FB0E201FF0E0FB48461FF077
:10CF8800A7FCDDF8249048461FF0A2FC904A914B7C
:10CF980012681A6048460A2388F8003014F02EFDFB
:10CFA800ADE71FF01BFB8C4B002105208DE803002B
:10CFB800A3F108020291532015F004FD00287FF424
:10CFC80069AF864ABB781060082288F800201AE703
:10CFD8001FF004FB824A0292A2F10C03252101935F
:10CFE8000091A2F10A035021163A492015F0EAFCF3
:10CFF80000287FF44FAF794ABB7810604FF0FF31BB
:10D008005160072288F80020FDE6DFF8D0911FF074
:10D01800E5FA744AD9F80430126864339342BFF4CD
:10D0280039AF40201FF0B2FA00287FF433AFD9F8A7
:10D0380000306D49DFF8B4B14FF0400A11E00591B6
:10D048001FF07CFBDBF80020D9F800300599013A85
:10D058000133BAF1010ACBF80020C9F8003001F019
:10D06800F682CB5C1846002BE9D100234FF0FF3243
:10D07800C9F80030042388F80030C9F80420BB78C8
:10D08800C1E61FF0ABFA14F0A1FF00283FF402AF8D
:10D0980020F060FD00283FF4FDAE4D4A4D4B12686C
:10D0A8001A600A2388F80030BB78ACE64D4A4B4931
:10D0B80012684A604D4800220A600321026088F81D
:10D0C8000010A0E64A4ADFED4B7A92ED080A059374
:10D0D800B4EEE70AF1EE10FA40F2CC8420F07EFFBD
:10D0E800D4ED457A20EE270A20F0E2FEB0F5617F04
:10D0F800059B00F35C8607EE900AF8EEE76ADFED21
:10D108003E7A66EEA76A07EE903AB8EEE77AFDEE49
:10D11800E67A17EE903A2033402B41F224819FEDB6
:10D12800370A20F0C5FE00B207EE900AB8EEE77A9B
:10D13800334BD3ED037A77EE877AC3ED037AFDF7A5
:10D1480019BE0A9B93F800E00EF0010EBEF1000F25
:10D158007DF4BAAEFDF780BC2A4BDFED2B7A1E6852
:10D16800C4ED707A16F0805640F0238310F48006E0
:10D1780000F0B7810026B6EE007A67EE877AF4EE03
:10D18800E75AF1EE10FA48BFF0EE675A40F1118302
:10D19800C4ED815AFDF706BBF3F7A8FE0646FDF776
:10D1A800D3BD74EE667AB7EE007AF4EEC77AF1EE84
:10D1B80010FAC4ED707A40F33F8784EEA77A8DEDBC
:10D1C8000C7AFDF7E5BA00BF087100200471002051
:10D1D8001871002010710020000A0308D85500209B
:10D1E800520803086C570020EC07030874700020ED
:10D1F800E43600208FC2753CD06D393A000000003B
:10D20800D06200201454002000000080BAF1000F02
:10D2180000F0E78598ED007ADDED0C6ADFF81CC9AF
:10D2280025EE877AA6EE867AF0EE676AE7EE056A5B
:10D23800BDEEE67A17EE106A17EE100A9E42A8BFF6
:10D248001846B142C8BF084607EE100AB8EEC77ABA
:10D25800012A8CED007A3DF437AE98ED047ADDEDC5
:10D268000D6A25EE877AA6EE867AF0EE676AE7EE13
:10D27800056ABDEEE67A17EE106A17EE100A9E42AE
:10D28800A8BF1846B142C8BF084607EE100AB8EE54
:10D29800C77A022A8CED017A3DF416AE98ED087A29
:10D2A800DDED0E6A25EE877AA6EE867AF0EE676ADD
:10D2B800E7EE056ABDEEE67A17EE106A17EE100A79
:10D2C8009E42A8BF1846B142C8BF084607EE100ADA
:10D2D800B8EEC77A032A8CED027A3DF4F5AD98EDE5
:10D2E8000C7ADDED0F6A25EE877AA6EE867AF0EEE7
:10D2F800676AE7EE056ABDEEE67A17EE106A17EE82
:10D30800100A9E42A8BF1846B142C8BF084607EE99
:10D31800100AB8EEC77A042A8CED037A3DF4D4AD2E
:10D3280098ED107ADDED106A25EE877AA6EE867AFA
:10D33800F0EE676AE7EE056ABDEEE67A17EE106A68
:10D3480017EE100A9E42A8BF1846B142C8BF084649
:10D3580007EE100AB8EEC77A052A8CED047A3DF478
:10D36800B3AD98ED147ADDED116A25EE877AA6EE55
:10D37800867AF0EE676AE7EE056ABDEEE67A17EEA2
:10D38800106A17EE100A9E42A8BF1846B142C8BFDD
:10D39800084607EE100AB8EEC77A062A8CED057A19
:10D3A8003DF492AD98ED187ADDED126A25EE877A94
:10D3B800A6EE867AF0EE676AE7EE056ABDEEE67AD3
:10D3C80017EE106A17EE100A9E42A8BF1846B1421F
:10D3D800C8BF084607EE100AB8EEC77A072A8CEDD0
:10D3E800067A3DF471AD98ED1C7ADDED136A65EEB1
:10D3F800875AE6EE265AE5EE257AFDEEE77A17EE2D
:10D40800902A9342A8BF13468A42A8BF194607EE3E
:10D41800901AF8EEE77ACCED077AFDF755BDD800FB
:10D428003EF526ADFDF7ABBC012A40F3188607EEA2
:10D43800101AB8EEC77AC7EE876AB1EEE68AB9F174
:10D44800030F13D0BAF1000F09D007EE90AAF8EE37
:10D45800E77AF4EEC87AF1EE10FA00F1D287EB6EB3
:10D4680003EB560393FBF6F36B6212E4B0EE480A43
:10D4780020F01EFD00B2E5E7012A7FF73CAC07EE7D
:10D48800101AB8EEC77AC7EE876AB1EEE68A34E4B6
:10D49800012A40F3E88507EE101AB8EEC77AC7EEFE
:10D4A800876AB1EEE68AB9F1030F14D0BAF1000F1A
:10D4B80009D007EE90AAF8EEE77AF4EEC87AF1EE12
:10D4C80010FA00F19E872B6F03EB560393FBF6F3DC
:10D4D800AB62FFF7F7BBB0EE480A20F0E9FC00B2F8
:10D4E800E4E7B6EE007AF4EEC75AF1EE10FA3FF729
:10D4F80042AEFDF757B9D8ED004A9DED0C4ADFF86A
:10D508003CC665EEA44AFDEEC73AE4EE064AB0EE24
:10D51800674AA4EE854A13EE901AF4EEC46AF1EE57
:10D5280010FAF0EE444A88BFF0EE474AFDEEE44AAE
:10D5380014EE900A14EE906A9842A8BF1E468142E3
:10D54800C8BF0E4604EE906AF8EEE44A012ACCED14
:10D55800004A3DF47DAAD8ED044A9DED0D4A65EEDA
:10D56800A44AE4EE064AB0EE674AA4EE854AF4EE11
:10D57800C46AF1EE10FAF0EE444A88BFF0EE474A6A
:10D58800FDEEE44A14EE900A14EE906A9842A8BFA1
:10D598001E468842B8BF0E4604EE906AF8EEE44A8A
:10D5A800022ACCED014A3DF453AAD8ED084A9DED74
:10D5B8000E4A65EEA44AE4EE064AB0EE674AA4EEC7
:10D5C800854AF4EEC46AF1EE10FAF0EE444A88BFD8
:10D5D800F0EE474AFDEEE44A14EE900A14EE906A23
:10D5E8009842A8BF1E468842B8BF0E4604EE906A0D
:10D5F800F8EEE44A032ACCED024A3DF429AAD8ED14
:10D608000C4A9DED0F4A65EEA44AE4EE064AB0EED8
:10D61800674AA4EE854AF4EEC46AF1EE10FAF0EE19
:10D62800444A88BFF0EE474AFDEEE44A14EE900AF9
:10D6380014EE906A9842A8BF1E468842B8BF0E46AC
:10D6480004EE906AF8EEE44A042ACCED034A3DF46D
:10D65800FFA9D8ED104A9DED104A65EEA44AE4EE04
:10D66800064AB0EE674AA4EE854AF4EEC46AF1EEC3
:10D6780010FAF0EE444A88BFF0EE474AFDEEE44A5D
:10D6880014EE900A14EE906A9842A8BF1E4688428B
:10D69800B8BF0E4604EE906AF8EEE44A052ACCEDCF
:10D6A800044A3DF4D5A9D8ED144A9DED114A65EE1A
:10D6B800A44AE4EE064AB0EE674AA4EE854AF4EEC0
:10D6C800C46AF1EE10FAF0EE444A88BFF0EE474A19
:10D6D800FDEEE44A14EE900A14EE906A9842A8BF50
:10D6E8001E468842B8BF0E4604EE906AF8EEE44A39
:10D6F800062ACCED054A3DF4ABA9D8ED184A9DEDB4
:10D70800124A65EEA44AE4EE064AB0EE674AA4EE71
:10D71800854AF4EEC46AF1EE10FAF0EE444A88BF86
:10D72800F0EE474AFDEEE44A14EE900A14EE906AD1
:10D738009842A8BF1E468842B8BF0E4604EE906ABB
:10D74800F8EEE44A072ACCED064A3DF481A9D8ED63
:10D758001C4A9DED134A65EEA45AE6EE045AE5EE1E
:10D76800257AF4EEE76AF1EE10FAC8BFF0EE477AD0
:10D77800FEF7D6BE8223FCF720BBDFEDEB7AFCF781
:10D78800E7BAD4F8B46153003EB1981801EB8000B1
:10D7980076784078B042BDF415AA134401EB8301B2
:10D7A8000023C4F8B411A4F80832C4F80C32FDF709
:10D7B80009BAB7EE007A77EE677AF4EEE75AF1EE37
:10D7C80010FA88BFF0EE675AE2E4D8ED004A9DED02
:10D7D8000C4ADFF868C365EEA44AFDEEC73AE4EEEA
:10D7E800064AB0EE674AA4EE854A13EE901AF4EEA4
:10D7F800C46AF1EE10FAF0EE444A88BFF0EE474AE8
:10D80800FDEEE44A14EE900A14EE906A9842A8BF1E
:10D818001E468142C8BF0E4604EE906AF8EEE44AFE
:10D82800012ACCED004A3DF44AABD8ED044A9DEDFF
:10D838000D4A65EEA44AE4EE064AB0EE674AA4EE45
:10D84800854AF4EEC46AF1EE10FAF0EE444A88BF55
:10D85800F0EE474AFDEEE44A14EE900A14EE906AA0
:10D868009842A8BF1E468842B8BF0E4604EE906A8A
:10D87800F8EEE44A022ACCED014A3DF420ABD8ED9B
:10D88800084A9DED0E4A65EEA44AE4EE064AB0EE5B
:10D89800674AA4EE854AF4EEC46AF1EE10FAF0EE97
:10D8A800444A88BFF0EE474AFDEEE44A14EE900A77
:10D8B80014EE906A9842A8BF1E468842B8BF0E462A
:10D8C80004EE906AF8EEE44A032ACCED024A3DF4ED
:10D8D800F6AAD8ED0C4A9DED0F4A65EEA44AE4EE8F
:10D8E800064AB0EE674AA4EE854AF4EEC46AF1EE41
:10D8F80010FAF0EE444A88BFF0EE474AFDEEE44ADB
:10D9080014EE900A14EE906A9842A8BF1E46884208
:10D91800B8BF0E4604EE906AF8EEE44A042ACCED4D
:10D92800034A3DF4CCAAD8ED104A9DED104A65EEA5
:10D93800A44AE4EE064AB0EE674AA4EE854AF4EE3D
:10D94800C46AF1EE10FAF0EE444A88BFF0EE474A96
:10D95800FDEEE44A14EE900A14EE906A9842A8BFCD
:10D968001E468842B8BF0E4604EE906AF8EEE44AB6
:10D97800052ACCED044A3DF4A2AAD8ED144A9DED3F
:10D98800114A65EEA44AE4EE064AB0EE674AA4EEF0
:10D99800854AF4EEC46AF1EE10FAF0EE444A88BF04
:10D9A800F0EE474AFDEEE44A14EE900A14EE906A4F
:10D9B8009842A8BF1E468842B8BF0E4604EE906A39
:10D9C800F8EEE44A062ACCED054A3DF478AAD8EDEB
:10D9D800184A9DED124A65EEA44AE4EE064AB0EEF6
:10D9E800674AA4EE854AF4EEC46AF1EE10FAF0EE46
:10D9F800444A88BFF0EE474AFDEEE44A14EE900A26
:10DA080014EE906A9842A8BF1E468842B8BF0E46D8
:10DA180004EE906AF8EEE44A072ACCED064A3DF493
:10DA28004EAAD8ED1C4A9DED134A65EEA45AE6EEBF
:10DA3800045AE5EE257AF4EEE76AF1EE10FAC8BF6B
:10DA4800F0EE477AFEF7D9B93849394A8968126839
:10DA580091423FF6DBA998F800200C3A022A7DF69D
:10DA680005AF94F88C2188F80030002A3DF4FEAE0A
:10DA7800FFF702BA9FED2F7AFFF75ABB2E4B4FEAFA
:10DA8800890E5FEA9A0901EB0E0C03EBC818A6444D
:10DA980000F0198509F101094FEA091908EB090095
:10DAA80008F110030CF110010EF1100213ED024AF7
:10DAB80013ED035A13ED016A13ED047A51ED024A8E
:10DAC80051ED035A51ED016A51ED047A64EE244A8E
:10DAD80065EE255A66EE266A67EE277A1033984275
:10DAE80042ED024A42ED035A42ED016A42ED047AE0
:10DAF80001F1100102F11002D8D1A9F11009C844AE
:10DB08000CEB0901CE441AF0030A3EF4E3ADB8EC7D
:10DB1800017AF1EC017A67EE277ABAF1010AEEECA4
:10DB2800017AF4D1FEF7D6BD00000243FC130020B1
:10DB38002C56002000000000284A002054540020E1
:10DB4800BAF1000F00F09083DFF85C869DED0C4A77
:10DB5800D8ED004A65EEA44AE4EE064AB0EE674AFC
:10DB6800A4EE854AF0EE444AB9F1000F06D0F4EE6F
:10DB7800446AF1EE10FAC8BFF0EE474ABDEEC77A24
:10DB880017EE101ABDEEE47A04EE901A17EE100A9A
:10DB9800814200F388849842A8BF184607EE100A0D
:10DBA800B8EEC77ADFF804C6012A8CED007A3DF496
:10DBB8008BA998ED047A9DED0D4A25EE877AA4EE9F
:10DBC800067AB0EE674AA7EE054AB0EE447AB9F194
:10DBD800000F00F05784F4EEC46AF1EE10FA40F337
:10DBE800518408469842A8BF184607EE100AB8EEB6
:10DBF800C77A022A8CED017A3DF466A998ED087A75
:10DC08009DED0E4A25EE877AA4EE067AB0EE674AB5
:10DC1800A7EE054AB0EE447AB9F1000F00F0278468
:10DC2800F4EEC46AF1EE10FA40F3218408469842F3
:10DC3800A8BF184607EE100AB8EEC77A032A8CED7B
:10DC4800027A3DF441A998ED0C7A9DED0F4A25EE34
:10DC5800877AA4EE067AB0EE674AA7EE054AB0EED8
:10DC6800447AB9F1000F00F0F883F4EEC46AF1EEDB
:10DC780010FA40F3F28308469842A8BF184607EE08
:10DC8800100AB8EEC77A042A8CED037A3DF41CA971
:10DC980098ED107A9DED104A25EE877AA4EE067A63
:10DCA800B0EE674AA7EE054AB0EE447AB9F1000F24
:10DCB80000F0C983F4EEC46AF1EE10FA40F3C383AE
:10DCC80008469842A8BF184607EE100AB8EEC77A69
:10DCD800052A8CED047A3DF4F7A898ED147A9DEDA9
:10DCE800114A25EE877AA4EE067AB0EE674AA7EEC7
:10DCF800054AB0EE447AB9F1000F00F09A83F4EEC9
:10DD0800C46AF1EE10FA40F3948308469842A8BF1B
:10DD1800184607EE100AB8EEC77A062A8CED057A7F
:10DD28003DF4D2A898ED187A9DED124A25EE877A2F
:10DD3800A4EE067AB0EE674AA7EE054AB0EE447A3A
:10DD4800B9F1000F00F06B83F4EEC46AF1EE10FA3B
:10DD580040F3658308469842A8BF184607EE100AA4
:10DD6800B8EEC77A072A8CED067A3DF4ADA898ED8F
:10DD78001C7A9DED134A65EE875AE4EE065AE5EEE5
:10DD8800857AB9F1000F00F04283F4EEE67AF1EEFD
:10DD980010FA40F13C830A469A42A8BF1A4604EE9C
:10DDA800902AF8EEE44ACCED074AFDF78DB807EE65
:10DDB800903ADFEDED6AB8EEE77A66EEA65A9FED87
:10DDC800EB5A9FEDEB6ADFEDEB7AA5EE856A26EE5E
:10DDD800A55AE5EE867AE5EE276A26EE870AFFF76A
:10DDE800A0B9D8ED006ADDED0C4A65EEA66AE4EE4E
:10DDF800866AF0EE674AE6EE854AFDEEE46A16EEBC
:10DE080090EA714500F341819E45A8BF9E4606EE03
:10DE180090EAF8EEE66A002E00F06A84DFF88CC318
:10DE2800012ACCED006A3DF44FA8D8ED046ADDED77
:10DE38000D4A65EEA66AE4EE866AF0EE674AE6EEFB
:10DE4800854AFDEEE46A16EE90EA714500F3FA8120
:10DE58009E45A8BF9E4606EE90EAF8EEE66A002EBA
:10DE680000F03B84022ACCED016A3DF42DA8D8EDE0
:10DE7800086ADDED0E4A65EEA66AE4EE866AF0EE03
:10DE8800674AE6EE854AFDEEE46A16EE90EA7145C9
:10DE980000F3D5819E45A8BF9E4606EE90EAF8EEAF
:10DEA800E66A002E00F0EA83032ACCED026A3DF40C
:10DEB8000BA8D8ED0C6ADDED0F4A65EEA66AE4EE14
:10DEC800866AF0EE674AE6EE854AFDEEE46A16EEEB
:10DED80090EA714500F3B0819E45A8BF9E4606EEC4
:10DEE80090EAF8EEE66A002E00F0BE83042ACCED34
:10DEF800036A3CF4E9AFD8ED106ADDED104A65EE2F
:10DF0800A66AE4EE866AF0EE674AE6EE854AFDEE1A
:10DF1800E46A16EE90EA714500F38B819E45A8BF2E
:10DF28009E4606EE90EAF8EEE66A002E00F085833B
:10DF3800052ACCED046A3CF4C7AFD8ED146ADDEDD0
:10DF4800114A65EEA66AE4EE866AF0EE674AE6EEE6
:10DF5800854AFDEEE46A16EE90EA714500F3758194
:10DF68009E45A8BF9E4606EE90EAF8EEE66A002EA9
:10DF780000F0A983062ACCED056A3CF4A5AFD8EDDC
:10DF8800186ADDED124A65EEA66AE4EE866AF0EEDE
:10DF9800674AE6EE854AFDEEE46A16EE90EA7145B8
:10DFA80000F33F819E45A8BF9E4606EE90EAF8EE34
:10DFB800E66A002E00F0BB83072ACCED066A3CF423
:10DFC80083AFD8ED1C6ADDED134A65EEA65AE4EE80
:10DFD800865AE5EE257AFDEEE77A17EE902A914209
:10DFE80003DC9A42A8BF1A46114607EE901AF8EECB
:10DFF800E77A002E7FF40FAA069B002B7FF40BAA6A
:10E00800059B5B45B8BFF0EE477AFFF704BA77EE99
:10E01800C76AF0EE477AFEF765BDBCF834309FED6D
:10E02800567A07EE903AF8EEE77A544B67EE877A1D
:10E03800C3ED007AFCF7A3BE514B1E6816F080565C
:10E048007FF499A8FFF792B84E4BFCF7EFBE4E4B02
:10E058001B78032B00F041820023FEF77CBE9FED66
:10E068004B8AFFF7ECB99FED498AFFF71CBA9FED81
:10E07800480ADFF83C8125EE800A1FF019FFD4F822
:10E08800A861A8F80600FBF7ACBE06EE901AC0E639
:10E0980093ED000A0593079106921FF009FFDFF838
:10E0A80014E1DFF814C1DEF8ECE0DFF80481069A29
:10E0B800A8F800008CFB0E3C4FEAEE7ECEEBAC1EBF
:10E0C80007EE90EAF8EEE77A059B0799FDEEE77A06
:10E0D80017EE900AA8F80200FCF7ADBE07EE907A9A
:10E0E800F8EEE78ADFED2B7A9FED340A84F8847125
:10E0F80068EEA78A38EE800AFDEEC07A17EE903AED
:10E108002033402B40F2C9819FED200A1B4BFDEEC6
:10E11800E87A83ED010A17EE903A2033402B00F29B
:10E12800BF81DFED277AF4EEE78AF1EE10FA40F3CB
:10E13800FB81DFED196ADFED197A01E0F0EE478A1D
:10E14800F4EEE78AF1EE10FA38EEE67AF6DCDFED67
:10E15800147AB4EEE77AF1EE10FA40F15E829FEDA0
:10E168000E6ADFED106A35E084F9223F92E741B983
:10E178009730083C15A82ABE6F12833A7800002011
:10E1880014540020D06200208651002000000000B6
:10E198000000C84235FA8E3CDB0FC940E4CB16417B
:10E1A800DB0F49C0E4CB16C1A4380020545400202A
:10E1B800FC6100200C100020D34D6210DB0FC93F1A
:10E1C800DB0F494092E741B99730083C15A82ABEB1
:10E1D800B0EE677AB4EEE67AF1EE10FA77EE067AE8
:10E1E800F6D41FED0A7AF4EEC77AF1EE10FA40F38E
:10E1F8005E811FED0D7A77EE677A27EEA76A5FEDED
:10E208000F5A5FED0F6A1FED0F7AE6EE256A67EE8B
:10E21800865AA6EE267AE5EE877AC4ED627AFDF78D
:10E228009ABE06EE901AC2E6C149C24A8C46FEF76B
:10E2380040BA06EE901A76E606EE901A51E606EE19
:10E24800901A2CE606EE901A07E606EE901A8CE66F
:10E25800F2F74CFEB84BDFF80C831F78069BC01A08
:10E26800A8F80200FEF753BAFDEEC74A0DF1300ECA
:10E278009A46DFF8F4C2DFF8F48214EE901A0EEB37
:10E2880082024B4606E07245E8EC014A0CF1100C9C
:10E298003CF41AAEDCED004ABEEC014A65EEA44A35
:10E2A800E6EE044AB0EE674AA5EE244AF0EE444A88
:10E2B80033B1F4EE446AF1EE10FAC8BFF0EE474A03
:10E2C800FDEEE44A14EE909A494504EE901A04DCF7
:10E2D800D145A8BFD14604EE909AF8EEE44A002E44
:10E2E800D1D106980028CED105985845B8BFF0EE90
:10E2F800474AC8E7F2F7FAFD069BDFF86882D4F8C8
:10E30800AC91D4F8A861C01AA8F80200FEF761BA67
:10E318008A4A126802F59C520832C4F8902198F88B
:10E328000020012A7DF4A2AA94F88C21002A7DF409
:10E338009DAA032B00F091811FF034FA012384F881
:10E348008C31FDF793BAF2F7D1FD7B4BDFF81482DD
:10E358001F78069B99F80020D4F8A861C01AA8F87D
:10E368000400FEF794BBDFED767AF4EEE76AF1EE8F
:10E3780010FA40F3CB81DFED735A9FED736A01E029
:10E38800F0EE676AF4EEC66AF1EE10FA76EEE57A18
:10E39800F6DCDFED6E6AF4EEE67AF1EE10FA40F1A3
:10E3A800B281DFED685A9FED6A6A01E0F0EE667AA5
:10E3B800F4EEC67AF1EE10FA77EEA56AF6D4DFED40
:10E3C800657AF4EEE76AF1EE10FA04DDDFED5C7AC7
:10E3D80077EEE66AF1E4DFED607AF4EEE76AF1EEF3
:10E3E80010FA44BFDFED597A77EEE66AE5E409985A
:10E3F80013F004FBFEF783BD4E4800F1800CFEF7D6
:10E408002DBBA8F80600A5F8B460FCF7E3BBFDEE49
:10E41800E77A17EE902A8A42FFF6C3ACBCE4BDEE59
:10E42800C77A17EE100A8842BFF695AC07EE101AA5
:10E4380096E4BDEEC77A17EE100A8842BFF666ACBE
:10E4480007EE101A67E4BDEEC77A17EE100A884285
:10E45800BFF637AC07EE101A38E4BDEEC77A17EEF0
:10E46800100A8842BFF608AC07EE101A09E4BDEEA0
:10E47800C77A17EE100A8842BFF6D9AB07EE101A12
:10E48800FFF7DABBBDEEC77A17EE100A8842BFF66F
:10E49800A9AB07EE101AFFF7AABBF4F783FD35E620
:10E4A800DFED2E7AB9E607EE101AFFF779BB9FED7C
:10E4B8002A7AF4EEC77AF1EE10FA44BF9FED237A78
:10E4C80077EE677A99E66146FFF71DBBF4F778FEA9
:10E4D80000283EF4DFACFEF7D7BC03F023FDFCF7C1
:10E4E80071BB80200EF01AFE08B102F0C9FF1FF0C0
:10E4F80059F9FEF70DBD94F8E031002B7BF4DAAE44
:10E50800FBF7C5BEDFF86890D9F8000002F08CFF71
:10E51800134B1B780022022BC9F800207EF4D7ACDD
:10E5280003F02EFCFEF7D3BCB0EE687A0FE600BF0E
:10E53800A84B00200C210020F86100206C57002017
:10E54800DB0F4940DB0FC940E4CB1641DB0F49C064
:10E55800E4CB16C1DB0FC93FDB0FC9BF00000000C9
:10E5680024560020FC610020A438002054540020C8
:10E5780078700020734A744B10681B689847089B92
:10E58800DBED007A93ED007A704BD7ED006A83EDEE
:10E59800020A6F4B67EE277A2B4427EE8C7AD3ED6D
:10E5A800007A6C4B67EE277AF0EE665AE7EE8D5AE2
:10E5B80093ED006AB1EE467AB4EEE57AF1EE10FA20
:10E5C80031DD654B1B78012B02D0192B7BF4E9ADAB
:10E5D800DFED627AB4EEE7DAF1EE10FACCBF012390
:10E5E8000023FBF7E9BD5E4BD3ED007AB1EE677A05
:10E5F800B4EEC7DAF1EE10FA12D4B4EEE7DAF1EEBF
:10E6080010FA88BFB0EE67DA564BC7ED00BA1B6840
:10E618009342BBF687ADFCF7A4BEF0EE477AE0E57F
:10E62800B0EE47DAF0E7B4EEE56AF1EE10FA8CBF27
:10E63800B0EE657AB0EE467AC3E7069800287FF414
:10E6480077AC05985845B8BFF0EE476A70E4CB5CE4
:10E65800002B7EF41FACFEF708BD80200EF05EFD97
:10E6680000287DF403A967E6069800287FF43EACED
:10E6780005985845B8BFF0EE476A37E40698002871
:10E688007FF412AC05985845B8BFF0EE476A0BE422
:10E69800132B05D1B0EE480A1FF00AFCAAF80000B7
:10E6A800B0EE480AD5F814322F4898472F4B1B78FC
:10E6B800132BB0EE408A7BF4D5AB1FF0F9FBAAF818
:10E6C8000200FBF7CFBB069800287FF453AC0598EF
:10E6D8005845B8BFF0EE476A4CE4069800287FF426
:10E6E800C1AB05985845B8BFF0EE476AFFF7BABB0B
:10E6F800069800287FF492AB05985845B8BFF0EE0D
:10E70800476AFFF78BBBF0EE676A58E6F0EE667A69
:10E718003FE645201EF012F8FF201EF00FF81448BF
:10E728001DF080FF48461EF009F8FEF79FBB0698CB
:10E7380000287FF441AC05985845B8BFF0EE476A09
:10E748003AE400BF6C3500208035002020540020BA
:10E7580090350020F8350020543300200000964200
:10E76800F4350020D835002048670020F8610020E3
:10E77800682F03082DE9F04F2DED028B984B994A2D
:10E788001C7893B000F59C412031814606911160B8
:10E79800002C00F07C86944A1268904240F28A80ED
:10E7A800924A93491768934DDFF888B20492013C66
:10E7B80002911C7007F48057002F40F08880029B5C
:10E7C8005B7D002B40F02D86049B1B681E0401F125
:10E7D800FF80894B99459BF8023000F20085002B99
:10E7E80040F00185854B0593049B1F6817F48059F9
:10E7F80040F0BB85029BB5F906605B8B9E42B4BFB7
:10E80800002601267E4B1B6813F0805369D0059AB9
:10E81800127812F001026AD002987A49408C91ED80
:10E82800037A039107EE900AF8EEE77AB4EEE77AF6
:10E83800F1EE10FA81F28081002E60D1724C94F8CA
:10E84800A01000295BD171487149006890F82D002B
:10E8580000240C604C608C606E49002850D1087010
:10E86800002A51D0F8064FD56B4A1278D1064BD4FE
:10E87800B9F1000F48D1002B46D17A0244D4674B36
:10E888001B78002B01F0FD86654B9B78002E41F02C
:10E8980030873BB1634A644B12681B689B1A002B94
:10E8A800C1F21F871020584C03F058FB012384F84D
:10E8B800A13029E04D4B4E4A1F68049307F4805756
:10E8C80002924C4DDFF86CB1002F3FF478AF002175
:10E8D8004B48F4F73FFC00287FF471AF15F0EEFECB
:10E8E8006DE77C0293D4059A127802F00102464C37
:10E8F800002184F8A01043490391002EA3D0454974
:10E9080001200870002AADD1484B1A78002A50D14E
:10E918000299B5F900E0488B898BB5F9024070453A
:10E92800B4BF8027002747F040037145D8BF3B4656
:10E938009B0843F08007A042B8BF3B4643F040071E
:10E94800A142C8BF3B469B08B5F90440B5F906701B
:10E9580043F0800EA042B8BF734643F0400EA14278
:10E96800C8BF73469B0843F0800E274C8742C8BF38
:10E97800734643F0400E94F8A2C08F42B8BF734666
:10E988009C4501F0BF82A4F8A42084F8A62023495E
:10E9980084F8A2300F78002F01F01F825F2B01F05E
:10E9A8008B826F2B01F02481059B1B78DE0741F1D8
:10E9B800E880049B1B6803F00403002B40F02086CA
:10E9C8000DF140081A4C0022C8F8042004F150093F
:10E9D800109240F6330A192740F283362FE000BF21
:10E9E800B04D002064490020AC4D0020E4600020B8
:10E9F8005C3E0020506F0020404B4C004D3C0020F6
:10EA080014540020D062002020230020F83A00206F
:10EA18002C540020EC2200201C540020221C002032
:10EA2800205600206C570020A0580020144F0020CA
:10EA3800485600209C51002004344C4520D0A27830
:10EA4800E3789A4217FB0261F6D26278043217FB28
:10EA5800036335F912205245A8BF5246B2F5617FCB
:10EA6800B8BF4FF461728A42E6DD9A42E4DC21784D
:10EA78002429E1D840460434F4F75CFB4C45DED148
:10EA8800624A634B177898E8030083E80300002F75
:10EA980000F03F855F4B07935D480121F4F75AFB6F
:10EAA800002840F0A9829BF80330002B40F0A48294
:10EAB800594B0693594C23881EB226F001061FFABB
:10EAC80086F84345A4F8008000F0E187544E4FF0E3
:10EAD80002090E2014274FF0FF0A86F8009077707D
:10EAE80086F802A003F03AFA49464948B4F800808B
:10EAF800F4F730FB002841F0AB8128F002039BB209
:10EB0800434523800BD0464B1421FF2202260E20BA
:10EB18001E7059709A7003F021FAB4F80080414BC6
:10EB2800414A19785068099318F0030F08BF81F01B
:10EB38000201C1F340010892F3F7B8FB24213448DD
:10EB4800F4F708FB30B9059A13785E0744BF23F041
:10EB580004031370069B1B6813F00A0F1AD00621D2
:10EB68002B48F4F7F7FA002800F0B48723885806F2
:10EB780041F1B28007212648F4F7ECFA50B12B4B4B
:10EB88002B4AB3F904302B4982FB0302DB17C3EB92
:10EB9800A2030B800C211E48F4F7DCFA2288002817
:10EBA80000F04A8242F480739A42238009D01C4BB9
:10EBB80002201421FF2218700E2059709A7003F059
:10EBC800CDF91D4B1B78082B00F042820E2B00F06C
:10EBD8003F82049B1B68590561D5184B1B79002B94
:10EBE80000F0258114210A48F4F7B4FA002840F00F
:10EBF800238112F037FA012003F08CF800284ED058
:10EC0800DFF83C9000264FF0CC0A1EE0E73A0020DF
:10EC180014540020F46F0020203B00208251002073
:10EC28004C39002034570020385700206C3B002016
:10EC3800676666669C58002044560020C062002023
:10EC4800A06B0020DEB2022E29D80AFB06F8731C3E
:10EC580059F80870002FF5D1C378D04A90F902000E
:10EC680052F8233001970322009201213A4602F01C
:10EC78001FFC034606EB460000EB0010069353B159
:10EC8800394609EB8000CC2221F01FFA069B49F88F
:10EC980008300136F6B218F0B9F90028D3D1059B2F
:10ECA8001E7816F0010600F02982BD4B01221A7069
:10ECB800079BB5F906101B68BA485A890127914283
:10ECC800077080F20182B84B4FF07E521A60B74A43
:10ECD800029BB5F900E01F8B92F90430107892F886
:10ECE80001C0002BAEEB070314BF01224FF0FF3227
:10ECF800002BB8BF5B42B3F5FA7FA8BF4FF4FA7395
:10ED0800984280F2DE811B1A07EE903AF8EEE77A15
:10ED1800039BBE45C3ED007A03DAF1EE677AC3EDD3
:10ED2800007AB5F902E0AEEB0703002BB8BF5B42EF
:10ED3800B3F5FA7FA8BF4FF4FA73984280F2BE8108
:10ED48001B1A07EE903AF8EEE77A039B7745C3ED76
:10ED5800017A03DDF1EE677AC3ED017AB5F90400B3
:10ED6800C31B002BB8BF5B42B3F5FA7FA8BF4FF4B3
:10ED7800FA736345CCBFA3EB0C03002302FB03F338
:10ED880007EE903A039A049BF8EEE77AB842C2ED90
:10ED9800027ABCBFF1EE677AC2ED027A1A6812F401
:10EDA800805200F06881B1F5FA6F814BA8BF4FF42B
:10EDB800FA61B1F57A7F1878B8BF4FF47A71A1F586
:10EDC8007A71002840F070817A4D7B4885FB013EBE
:10EDD800CB17C3EB6E1303F1010E6FF0630C30F920
:10EDE8001EE030F913000CFB0313AEEB000103FB2C
:10EDF80001F385FB0315DB17C3EB651303441BB253
:10EE080007EE903A039BB8EEE78A83ED038A002A5F
:10EE180040F03C8423885B0624D4002E40F0B08068
:10EE28001DF0D7F913B0BDEC028BBDE8F08F059B40
:10EE38001B78DA077FF5DDAE3C200EF06FF900286D
:10EE48003FF42DAF02F01CFB3C200EF009F900281E
:10EE58003FF425AF02F014FB3C200EF001F9002826
:10EE6800F0D11CE7554B564AB3F904305549DFED4C
:10EE7800566A09889FED557A82FB0302DB17C3EBBC
:10EE8800A2035B1A1BB207EE903AF8EEE77A67EE38
:10EE9800A67A77EE876ABDEEE66A16EE103A203358
:10EEA800402B40F22587DFED4A6ABDEEE77A17EE80
:10EEB800103A2033402B00F217879FED467AF4EE84
:10EEC800C77AF1EE10FA41F3AF82DFED435A9FEDB6
:10EED800436A01E0F0EE477AF4EEC67AF1EE10FAF2
:10EEE80037EEE57AF6DCDFED3E7AB4EEE77AF1EE5E
:10EEF80010FA41F19D82DFED385A9FED3A6A01E040
:10EF0800B0EE677AB4EEC67AF1EE10FA77EE257AAB
:10EF1800F6D49FED2E7AF4EEC77AF1EE10FA00F3EC
:10EF280023869FED317AF4EEC77AF1EE10FA44BFEA
:10EF38009FED2B7A77EE677A67EEA75A9FED2B5AEB
:10EF48009FED2B6A9FED2B7AA5EE856A27EEA55AD1
:10EF5800A5EE867AE5EE077A039A92ED016AD2ED7C
:10EF6800005A27EEC67A65EEA77AA5EEA67AE6EEEF
:10EF7800267A82ED007AC2ED017A002E3FF450AF76
:10EF8800099B1978089B01F001011868F3F78EF9BD
:10EF980013B0BDEC028BBDE8F08F00BF6C230308F3
:10EFA8004E3C002024220020C8220020FC550020CE
:10EFB800C02400201F85EB51F86F00206C3B002017
:10EFC800676666669C58002035FA8E3CDB0FC93FA1
:10EFD80000000000DB0F4940DB0FC940E4CB1641BD
:10EFE800DB0F49C0E4CB16C1DB0FC9BF92E741B9BB
:10EFF8009730083C15A82ABEB64B06931B689F0796
:10F008007FF558ADB44CB4F8008018F0010F7FF4C8
:10F0180074AD48F00103984523803FF46EADAF4BC3
:10F02800022214211A700E20FF2259709A7002F0E1
:10F0380095FFB4F8008060E522F480739BB29A4291
:10F0480023807FF4B4ADA64B1B78082B7FF4BEADAC
:10F05800228822F040039BB29A4223803FF4B9AD44
:10F068009E4B02201421FF2218700E2059709A70AE
:10F0780002F074FFADE5029B588B8142C0F2148404
:10F08800B1F5FA6FD4BFC0EB0101C0F5FA614FF4D6
:10F098007A7303FB01F1934B1D78C0F5FA60B1FB5D
:10F0A800F0F1002D3FF490AE5B788F4801FB03F33D
:10F0B80080FB0301DB17C3EB611185E6DFED8B7A7B
:10F0C80043E6DFED8A7A23E6B1F5FA6F80F2EF8343
:10F0D800187A8B1A03FB00F3C2F5FA6293FBF2F37A
:10F0E800C3F1640307EE903AF8EEE77A9FED807A71
:10F0F800804B67EE877AC3ED007AE8E57E4B1B7894
:10F108000693002B7FF4D4ADDFF81CA2DFF81C9225
:10F118001AF8030C99F800805146AAF103071CF06D
:10F12800D5FD002800F0C983069BB8F1000F53D124
:10F1380007F1080178791CF0C9FD002841F0D98150
:10F148006E49B87A1CF0C2FD002800F0CA83B8F1F5
:10F15800020F41F0D1816A49F87B1CF0B7FD002805
:10F1680041F0A7816749387D1CF0B0FD002800F008
:10F17800CA83B8F1040F41F09F816349787E1CF07F
:10F18800A5FD002841F09B816049B87F1CF09EFDD9
:10F19800002800F0CA83B8F1060F41F093815C495A
:10F1A80097F823001CF092FD002840F04487594945
:10F1B80097F828001CF08AFD002800F0CA83B8F1EF
:10F1C800080F40F04987544997F82D001CF07EFD40
:10F1D80000283FF46DAD09231A4600F02EBF13B97D
:10F1E80001238BF802304D4B05931B201F789BF8A9
:10F1F80021601CF095FD012E07F00109824600F000
:10F20800578607F0020303939BF82030DFF820812C
:10F21800434C052B00F29C80DFE813F08C00500073
:10F228000600DD000101BF00012E04BF05238BF895
:10F238002030B9F1000F00F01581029B394FB3F966
:10F248001810B8F80030002261F30F0263F31F4270
:10F25800002361F30F0361F31F436A603968DBF829
:10F2680014202B608A42C0F04E84012E41F07B822C
:10F2780003229BF820300392CBE71CF07DFD012888
:10F2880008D1284FB8F802303A68642101FB0323FB
:10F29800CBF81030BAF1000F04D098F80630002BE4
:10F2A80040F09080012E53D01E4FDBF810203B68B1
:10F2B8009A42C0F0788601238BF82030012E6CD05A
:10F2C80098F80730012B00F0D78009F08FFA9BF8E7
:10F2D80020309EE7203B0020825100204C3900203E
:10F2E80044560020C02400201F85EB510000000078
:10F2F8000AD7233CC82200204E3C00205838002062
:10F308005D38002062380020673800206C38002003
:10F3180071380020763800207B3800204D3C0020D2
:10F32800C05100206C5700204E380020800000207B
:10F3380044390020B9F1000F9FD14FF48060BAF131
:10F34800000F00F0C4831DF0CFFB0023CBF8103072
:10F35800039B002B3FF448AA039802F0FFFD049B8F
:10F368001F6817F480593FF445AA1D21B648F3F7E2
:10F37800F1FE00287FF43EAAB44A029BD2881B8B78
:10F38800B5F90660991A8E4240F3028613449E42EC
:10F39800B4BF00260126FFF735BAAD4F3A68B8F872
:10F3A8000230642101FB03234FF480600022CBF874
:10F3B80010308BF820208BF803201DF07DFB9BF884
:10F3C800203026E709F012FA03224FF47A738BF8FB
:10F3D8002020CBF81C309E4F238843F00203238063
:10F3E80015F06CF93A68DBF81C3013440422CBF8AA
:10F3F80018308BF82020012E40F0CD853B68DBF8D3
:10F4080018209A42A4D2934B187818B91CF088FC9B
:10F4180000289DD1238823F002032380BEE78C4F68
:10F42800E9E7029A013BD27D35F91330002A40F012
:10F438006583A3F57A73B3F57A7FA8BF4FF47A731F
:10F4480023EAE37307EE903A9FED837AF8EEE77AC2
:10F4580067EE877A814AFCEEE77A17EE903A1380D6
:10F46800FFF7B7B97A4F3B6847F230520323CBF81E
:10F478001C208BF82030AFE709F0B8F9032240F6DA
:10F48800B8338BF82020CBF81C30714FA4E7744FA9
:10F498003B78002B00F0DC87724BDFF8DC81DFF86B
:10F4A800DCB1DFF8DCA1029345465E46039099463D
:10F4B8000EE019F804109847032C28DC88B93B782B
:10F4C8002AF8020F01349C4205F1040580F20C81F0
:10F4D800072CE1B23046DBF80430EADD984700B289
:10F4E800EDE738F824206B88801A4FF47A719B1A5C
:10F4F80001FB00F040F6CA0290FBF3F0084490428A
:10F5080040F2EE23A8BF10469842B8BF184600B292
:10F51800D5E7DFF870A1DFF87081534C0AF15A067D
:10F528004FF0010951461AF8010C1CF0CFFBF8B155
:10F538009AF804009AF802309AF803E000EB4001C8
:10F5480004EB8101013BD1F8B42003EB43034344AE
:10F5580093420DD094F8E02081F8B0E009FA00F069
:10F5680022EA0000C1F8B430C1F8B87084F8E000AD
:10F578000AF1060AB245D5D13C4B07931946344ADD
:10F588003B4B3C4C09681B78D2F8009008910693D5
:10F59800A4F1B00A002663685BB31F784FB3A26872
:10F5A800A9EB0202002A0ADB9AF8E0200121B14007
:10F5B80022EA010209F5FA718AF8E020A160069AA8
:10F5C800BAB1227859780432D2B2002940F0BA820E
:10F5D800029935F91220098B01F1C800824240F3E3
:10F5E800A9849AF8E0109A7841FA06F3D90740F10D
:10F5F8001D850136042E04F10C04CCD1FFF74CBA5A
:10F60800194C94F8AA3053B1059B1B78D80706D536
:10F61800029BB5F906205B8B9A4200F3DC8411212A
:10F628000948F3F797FD002800F0748294F8AE308B
:10F638002BB994F8A83013B93223A4F8AC300123BD
:10F6480084F8AE30FFF7BCB9145400202C390020E0
:10F658006C570020221C0020AAF1823F8051002014
:10F66800245A00205C3E002020230020F46F002054
:10F6780051510020D02300203C5A0020943B002008
:10F688001E23002065370020200A03081D21B748E3
:10F69800F3F760FD00283FF4BDAB9BF80330002B67
:10F6A8007FF4B8ABDFEDB27AB24938EE678AC7F5B6
:10F6B800FA63FDEEC87A1BB2CDED027ABDF90820D7
:10F6C800120381FB0201D217C2EBA11203FB02F362
:10F6D80043F30F333B4407EE903A039BF8EEE77A87
:10F6E800C3ED037AFFF796BBDDF80C90A24A0492AB
:10F6F8001146A04A096842F2010AA2FB092B11EA45
:10F708000A0A4FEA9B1B00F001829C4D9C489D4CC5
:10F718009D4A95F800E0007884F800E01070BEF18A
:10F72800000F04D0984A92F800E08EF0010E974C32
:10F738000F2084F82400002B00F05C83944B0B937B
:10F748001B780A931E463B78029F924AB7F824C05A
:10F75800DFF8748209903D46FF8C08973746A2FB74
:10F76800066252082D8B0E9502EB420294F8255042
:10F778000C95BA1AD2B201F48051079204F1280606
:10F788000BF596726746844DCDF80CE0A4465446B6
:10F79800DDF830A00F9100200592CDF834909E46F8
:10F7A800039B002B00F03D823CF910101FFA81F9F1
:10F7B800B9454FEA400203D3089B994540F273824A
:10F7C80058F820108B4580F03582A95E002C40F057
:10F7D800498201307045A95206F10606E0DB099816
:10F7E8006E4ADDF834908CF824000F2864465146A0
:10F7F8000CBF01210021734684F825A0117000F088
:10F80800FF82DFF8C8B1664E664F34883868DBF887
:10F818000810DBF80420CBF80C0044F00404401A6C
:10F828009042574F3480584C4FF0010188BF002256
:10F838003970217088BF8BF82120002B00F0F582E9
:10F84800049A02991768584EB1F824C0B1F818E024
:10F85800514817F48057344640F00C8339460EE07F
:10F86800627802EB820202EB820202F2EE2292B28C
:10F8780001318B4220F8022B04F102040ED016F855
:10F888001120002A00F01382022AE9D001310288EF
:10F8980020F8022B8B4204F10204F0D10B9A137862
:10F8A80001331370FEF788BF1146FFF7F4BB1B7ACC
:10F8B800C3F1640307EE903A16E40AF1050178797A
:10F8C8001CF004FA00283FF43BACB8F1010F40F0FB
:10F8D800108607F10D01B87A1CF0F8F9002840F0FD
:10F8E8000B863249F87B1CF0F1F900283FF43AAC5A
:10F8F800B8F1030F40F0DD852D49387D1CF0E6F99D
:10F90800002840F0D9852B49787E1CF0DFF90028C3
:10F918003FF43AACB8F1050F40F0D1852649B87FDD
:10F928001CF0D4F9002840F0CD85244997F823002D
:10F938001CF0CCF900283FF43AACB8F1070F40F0BE
:10F948007A831F4997F828001CF0C0F9002840F076
:10F9580083831C4997F82D001CF0B8F900283FF460
:10F96800A7A9B8F1090F3FF4A3A934E4145400205F
:10F9780000007A44D34D6210E46000204049002022
:10F988004801002051510020490100202023002077
:10F99800D1590020ABAAAAAA506F0020923B0020A0
:10F9A800C05100206C570020705A00205D3800209C
:10F9B80062380020673800206C3800207138002039
:10F9C800763800207B380020D45900209C51002034
:10F9D800CD4CD4F88830A9EB0303002BFEF6F9AE22
:10F9E800CA4A94F88C30517C069AC4F888200133AE
:10F9F800C74A029E32F81120B17D03F00F0384F844
:10FA08008C30234492B292FBF1F283F8902094F860
:10FA1800901094F8912094F8923094F89C000A443D
:10FA280094F89310134494F89420194494F895305A
:10FA38000A4494F89610134494F89720194494F8BB
:10FA480098300A4494F89910134494F89A20194469
:10FA580094F89B300A44134494F89D1094F89F201E
:10FA6800184494F89E3001440B441A4442F30B1294
:10FA7800642AF17DA8BF642213B209B1C2F16403FC
:10FA880007EE903A9FEDA37AF8EEE77AE0E40221D8
:10FA9800A148F3F75FFB00283FF42FA8268018F051
:10FAA800020F7FF43CA848F00203434523803FF44B
:10FAB80036A89A4B022214211A700E20FF22597080
:10FAC8009A7002F04BFAB4F80080FFF728B81CF0DF
:10FAD800F3FF3AE4228822F040039BB29A42238043
:10FAE8003FF448A88D4B02201421FF2218700E20E5
:10FAF80059709A7002F032FAFFF73CB8C3F53B63CD
:10FB080008331BB295E403230393ADE4844A92F8C7
:10FB180000E004E694F8A830002B3EF451AF059BB2
:10FB28001B7813F001037EF44BAF012284F8A83050
:10FB380084F8A920FEF744BF734C012184F8A01073
:10FB4800FEF7DDBE012900F032849AF8E020012397
:10FB5800B34001361343042E8AF8E03004F10C0454
:10FB68007FF419ADFEF798BF9FED797A77EE677A43
:10FB7800FFF7E2B9059B6B4A1B781060DB0700F1C1
:10FB8800388294F8A60000287EF413AFB4F9A430A4
:10FB9800322B7EF70EAF94F8A2200121572A84F861
:10FBA800A61000F09284049B1B6813F0040302D093
:10FBB8005A2A00F04F855D2A00F0FB845B2A00F08A
:10FBC80021855E2A00F02285562A00F03485972A7E
:10FBD80000F02785A72A40F0B3845349049B0A788C
:10FBE8001B6842F004020A7003F00403FEF7E5BE46
:10FBF800B2F5FA7FFEF6DDAE94F8A620002A7EF470
:10FC0800D8AE059B1B780121DF0784F8A61000F108
:10FC18008F8414F099F8049B1B6803F00403FEF723
:10FC2800CCBE002F3DD058F820108B454FEA40023B
:10FC3800FFF4CBAD3D4B995C03EB0209002900F0C2
:10FC4800F980022946D199F8011001EB810101EBF5
:10FC5800810101F2EE2189B2032832DD09B2002CBC
:10FC68003FF4B7AD079B26F81310BAF1000F03D184
:10FC78000A9B022B7FF6ADADB6F800A07188B6F8E6
:10FC880004902B4B514489440FFA89F983FB0931BD
:10FC9800284BA1EBE97123F8029009B24FF0010A51
:10FCA80097E539464200059B48F820308EE5CAB2F0
:10FCB800022A04D9032A7FF4E9AD6246D8E57246E0
:10FCC800D6E5012303FA00F9099B23EA090309B2DF
:10FCD80009937BE5A95ABFE743F04002934222808B
:10FCE8007FF400AFFEF746BFDFED137AFFF734B9B4
:10FCF800F4EEC77AF1EE10FA40F3A783DFED115A5C
:10FD08009FED0E6A2EE000BF20230020AC64002087
:10FD1800C864002014AE2341145400204C3900203C
:10FD280051510020A45800201C540020705A002073
:10FD3800565555559023002000000000E4CB16418D
:10FD4800DB0F49C0DB0FC940E4CB16C1DB0FC93F4D
:10FD5800DB0F494092E741B99730083C15A82ABE05
:10FD6800F0EE476AF4EEC66AF1EE10FA36EEE57A7E
:10FD7800F6DC5FED0D6AB4EEE67AF1EE10FA40F1CA
:10FD880087835FED105A1FED106A01E0B0EE667AC6
:10FD9800B4EEC67AF1EE10FA77EE256AF6D41FEDC6
:10FDA800157AF4EEC76AF1EE10FA40F39F801FED62
:10FDB800187A77EE666A66EEA65A1FED1A5A1FED94
:10FDC8001A6A1FED1A7AA5EE856A26EEA55AA5EEDF
:10FDD800867AE5EE076AFFF768B83946C248F3F74E
:10FDE800B9F900283FF4C6AE84F8A77013F0ACFF49
:10FDF800FEF7DABDBD49BE4A0B91BE4D0121117017
:10FE08001B21B9480393F3F7A5F9039B00287FF456
:10FE1800F8ACDFF800B3B84FDBF80C203B68CBF840
:10FE280008309B1AC82B00F23683049B1F6807F41E
:10FE3800805733E5C1B2022940F2B78203297FF423
:10FE480049AF0E9B19460F9B002B08BF394603E7A5
:10FE580028F0010292B2424522803FF420AE0E20E3
:10FE680086F80090777086F802A002F077F8B4F868
:10FE7800008014E600210FE0627802EB820202EBB8
:10FE8800820202F2EE2292B20131994220F8022B4C
:10FE980004F102043FF402AD16F811201AB1022A47
:10FEA800EAD00288F0E7CAB2032AFAD87246EBE72A
:10FEB80000230393FFF7A8B9B2F5FA7FFEF679ADF0
:10FEC80094F8A630002B7EF474AD059B1B780121B5
:10FED80013EA010084F8A61000F0BE8214F0EEFBCD
:10FEE800049B1B6803F00403FEF767BD9FED837A4C
:10FEF800F4EEC76AF1EE10FA44BF9FED817A77EE0F
:10FF0800666A58E77F4A80491068B4F9A420C7692F
:10FF180081FB07018911FF17781A00F5FF407F3030
:10FF280082423EF734ADC91B0A4412B2A4F8A42099
:10FF3800FEF72DBDC8398A4240DA9AF8E0109A785F
:10FF480041FA06F3DB073FF554AB52420120099210
:10FF580002F0E4F87B1E099A162B00F21B81DFE8F9
:10FF680013F0BC01D201A301FB01E8010F027601E5
:10FF780061014A0133011C011901FB0109010F024A
:10FF880076016101F300DD00AC008B0194007E0076
:10FF98000126FEF737BC3A68DBF81C301344CBF86F
:10FFA8001830FFF7D5B908F021FC032240F6B83322
:10FFB8008BF82020CBF81C30FFF70EBA9AF8E03007
:10FFC8000122B24023EA020309F5FA728AF8E03006
:10FFD800A260FFF70EBB00214348F3F7BBF80028E7
:10FFE8007FF41DAB322384F8AA00A4F8AC30FFF7E5
:08FFF80016BB464B1B78002BE1
:020000040801F1
:100000003EF4DBAC9BF80330002B7EF4D6AC94F8C6
:10001000A7300133DBB2032B84F8A7307EF6CDACDA
:100020003D4B5B7813B9002E7EF4C7AC14F04AFB4D
:10003000FEF7BEBC002A0CBF012002208BE707237D
:100040001A4602EB8202174489F80030B9787878B2
:100050000AF0C2FC059B1E7806F00106FEF72CBED6
:1000600008231A46EDE7DAF8E400DFF8B48090F8E8
:10007000361098F8023011446429A8BF642121EA9F
:10008000E17180F83610002B40F0658307F0ACFC7E
:100090005FE5DAF8E400DFF8888090F8371098F828
:1000A00002301144FE29A8BFFE2121EAE17180F847
:1000B0003710002BEAD016201BF094FEDAF8E4008B
:1000C000E4E7DAF8E400DFF8588081781144C829C1
:1000D000A8BFC82121EAE171817098F80230002B95
:1000E000D4D014201BF07EFEDAF8E400CEE700BF87
:1000F00014540020D1590020923B0020506F002062
:100100006C570020DB0FC9BFDB0F49C0FC53002038
:10011000D34D621051510020205600209C510020E8
:10012000E84E0020DAF8E400DFF8A48641781144B4
:10013000C829A8BFC82121EAE171417098F80230AE
:10014000002BA3D013201BF04DFEDAF8E4009DE74E
:10015000DAF8E400DFF8788601781144C829A8BFEE
:10016000C82121EAE171017098F80230002B8DD08E
:1001700012201BF037FEDAF8E40087E7DFF850863C
:10018000089898F80230417911446429A8BF642185
:1001900021EAE1714171002B40F03E83DAF8E4007E
:1001A00074E7DAF8E400DFF82886017A98F802307C
:1001B0001144C829A8BFC82121EAE1710172002BAE
:1001C0003FF464AF0B201BF00DFEDAF8E4005DE7AE
:1001D000DAF8E400DFF8F885C17998F802301144C4
:1001E000C829A8BFC82121EAE171C171002B3FF4E1
:1001F0004DAF0A201BF0F6FDDAF8E40046E7DAF826
:10020000E400DFF8CC85817998F802301144C829E0
:10021000A8BFC82121EAE1718171002B3FF436AFFC
:1002200009201BF0DFFDDAF8E4002FE7DAF8E4003C
:10023000DFF89C85417998F802301144C829A8BF9D
:10024000C82121EAE1714171002B40F0C882112FD1
:100250007FF43BAF1AE7DAF8E400DFF87485017940
:1002600098F802301144C829A8BFC82121EAE171D9
:100270000171002B40F07382102F7FF457AF05E718
:100280000898DFF84C8541781144B1F5967FA8BFF6
:100290004FF4967121EAE171417098F80230002B19
:1002A0003FF47CAF15201BF09DFDDAF8E400EDE68D
:1002B0000899DFF81C850F791744642FA8BF6427BD
:1002C00027EAE7770F711BF0A7FD98F80230002BA3
:1002D0003FF464AF032039461BF084FDDAF8E400F4
:1002E000D4E60898DFF8E88401781144FA29A8BF19
:1002F000FA2121EAE171017098F80230002B3FF4F5
:100300004DAF01201BF06EFDDAF8E400BEE6089860
:10031000DFF8BC84817811446429A8BF642121EAF4
:10032000E171817098F80230002B3FF437AF022062
:100330001BF058FDDAF8E400A8E60898DFF890848E
:10034000C17998F80230114481F30801C171002B82
:100350003FF424AF05201BF045FDDAF8E40095E6F4
:10036000089BDFF86C84997998F80200114464299D
:10037000A8BF642121EAE1719971002840F0378219
:100380000D2F7FF4FDAE09E7DAF8E400DFF84084D2
:10039000C17898F802301144C829A8BFC82121EAC1
:1003A000E171C170002B40F0B3810F2F7FF4D4AE08
:1003B0006CE60E9954E435F912209978B2F5617F14
:1003C0004FF4966393FBF1F33ADB40F6330191422D
:1003D000A8BF11460C2FA1F5617191FBF3F100F05C
:1003E000FB80182F7FF4B5ABC9B2C8290B46A8BF54
:1003F000C823DAF8E400C27DDFB297423FF4A9AB2C
:100400009A1ADFF8CC83C77548BF0732D71098F81F
:1004100002300137FFB23BB9002F3FF49AAB3846A8
:1004200001F080FEFFF795BB18201BF0DBFCF3E723
:10043000B0EE677AFEF75BBDF0EE477AFEF76DBD72
:100440000C2F00F0E080182F7FF483AB00210B46C7
:10045000CFE7B0EE667A90E4C74A0292FFF74AB956
:10046000C64B1B6813F4003340F0D8801846C449CB
:100470000E5C0F2E00F10C0045D00133152BF7D187
:10048000049B1B68FA3A0021A4F8A42003F004039B
:1004900084F8A610FEF795BAF0EE476A83E4B94AED
:1004A000049B1F68138823F004031380012307F4BF
:1004B00080578BF82130FFF7F5B903231A46C0E5C2
:1004C00004231A46BDE505231A46BAE506231A4653
:1004D000B7E5AD4BAD491A684FF47A73B3FBF2F34D
:1004E000C3EB431203EB8202049B1B68D200A1F80A
:1004F000B42003F00403FEF764BA01231A46A0E512
:1005000002231A469DE5A24FD7F800E05800BEF13D
:10051000000F07D0C61801EB86069EF801E076783A
:100520007645ADD218449B4E9B4B01EB80010020D9
:10053000396030801860A3E7049B98491B680A6003
:1005400003F00403FEF73DBA0021BB2A109100F02E
:10055000C980B72A00F0C280BE2A00F0BD80BD2A43
:1005600000F0A380792A00F0EF807A2A00F0E5807D
:100570009E2A00F0DC809D2A00F0D280AE2A00F096
:100580007681AD2A00F06C81EF2A00F06381FD2AAC
:1005900000F05A81FB2A00F05181FE2A00F04881C8
:1005A000F72A00F03F817B2A7EF407AA4FF4FA6114
:1005B000022002F037FDFEF700BA794B002201203D
:1005C0007849794C0B60227001F0ACFD049B1B68EC
:1005D00003F00403FEF7F5B9CFB2734B09915B78D2
:1005E000BB423FF4B6AADFF8E881384602F0E6FDE8
:1005F00098F8023009991BB1C9B20C201BF0F2FB2C
:100600000137FFB208E700273946E6E7674B0122CA
:100610000220D5E7664B02220320D1E7654B1B7809
:10062000032B00F0D780034621E7049B624A1B6836
:100630004FF4C871118003F00403FEF7C2B90EF045
:1006400039FDF2F75BF90EF01DFDF5F7EBF801202F
:1006500001F068FD94F8A220FFF7BDBA94F8A82035
:10066000002A40F0D38094F8AA3083F0010384F884
:10067000AA30002B40F0C1800C2001F073FC049BD9
:100680001B6803F00403FEF79CB9002E3EF40EA98C
:100690004A4C94F8A130002B3EF43AA901F046FCF4
:1006A000002384F8A130FEF733B94FF6FE73444AB5
:1006B000D0899689014433449381D1810EF0FAFCAC
:1006C000F2F71CF90EF0DEFCF5F7ACF8012001F0B2
:1006D00029FDB4F8A420D3E60223E8E70B464FF641
:1006E000FE71E4E70B460221E1E7344C13F0EAFF28
:1006F000002384F8A130FEF70BB9002BC8D0314994
:10070000314A09684FF47A7000FB03131360BFE7A6
:100710000F2009921BF066FBDAF8E400099A44E620
:100720000021FF201DF020F894F8A22026E70120E8
:100730001DF01AF894F8A2201DE7244A137A43F01A
:1007400001031372FEF739B9204A137A23F001032B
:100750001372FEF732B917201BF044FB1EE5102080
:1007600009921BF03FFBDAF8E400099A84E50323C1
:100770000393FEF7F5BD00BF5C3E00205837002014
:100780005C100308C0510020D460002030650020B8
:10079000C02200201423002018230020A458002089
:1007A000CC4D0020F83A0020EC3A00201A4E0020F0
:1007B000684E002086510020127000202023002067
:1007C000045600206C570020A0580020783B0020E1
:1007D000E84E002001F0AAFBB4F9A42050E6112055
:1007E00009921BF0FFFADAF8E400099A2FE50D20D0
:1007F00009921BF0F7FA099AC2E50B2001F0B2FB4F
:10080000049B1B6803F00403FEF7DBB884F8A80020
:1008100084F8A910FEF7D5B80E201BF0E3FADAF839
:10082000E40033E40021042002F0FCFBFEF7C5B82D
:100830000021032002F0F6FBFEF7BFB800210220E2
:1008400002F0F0FBFEF7B9B80021012002F0EAFB4C
:10085000FEF7B3B80021084602F0E4FBFEF7ADB89E
:10086000FF2100201CF080FF94F8A2208CE60121DB
:1008700000201CF079FF94F8A22082E6084B19684A
:1008800061B130B45D68074C642202FB05F2B2FB33
:10089000F1F2228030BC002018605860704700BF21
:1008A00008240020BE390020704700BF6F4B1B7822
:1008B000002B3AD02DE9F0416D4B6E4D9B79AC6821
:1008C000A860013B82B0041B032B00F29C80DFE890
:1008D00003F04A0231291BF053FA002800F09B80F4
:1008E000654B66491B78B5F84220D1ED037AEA647E
:1008F000DB0700F1AA8002FB04F007EE900ADFEDAF
:10090000606A604BB8EEE77AD5ED127A5A60E7EE8E
:10091000267A1A60BDEEE77AC5ED127A85ED117A76
:1009200083ED027A02B0BDE8F081564A136053604D
:1009300093607047544B1B681801F3D5FF2018F0E3
:100940006BFE03780A2B88BF00214E4B9CBFB0F989
:100950000420B0F90610296588BF0A466A655A6006
:100960001A609960DEE7494A494BD279DFF8308155
:1009700033F81220B8F902304648B8F9001092B2A4
:1009800007EE902A40F6E44707FB02F6C3EB163366
:10099000B8EE670A4FF47A7606FB03F393FBF1F3A4
:1009A000AB61EFF7F7FED5F818E0D5ED047ADFED8F
:1009B000346AB8F90220334BB8F900C0C3F804E038
:1009C0000EFB04F007EE100AB8EEC77ABCEEC06A60
:1009D000E7EE267A8DED016ABDF80410C5ED047AC4
:1009E000BDEEE77A07FB01F7C2EB173706FB07F608
:1009F00083ED027A96FBFCF685ED037A6E611E604C
:100A000002B0BDE8F0811F4B00221A605A609A6064
:100A100002B0BDE8F0811C4B1B68DE067FF560AFBD
:100A2000154BB5F842201B78EA64D9077FF563AF10
:100A3000B5F94010184B00FB01F083FB0013C01701
:100A4000C0EBA3100244EA6455E7FDEEE77A134ECB
:100A500017EE900AA0F57A7101FB01F386FB0306FD
:100A6000D817C0EB26100844E2E700BFCE62002092
:100A70008C510020082400204D3C0020D062002032
:100A80002FE33E317C620020E4600020AC64002053
:100A9000C864002024240020D34D62101F85EB5130
:100AA000F4550020F0B53E4B5B79012B83B03DD06F
:100AB000022B0FD03B4B00221A805A803A4B1B78F6
:100AC000022B05D1374A394B5188128819805A8038
:100AD00003B0F0BD364B1B681B01EFD5FF2018F0AB
:100AE0009BFD03780A2B56D8B0F902203149D31761
:100AF00081FB0212C3EBA2039BB207EE903AB8EE61
:100B0000670A2D4C04F15C00A4F85A30EFF742FE5E
:100B1000FCEEC07A234AB4F85A30CDED017A538006
:100B2000BDF80430A4F858301380C7E7234A244B9B
:100B30009278214D33F81240A4B207EE904A05F1A5
:100B40008400B8EE670AEFF725FE1E4A15491078B3
:100B500096785378FCEEC07A00EB4010CDED017A28
:100B6000BDF8042044F6FB77C3EB033300FB0272AD
:100B700000FB0474B2FBF3F2B4FBF3F3B2FBF6F246
:100B8000B3FBF6F392B29BB2A5F88020A5F88230B1
:100B90000A804B8092E79FED0C0A0023B1E700BF6B
:100BA0008C51002088620020F8610020FC61002048
:100BB000E46000206766666608240020AC640020BC
:100BC000C8640020B74D002000000000F8B53422B2
:100BD000044600211FF07DFA142300225220A37046
:100BE0000E4BA272022701221E261F25642184F8C3
:100BF0003200C4F80330C4F80B30C4F81330C4F822
:100C00001B30C4F82330C4F82B30A77684F8226058
:100C100084F82A502186A2742280F8BD05040500BC
:100C20002DE9F0432F4DD5F8A83083B01BB195F8CE
:100C3000AC30022B02D003B0BDE8F0834FF02008A7
:100C40004046294C05F1B009012655271BF06CF8E8
:100C5000A0B199F800300BB9217891B908F10108D9
:100C60005FFA88F8B8F1230F04F1010409F10109D2
:100C7000E1D040461BF058F80028EAD189F800007E
:100C8000ECE7D5F8A80050B30DF1080EAA220EF833
:100C9000052D8DF802108DF800708DF801608DF82B
:100CA0000430694655225340082213F0800F02F1A8
:100CB000FF324FEA430318BF83F0310312F0FF0203
:100CC000DBB2F2D1714502D011F8012FEBE7AA2275
:100CD00069468DF803308DF804200CF061F989F82D
:100CE0000060BBE708240020680A03081F4B18783F
:100CF000002839D01E4A1389FBB11E4A9FED1E6A97
:100D0000D2ED026A07EE903AF8EEE66AF8EE677AFC
:100D100007EE103A77EEE66AB8EEC77A66EE866AB4
:100D2000C6EE877AFDEEE77A17EE900A6428A8BF30
:100D3000642020EAE070C0B2704710B40F4B5478C2
:100D40001B88117804FB1032091B642300FB01F09F
:100D500003FB02F3B3FBF0F06428A8BF64205DF846
:100D6000044B20EAE070C0B2704700BFCE620020A2
:100D70008C5100207C6200200000C8428862002064
:100D8000F8B52D4D2D4968792D4C2E4B2E4E042251
:100D900064270A7001284FF0000184F8B32084F81A
:100DA000B970A4F8B410A4F8B61084F8B810C4F858
:100DB000BC1031701980598021D0022810D0A97937
:100DC000224A00230129136084F8C03053609360E5
:100DD00023D0022912D11E4A636453609360F8BD88
:100DE000282204F158001FF074F94CF250319FEDA5
:100DF000190A04F15C00F2F753F9E0E7F8BD282284
:100E000004F180001FF065F94CF250319FED110A9A
:100E100004F18400F2F744F9D1E70F4AE36053602C
:100E20009360D3609FED0D0A02F110004CF2503137
:100E3000BDE8F840F2F734B98C510020865100200B
:100E40000824002088620020CE6200207C620020FE
:100E50004C240020CDCCCC3D14240020CDCCCC3E65
:100E60002DE9F04F794D81B0F0F744F8D5F8C8403E
:100E70000022C5F8C420002C00F0A580237D052B9E
:100E8000074617D9216A23690B44C31A9342B8BF96
:100E900005F1C8010ADBD5E0137D052B0AD9136AD9
:100EA00012691344FB1A002B80F2CC8051F8042FF6
:100EB000002AF1D14FF0010B0023B9461E46C5F8B8
:100EC000C43098469A46274623E07A6A39693B7DC2
:100ED000A9EB0204B4FBF1F40134A4B213FB04F354
:100EE000013301369BB2B6B23C83FB82984506D2F1
:100EF000BBF1000F01D1012C5FD99846BA46D5F855
:100F0000C430013305EB8302C5F8C430D2F8C87091
:100F100047B3BB68C3B1FC8A002CD6D1396A4846B6
:100F2000A9EB01019847D0B195F81831002B52D1A7
:100F30003B7DC7F82490013601334FF00102B6B271
:100F40003A83FB820124D1E73B6A3A69A9EB0304A7
:100F5000B4FBF2F4A4B23C8334BBFB8AC6E73C8307
:100F6000FB8AC3E72B686A683949013316443C465B
:100F700085E848004F46C1F800A0BAF1000F27D01D
:100F8000DAF8203095F81821AAF81640FB1ACAF8AA
:100F90001C30CAF82090002A35D1DAF80C304846C7
:100FA00001B0BDE8F04F18473B7D13FB04F301335C
:100FB00001369BB2B6B2FB8298E73A7D062A04BF9F
:100FC0009846BA469BE72B68214A01332B60146090
:100FD00001B0BDE8F08FEFF78DFF1E4B1E4A1F4C8E
:100FE00011681A68A0EB090002EB000E2268C3F832
:100FF00000E09042A1EB5111014438BF1046164A5F
:101000002060116094E7EFF775FFDAF80C300446C2
:101010009847EFF76FFFDAF82C20DAF82830DAF883
:101020003010001B9042A3EB53130344014438BF1C
:101030001046CAF82830CAF83010CAF82C0001B09F
:10104000BDE8F08F4FF0000B36E700BF082400200A
:10105000FC530020B0390020B4390020B8390020FA
:10106000F0B43423184F194A03FB00F3D2F81C6183
:10107000FC58FD18002E6B684B600C600DDDD2F83B
:10108000C8309D421DD0C832002303E052F8044FFF
:10109000A54216D00133B342F8D10022342303FB1A
:1010A00000700A720369CB60037D4B72836AC56A64
:1010B000046BC2690A615B094D618C61CB61F0BC54
:1010C00070470122EAE700BF0C100020082400202E
:1010D0002DE9F041244ED6F81C51122D27DC002DAD
:1010E0003DDDD6F8C830984221D005F1804106F1A7
:1010F000C807013907EB81013B4603E053F8042F91
:10110000904214D08B42F9D1D6F8C8409CB1237DCF
:10111000017D8B420ED3154A002405E052F8043FAE
:101120004BB11B7D8B4206D30134A542F6DA002079
:10113000BDE8F08100248046601C80002A1B011F4E
:1011400006EB840439443844920001351EF0A7FFB1
:10115000C4F8C880C6F81C510120BDE8F081E6D172
:1011600006F1C807D0E700BF08240020D0240020E3
:10117000142830D0122807D8184B342202FB003034
:1011800019B1C3680BB1A3E7704770B5144DD5F81A
:101190001C41002C0FDDD5F8C83098420CD005F169
:1011A000C8063346002203E053F8041F884206D0E5
:1011B0000132A242F8D170BD002205F1C8069000AC
:1011C000011DA21A920031443044013C1EF067FF19
:1011D000C5F81C4170BD034B1868D1E70C10002006
:1011E00008240020FC530020F0B50D4685B00646CB
:1011F0000068EFF7FFFF95E81800E41A0023039357
:1012000024238DF808304D238DF80930B5F90A30C4
:10121000FF2C2246A8BFFF2201333DD02B7B002BA1
:101220000CBF3E233C238DF80A30FE2C2B898DF811
:101230000B208DF80C3031DD23128DF80D408DF828
:101240000E3007273A4602A93068EFF7D9FF02AB04
:10125000DA190DF10B0100238A4221D1002C8DF8FF
:1012600007300CDD224629683068EFF7C9FF2B688C
:101270009DF807201919994216D18DF807200122EF
:101280000DF107013068EFF7BBFF3068EFF7ACFFF7
:1012900004F1090005B0F0BD2123C4E70527D1E71B
:1012A00011F8010B4340D7E713F8010B4240E2E786
:1012B00008B50E4B1978012913D00DD3022902D19C
:1012C0000020EFF7DBFFEFF715FE094B00F5F420E8
:1012D00000F59070186008BD00210846F1F71EF86F
:1012E000F1E70020F1F71AF8EDE700BF14700020D5
:1012F000187000202DE9F04F83B0484C484F019002
:10130000019803685B699847002840F08380DFF804
:1013100018914448D9F80430DFF810E1C3F308030A
:101320004FF00A0A4FF0100C4FF47A75002B3BD1A6
:10133000EFF31183002B37D10168A26800BF036867
:101340009942F9D1DEF8006005FB06F39B1AB3FB66
:10135000F6F305FB013101260091D9F80430C3F3FF
:101360000803002B3BD1EFF31183002B37D1036827
:10137000A16800BF02689342F9D1DEF800B005FB16
:101380000BF2521AB2FBFBF205FB0323009A9B1AE5
:10139000B3F57A7FE1D3BAF1010AB1D0D9F80430BC
:1013A000C3F30803002BC3D0EFF311828CF3128830
:1013B000A6682368D90302D501233B60A6680368A9
:1013C0003968D2B282F31188DEF80020194405FB97
:1013D00002F39B1BB3FBF2F305FB0131BBE7EFF319
:1013E00011888CF31288A1682368DB0344BF3E6038
:1013F000A16803683A685FFA88F888F31188DEF814
:1014000000801A4405FB08F35B1AB3FBF8F305FBF5
:101410000233BBE703B0BDE8F08F00BF10E000E08F
:10142000685700206C57002000ED00E07057002046
:10143000144B1A6890420FD09A68904218D01A69DB
:10144000904217D09A69904216D01A6A904215D0ED
:101450009A6A904214D07047002110B403EBC10483
:101460000022C262A28043F831205DF8044B70472D
:101470000121F2E70221F0E70321EEE70421ECE786
:101480000521EAE7083E0020F8B50A4E054600248B
:10149000A359AB4204EB060707D12846FFF7C8FF64
:1014A000CC22002138461EF014FECC34B4F5197F4E
:1014B000EED1F8BDA06B00202DE9F04F8F4D95F9CE
:1014C000064093B084429DF870A09DF874901CD0A3
:1014D00095F90E40844200F0A78395F916408442A6
:1014E00000F0B58395F91E40844200F0B38395F96E
:1014F0002640844200F0DC8395F92E40844200F0BF
:10150000DA83002013B0BDE8F08F4FF0000B4FEAF4
:10151000CB06AC19A488002CF3D11F460192884653
:101520001F28EED801A353F820F000BFB11901081D
:10153000B1190108B11901080315010803150108C3
:101540000315010803150108031501080315010817
:101550000315010803150108031501080315010807
:1015600003150108031501080315010803150108F7
:101570000315010803150108031501085518010892
:1015800003150108031501080315010803150108D7
:1015900003150108031501080315010803150108C7
:1015A000031501081D170108AD150108544AD37D24
:1015B000D47A0393184618F051FF0590204618F08E
:1015C0004DFF039B02901846F0F7ECF9049020467B
:1015D000F0F7E8F919F008030393029A00F0E482A7
:1015E000002A8ED0D37959078BD4464CC4F8B8233F
:1015F000C4F8B403C4F8B00318B10B210C238171F3
:10160000C3710AF0020302933F4B404984F885A35B
:1016100003F5807E1046019AC4F8AC23AEF58072C3
:101620004FF0000A4FF48073C4F894230122C4F8E9
:101630008C33C4F89033C4F898E3C4F8801384F86A
:10164000D0253946C4F8887384F88693C4F8A0A3DB
:10165000C4F89CA3C4F8A8A3C4F8A4A3C4F8CCA558
:1016600084F8C4A584F8C5A5019213F0C7F809F061
:101670000101D4F8B80315F04FFC029B244925481A
:10168000C4F8D415C4F8D8A5C4F8DC05D4F8B81348
:10169000002B00F0B282D4F8BC03002800F0AD8229
:1016A0000B6802689A4200F0A882019A84F8D1255A
:1016B000394613F0A3F8144BD4F8BC0303F50571B5
:1016C00012F0F2F9104BD4F8B803524603F5077143
:1016D000F3F7C6FD039B104C002B00F0A8822046B8
:1016E00013F0C0F80C481F242E440471A6F804809F
:1016F00045F83B0013B0BDE8F08F00BF083E002066
:10170000383E002008240020C8270020940A03083F
:10171000B5480208893C020888270020904A937D3A
:10172000947A0393184618F099FE0590204618F015
:1017300095FE039B02901846F0F734F9049020467A
:10174000F0F730F919F008030393029A00F00A82C7
:10175000002A3FF4D6AED37959073FF5D2AE814C7B
:10176000C4F85821C4F85401C4F8500110B10B2337
:101770008371C3710AF0020302937B4B7B4984F8A7
:1017800025A11046019AC4F84C214FF0000A4FF4ED
:10179000807203F5807EC4F83431C4F82C21C4F87B
:1017A0003021C4F838E1C4F82011C4F82871394652
:1017B00084F82691C4F840A1C4F83CA1C4F848A11B
:1017C000C4F844A184F870A3C4F86CA384F864A39B
:1017D00084F865A3019313F011F809F00101D4F81E
:1017E000580115F099FB029B6149624AC4F87C13C9
:1017F000C4F878A3C4F87423D4F85811002B00F06F
:10180000F281D4F85C01002800F0ED810A680368D9
:10181000934200F0E881012284F87123394612F0E6
:10182000EDFF019BD4F85C0103F5057112F03CF962
:10183000019BD4F85801524603F50771F3F710FDE8
:10184000039B002B00F0FB814B4813F00BF81E2488
:10185000494849E7494C4A48A369424F43F00103CC
:10186000A3611121F0F74AFB4548F0F703FDC820BA
:10187000EFF7A2FA4248F0F703FD636943F400333F
:10188000636103234FF000094FF4C05207A94FF0E2
:1018900090408DF821304FF0020307928DF82030F0
:1018A0008DF822908DF8239009F0EAFE4FF09043D6
:1018B0003448596A21F470415962596A41F46041CF
:1018C0005962596A21F470215962596A4FF4802291
:1018D00041F4602159624FF0010A0260122108238D
:1018E00007F5C560C7F8281687F82D3687F82EA6A5
:1018F00011F01AFC244B2548C3F80090E369244AF0
:10190000244943F40003E361234C036810604FF063
:10191000020222480A722160214901609847214B46
:101920002149D96007A84FF0020314248DF81D3017
:101930008DF81E908DF81FA08DF81C4014F07CFED1
:101940002A2307A88DF81C308DF81DA08DF81E9055
:1019500014F096FE154BC7F8E03507F5BC60C3E6FA
:10196000383E00200824002068250020940A03083F
:10197000893C0208B54802082825002000100240D2
:10198000185C002014040140D8004242D81B0020FB
:10199000A45A0020386B00202C6B0020945A0020A1
:1019A0008400002000ED00E00005FA056C0A030841
:1019B000C4B24B46204652463946F1F715FF03465E
:1019C00000283FF49EADC06C83F805A083F8069014
:1019D0000168019ADA6221F0010100224FF0010E44
:1019E0009F6083F850E01A62DA619A625A6201607D
:1019F00019F00401079700F00A814FF48052089211
:101A000019F0020240F0728109924FF480620021C5
:101A10001AF001090A920C9140F00281CDF82C9045
:101A200008221AF0020707A918BF0B92019314F0BD
:101A3000A7FD019B5A79987902F00201002915BF90
:101A40004FF440314FF480314FF4003E4FF0000E20
:101A500012F0010FDA6C08BF7146D2F804E010F002
:101A6000010F14BF41EA0E012EEA01015160916895
:101A700000074CBF41F0080121F008019160116896
:101A800041F001011160B9F1000F33D0196B002949
:101A900000F01E8107A8019314F09CFC019B9A6C36
:101AA000D3F80CC05969186B07924FF4805210920A
:101AB00000220891119280210B920D920E920992B0
:101AC00020220F92ADF828C00C9114F0B1FC019BBC
:101AD00007A9186B14F08CFC019B196BDA6C086871
:101AE00040F001000860906840F040009060496854
:101AF00089B21964002F2FD0596B002900F0EF80B4
:101B000007A8019314F066FC019B596C1A690791B0
:101B10004FF480510027586B1091ADF82820802198
:101B2000102209920C9111970B970D970E970F9712
:101B300014F07EFC019B07A9586B14F059FC019B23
:101B4000596BDA6C086840F0020008604F604F6023
:101B5000916841F080019160116841F001011846DF
:101B60001160C1E51AF0010C16D0059900293FF467
:101B7000C8ACC9794B073FF5C4AC5F49049BC1F8B9
:101B80005031059BC1F85831049B2BB14FF00C0E1E
:101B90000B2183F806E0D9711AF0020302935CD19D
:101BA000554CD4F85821E8E51AF0010E13D00599E8
:101BB00000293FF4A6ACC9794B073FF5A2AC4E49CA
:101BC000049BC1F8B033059BC1F8B833049B13B133
:101BD0000C219971D9711AF00203029352D1464C2B
:101BE000D4F8B82310E5454A0023084684F8713339
:101BF00002F10801F3F734FB22E6414A00230846CC
